:020000040800F2
:1000000030B1012059030008B74C000845420008F0
:10001000B54C0008591A0008E55700080000000018
:10002000000000000000000000000000990200082D
:10003000C91B000800000000F5020008494F000835
:1000400073030008730300087303000873030008B8
:1000500073030008730300087303000873030008A8
:100060007303000873030008730300087303000898
:100070007303000873030008730300085D1A000887
:1000800073030008730300087303000800000000F6
:1000900000000000000000000000000073030008E2
:1000A0007303000873030008095000087303000875
:1000B0007303000873030008730300087303000848
:1000C0007303000873030008730300087303000838
:1000D00073030008730300087303000800000000A6
:1000E0007303000873030008730300080000000096
:1000F0000000000000000000000000007303000882
:100100000000000073030008730300087303000875
:1001100000000000000000000000000000000000DF
:10012000691A0008E91A000873030008730300083D
:100130007303000800000000000000000000000041
:100140000000000000000000000000007303000831
:1001500073030008F51A000873030008AD57000880
:100160007303000873030008000000000000000093
:10017000000000000000000000000000000000007F
:1001800000000000730300080000000000000000F1
:10019000730300087303000800F002F800F06DF824
:1001A0000AA090E8000C82448344AAF10107DA45D2
:1001B00001D100F062F8AFF2090EBAE80F0013F0B7
:1001C000010F18BFFB1A43F001031847282303004F
:1001D000482303000A444FF0000C10F8013B13F0D1
:1001E000070408BF10F8014B1D1108BF10F8015B90
:1001F000641E05D010F8016B641E01F8016BF9D183
:1002000013F0080F1EBF10F8014BAD1C0C1B09D1D9
:100210006D1E58BF01F801CBFAD505E014F8016B4B
:1002200001F8016B6D1EF9D59142D6D370470000DD
:100230000023002400250026103A28BF78C1FBD8EF
:10024000520728BF30C148BF0B60704766292AF0AB
:100250008686002070471FB52AF077FE9DE80300D0
:1002600000F0ECFA00F074FD0400002000212AF0F8
:10027000ABF9E0601FBD10B510BD00F087FE114660
:10028000FFF7E9FF21F00AFD00F0A5FE03B4FFF738
:10029000F2FF03BC00F016FF2C4B19680868B0E8A9
:1002A000F04F80F30988BFF36F8F4FF0000080F3A9
:1002B000118870470000000008480068006880F35B
:1002C00008884FF0000080F3148862B661B6BFF36F
:1002D0004F8FBFF36F8F00DF00BF00BF08ED00E05E
:1002E000DFF80C00016841F470010160704700BF45
:1002F00088ED00E0EFF30980BFF36F8F134B1A68AE
:100300001EF0100F08BF20ED108A20E9F04F10609A
:1003100009B44FF0500080F31188BFF34F8FBFF343
:100320006F8F29F09FFA4FF0000080F3118809BC0D
:1003300019680868B0E8F04F1EF0100F08BFB0EC65
:10034000108A80F30988BFF36F8F7047A4000020E4
:10035000EFF30580704700000948804709480047CF
:10036000FEE7FEE7FEE7FEE7FEE7FEE7FEE7FEE765
:10037000FEE7FEE704480549054A064B70470000C2
:10038000F94F00089901000830AB012030B101207D
:1003900030AD012030AD012070B5064600F032FAD4
:1003A000056806F10B0020F00704B4429CBF002052
:1003B00070BD2B466A68BAB11068A04210D304F130
:1003C000080188423CBF5068586007D35168101933
:1003D00041601168091B016058601460101D70BDF8
:1003E00013465268002AE7D12146284600F012FA47
:1003F0000028DED170BD70B50446051F00F002FA7A
:100400000068002C14BF446870BD002C18BFAC42BB
:100410003CBF20466468F8D301680A18AA4218BF96
:10042000456003D12A6805461144016028684119D6
:10043000A1421CBF6C6070BD61686960216808449E
:10044000286070BD53EA020C00F069802DE9F04B82
:100450004FF00006002B1FBFB3FA83F503FA05F433
:1004600024FA05F65E4012BF1643B2FA82F502FA8C
:1004700005F4C5F120051EBF22FA05FC44EA0C0470
:10048000203556EA044C4FEA144418BF641C4FF060
:1004900000084FF00009904271EB030C39D300299A
:1004A00019BFB1FA81F701FA07F6B0FA80F700FA3E
:1004B00007F6C7F120071EBF20FA07FC46EA0C0624
:1004C0002037B6FBF4FCA7EB0507103F07F01F0B26
:1004D000CBF120060CFA0BFB2CFA06F644BFB34610
:1004E0000026202FA4BF5E464FF0000B5BEA060CEF
:1004F00008BF4FF0010B19EB0B09ABFB027C48EB7B
:100500000608C01B06FB02CC0BFB03CC71EB0C01F5
:10051000C1E70B46024641464846BDE8F08B13B59D
:100520004FF000004FF00001AFF30080BDE81C4029
:10053000704710B54C1084EA530404D54042C1F111
:10054000000138BF491E1B4204D55242C3F10003CB
:1005500038BF5B1EFFF776FF14F0804F04D0404297
:10056000C1F1000138BF491E14F0004F04D05242BF
:10057000C3F1000338BF5B1E10BD00000FB41CB5F3
:10058000074B06AA7B4469460090059800F0A1FB42
:100590000020694600F0B0FB1CBC5DF814FB0000B5
:1005A000710700002DE9F0474FF0000A8946044624
:1005B000C0F820A02046E1688847002876D025288A
:1005C00006D0D4E901219047206A401C2062F1E75F
:1005D000E168204600258847C4F81CA0064600278D
:1005E000C4F818A02A2E09D0304605F0D0F938B347
:1005F00004EB8708303EC8F8186019E059F8041B6E
:10060000204604EB87029161E1688847012F064686
:1006100018D1E069002820DA25F020051DE0D8F87F
:10062000180000EB800006EB40003038C8F81800D6
:100630002046E1688847064605F0A9F90028EED172
:10064000012F0AD02E2E08D12046E16888477F1C52
:100650000646022F45F02005C4DBA069002803DA16
:10066000404245F00105A061E80701D025F01005E2
:10067000B6B1A6F14100192802D8203645F400652C
:100680004A463146204625604D46FFF7DFFD58B10A
:10069000012806D0ED1D25F0070000F1080989E7C3
:1006A00004E005F1040985E730468AE7206ABDE8E1
:1006B000F087032A40F2308010F0030C00F0158020
:1006C00011F8013BBCF1020F624498BF11F801CB55
:1006D00000F8013B38BF11F8013BA2F1040298BFBA
:1006E00000F801CB38BF00F8013B11F0030300F024
:1006F0002580083AC0F0088051F8043B083A51F8C8
:1007000004CBA0E80810F5E7121D5CBF51F8043BCC
:1007100040F8043BAFF30080D20724BF11F8013B3F
:1007200011F801CB48BF11F8012B24BF00F8013BA1
:1007300000F801CB48BF00F8012B704710B5203AF4
:10074000C0F00B80B1E81850203AA0E81850B1E88A
:100750001850A0E81850BFF4F5AF5FEA027C24BF40
:10076000B1E81850A0E8185044BF18C918C0BDE837
:1007700010405FEA827C24BF51F8043B40F8043B00
:1007800008BF7047D20728BF31F8023B48BF11F8B5
:10079000012B28BF20F8023B48BF00F8012B70470F
:1007A00002F0FF0343EA032242EA024200F0ABBA3E
:1007B0004FF0000200B5134694469646203922BFFA
:1007C000A0E80C50A0E80C50B1F12001BFF4F7AF45
:1007D000090728BFA0E80C5048BF0CC05DF804EB27
:1007E000890028BF40F8042B08BF704748BF20F895
:1007F000022B11F0804F18BF00F8012B7047704793
:100800007047704700487047D4AA0120704770476E
:100810007047704738B504460A4600206946AFF372
:100820000080002808BF38BD02460099204600F02D
:1008300093FA012038BD012000F0A0BBF8B5AFF35A
:100840000080054600200C46102000BF0646A8196F
:10085000A0420DD9324669460020AFF30080070060
:1008600008BF00F08BFB0098A04218BF0546C419D2
:10087000FFF7C8FF05600746F01D20F00700461986
:10088000284600F00AF8B44208BFF8BDA21B314662
:100890003868BDE8F84000F05FBA00210160C0E9A7
:1008A000011070471020704770472DE9FF4F0C462C
:1008B0001E464FF0FF378BB0D2E90001DDF86080B3
:1008C0000A908A46C1F30A5505B93D4600210846FB
:1008D0004FF00000BAF1000F00F4400005DA00EB21
:1008E00080004FF4400101EA50004FEA9059B9F1FD
:1008F000010F00DDB9460A9850EA4A000ED044F6CE
:100900001050A5F2FF3545432F14B8F1000F1ED04B
:100910007542291E1EDDC9F100021CE0B8F1010F6D
:100920004FF0000001D0302103E0F24305E02154F4
:10093000401CB042FBDB30460022002121540B99C1
:10094000C1F80880C1E900200FB0BDE8F08FBD1BE1
:100950006D1CDEE74A4600DA694206A800F09CFA00
:1009600006AB93E8070003AB83E8070050460A99FB
:1009700000F0CEFB8DE80700A0F500501F38009076
:100980000398002D0ADD42F21F014A460844002365
:1009900003A90390684600F037FE09E0A0F5005077
:1009A0004A461F38002303A90390684600F041FE21
:1009B0008DE807000004000C03D04FF0FF30410821
:1009C00000E01046B8F1000F03D000220092154657
:1009D0001EE0751E05D400F0D9F9303262556D1E47
:1009E000F9D5B3460122084302D000227F1C04E05F
:1009F0002078302801D100227F1E002A099784D058
:100A00001DE0112D07DA00F0C1F9303262556D1C7E
:100A100050EA0102F5D1084302D00098C8B10EE0B7
:100A20000021681E05E0235C625C63542254401E72
:100A3000491C8142F7DBAB46A81B401E09900020F1
:100A400004F80B000B98099AC0F80880C0E9002B45
:100A50007AE711264FF0000857E72DE9F04F884656
:100A60000446D21D22F0070191B0D1E90001CDE981
:100A70000A0104F0E9FE02460B98C00F01D02D20B8
:100A800007E02068810701D52B2002E0202101EA40
:100A9000C000032A099001D0072A05DB034641461E
:100AA000204600F0B9F90BE12078800601D5E06915
:100AB00000E00620B8F1650F814606D0B8F1660F58
:100AC00018D0B8F1670F70D131E00020B9F1110FE3
:100AD000009001DB112301E009F101030AAA01A939
:100AE0000CA8FFF7E2FEDDE90C70002609F1010514
:100AF000834647E001204B4600904FF000470AAA8A
:100B000001A90CA8FFF7D1FEDDE90DB00C995D46F7
:100B1000002610B909F101000D18B9EB050003D446
:100B2000C0F1FF3609F10105A5EB09002BE0B9F191
:100B3000010F01DA4FF001090020B9F1110F009007
:100B4000484601DD112300E003460AAA01A90CA8CA
:100B5000FFF7ABFEDDE90C704D460026834620789A
:100B600000070AD4AB4500DA5D4601A8012D04DD7B
:100B7000411911F8011C302907D04F4502DA17F14D
:100B8000040F04DA012082460FE06D1EEEE7002F0D
:100B900002DCED1B3E4403E0781CA84200DD7D1C16
:100BA000B81B00F1010A4FF000472078000703D47A
:100BB000AA4501DB4FF0FF3A0021B7F1004F0DF1DC
:100BC00043088DF8431024D002202B23002F01DA94
:100BD0007F422D230A21021EA0F1010000DC5FB13B
:100BE00097FBF1FC97FBF1F201FB1C7C17460CF123
:100BF000300C08F801CDEEE7A8F101000370218860
:100C0000090501D5452100E06521A0F1010800F8A2
:100C1000011C09980FA9A1EB0807FF1D00B10120D5
:100C2000411901EBEA70A1693844081A401EA0611D
:100C30002078C00602D42046AFF30080099828B17E
:100C4000D4E901219047206A401C20622078C00628
:100C500022D52046AFF300801EE0002E04DBB34512
:100C600002DD01A8805D00E03020D4E90121904739
:100C7000206A401C2062761CAAF101005FEA000A8B
:100C80000AD100F065F8C0680168405CD4E9012130
:100C90009047206A401C2062281EA5F10105DCDC7B
:100CA00007E0D4E9012118F8010B9047206A401CA5
:100CB0002062381EA7F10107F3DC2046AFF3008065
:100CC000032011B041E6000001694A1C0261087866
:100CD000704700B58FB0CDE901310021059105497C
:100CE0007944CDE9031011466846FFF75BFC0FB06D
:100CF00000BD0000E5FFFFFF0A6802F8010B0A6073
:100D000070474FF000020429C0F0128010F0030C6D
:100D10003FF450ADCCF1040CBCF1020F18BF00F849
:100D2000012BA8BF20F8022BA1EB0C01FFF742BD5D
:100D30005FEAC17C24BF00F8012B00F8012B48BFFB
:100D400000F8012B7047000000487047CCAA012032
:100D500000487047ECAA0120034640688C460028F2
:100D600018BF88423CBF03464068F8D3186818444F
:100D7000884207D00CF1030020F00700001D411A43
:100D8000521A0146081D0A60FFF735BB30B5B0F1B5
:100D90000A024FEA900E71F100034EEA817EB0EB39
:100DA0000E0061EB91014FEA101E4EEA017E10EB3E
:100DB0000E0041EB11114FEA102E4EEA016E10EBBE
:100DC0000E0041EB11214FEA104E4EEA014E10EB9E
:100DD0000E0041EB1141401841F100014FEAD000F3
:100DE00040EA41704FEAD10110EB80054FEA8104DF
:100DF00044EA907444EB01046D1944EB0404521B63
:100E0000A3414FF0000348BF0A3200D530BD401C5B
:100E100041F1000130BD00002DE9F0411F460446BC
:100E200003260168072A01F4006004DB08B116A557
:100E300005E016A503E008B115A500E015A521F011
:100E400010002060A069C01EA0610FB1401EA0610B
:100E50002046AFF300804FB1D4E9012138469047D6
:100E6000206A401C2062C01C206206E0206AFAE76B
:100E7000D4E9012115F8010B9047761EF8D22046DF
:100E8000AFF30080BDE8F0814E414E006E616E0010
:100E9000494E4600696E66002DE9F04781461646C8
:100EA0008AB0354878440DC88DE80D003248784442
:100EB000801C03AC0DC884E80D0041F69B3008444B
:100EC000372190FBF1F290FBF1F5A5F1800501FBD4
:100ED00012041B3C02D56442012000E00020DFF830
:100EE00098A080460027FA44AAF1BE0A0EE0E00767
:100EF0000AD03246684607EB470101230AEB81011D
:100F000000F097FB8DE8070064107F1C002CEED1E9
:100F1000194F7F44AE3F19E0E80715D007EB0410E6
:100F20000DF1180A90E80E008AE80E00C068F04241
:100F300001D1981908903246012306A903A800F0B0
:100F400078FB03AB83E807006D10641C002DE3D130
:100F50004FF0010332466946B8F1000F03A802D0F2
:100F600000F052FB01E000F064FBC9E90001C9F8A0
:100F700008200AB0BDE8F087140F030010B500F098
:100F800039F8BDE8104000F02FB870477546FFF7FC
:100F9000DBFEAE4605006946534620F00700854655
:100FA00018B020B5FFF7E6F9BDE820404FF0000685
:100FB0004FF000074FF000084FF0000B21F0070141
:100FC000AC46ACE8C009ACE8C009ACE8C009ACE884
:100FD000C0098D46704710B50446AFF30080204627
:100FE000BDE81040FFF752B9002801D000F06AB800
:100FF0007047000010B5012805D0002103A000F0C3
:1010000067F8012010BD09A1F8E7000053494752D5
:10101000544D454D3A204F7574206F6620686561C8
:1010200070206D656D6F7279000000003A20486590
:101030006170206D656D6F727920636F727275706B
:10104000746564004FF0013C50F8042B51F8043BE8
:101050009A4221D1A2EB0C03934313EACC1317D18C
:1010600050F8042B51F8043B9A4215D1A2EB0C0323
:10107000934313EACC130BD150F8042B51F8043BE3
:101080009A4209D1A2EB0C03934313EACC13DBD0B1
:101090004FF00000704700BFD01A01BAB1FA81F1D9
:1010A00001F0180122FA01F0CB40C1F12001DBB2BE
:1010B000C0B2C01A2CFA01F3D11A914311EAC3113C
:1010C000E6D1704701491820ABBEFEE726000200BA
:1010D00070B505460C460A2000E06D1C00F011F8C2
:1010E00035B128780028F8D102E0641C00F009F836
:1010F00014B120780028F8D1BDE870400A20AFF381
:10110000008008B569468DF800000320ABBE08BD1D
:101110005FEA400C08BF91F0000F4FEA8C234FEAC2
:10112000C12243EA51514FEA1C5018BF00F5F0406C
:101130004FEA300018BF41F000415FEA6C5C00F0FC
:101140002980BCF1FF3F08BF40F080407047130C7E
:1011500006BF12044FF0100C4FF0000C130E04BF2A
:1011600012020CF1080C130F04BF12010CF1040C55
:10117000930F04BF92000CF1020CD30F04BF520076
:101180000CF1010C11464FF00002A0F11F00A0EB82
:101190000C00704711F0004F08BF704731F000415C
:1011A0003FF4D5AF0B0C06BF09044FF0100C4FF005
:1011B000000C0B0E04BF09020CF1080C0B0F04BF4E
:1011C00009010CF1040C8B0F04BF89000CF1020C17
:1011D000CB0F04BF49000CF1010CCCF12003A0EBB4
:1011E0000C0022FA03F302FA0CF241EA030100F1C7
:1011F0000100704720F07F4C80EA030023F07F4716
:10120000ACEB070303F57C5300F0004003F1FF0350
:101210002DE980494FEA154B09B44FEA144325EAFA
:101220000B4E24EA03480FF2042606EB1327490865
:101230003E785FEA320203FB0667C7F5000707FB4B
:1012400006F64FEA54374FEAD64606F1020607FB88
:10125000066CCCF1005C4FEA1C472CEA074C07FBFC
:1012600006F40CFB06F504EB15464FEA961634BF60
:1012700000204FF000404FEAD13706FB07FC4FEA51
:101280001C4C0CFB0BF7D21B03FB0CF761EB0701AB
:101290000CFB0EF7B0EB074072EB17420CFB08F7A4
:1012A00034BFA2EB0742B2EB074261EB17414FEAB2
:1012B0000C444FEA910706FB07FC4FEA1C4C0CFB61
:1012C0000BF7B0EBC74072EB573203FB0CF734BFA0
:1012D000A2EBC742B2EBC74261EB57310CFB0EF7F2
:1012E000B0EBC70072EB57720CFB08F734BFA2EBF0
:1012F000C702B2EBC70261EB5771039F4FEA8161EE
:1013000041EA921104EBCC044FEAD1374FEA8262F2
:1013100006FB07FC42EA90124FEA80604FEA1C4C41
:101320000CFB0BF7D21B03FB0CF761EB07010CFB6B
:101330000EF7B0EB074072EB17420CFB08F734BF17
:10134000A2EB0742B2EB074261EB17414FEA8C5523
:101350004FEA910704EB9C2406FB07FC4FEA1C4C68
:101360000CFB0BF7B0EBC74072EB573203FB0CF7EB
:1013700034BFA2EBC742B2EBC74261EB57310CFB63
:101380000EF7B0EBC70072EB57720CFB08F734BFD7
:10139000A2EBC702B2EBC70261EB577115EB4C250C
:1013A0004FEA816141EA92114FEA82624FEAD137F6
:1013B00042EA901206FB07FC44F100044FEA806009
:1013C0004FEA1C4C0CFB0BF7D21B03FB0CF761EB39
:1013D00007010CFB0EF7B0EB074072EB17420CFB5A
:1013E00008F734BFA2EB0742B2EB074261EB1741AB
:1013F00015EB1C154FEA813141EA92414FEA8232E6
:1014000042EA90424FEA80304FEA0C7644F1000401
:1014100048EA03434EEA0B484FF0000EB2EB080CCB
:1014200071EB030724BF624639464EEB0E0E4FF0B8
:10143000000B0018524149414BEB0B0BB2EB080C6F
:1014400071EB03077BF1000B24BF624639464EEB7C
:101450000E0E4FF0000B0018524149414BEB0B0BA5
:10146000B2EB080C71EB03077BF1000B24BF624663
:1014700039464EEB0E0E51EA020718BF46F0010640
:1014800016EB0E7655F1000254F1000103D5BDE8CC
:101490008901BDE80088BDE88901BDE80048B619AA
:1014A000524141EB0101A3F10103704780807F7E2F
:1014B0007D7C7B7A797877767675747372717170CA
:1014C0006F6E6E6D6C6C6B6A6A696868676666657C
:1014D0006464636362616160605F5F5E5E5D5D5C0A
:1014E0005C5B5B5A5A59595858575756565555557B
:1014F0005454535352525251515050504F4F4F4EDB
:101500004E4D4D4D4C4C4C4B4B4B4A4A4A49494928
:10151000484848474747474646464545454444446A
:10152000444343434342424242414141002B9C4693
:1015300030D477002BD01CB54FEA370703B44FF0F7
:1015400010004FF01001BAF1000F06D0BCF1000FEF
:10155000DCBF40F0080040F008014FF000000FBC75
:10156000BDE810400BF1010BBBF1010F08BF5FEAB2
:10157000170722BF12F1010211F101014FF00041E2
:1015800043F1000300F0004043EA00007047F9D344
:101590005708D0E746EA064613F1400F4FEA1646D1
:1015A0001FDD13F1200FDFBF16430A460021203351
:1015B0005B42BED0C3F1200746EA064602FA07F7AF
:1015C0004FEA164646EA0706C3F1200722FA03F25D
:1015D00001FA07F721FA03F14FF0000342EA07028C
:1015E000A7E746EA020646EA06464FEA164646EAF4
:1015F0000106BCBF46EA0646360C4FF000034FF02A
:1016000000024FF0000194E72DE9804C9A46934682
:1016100070B491E8380007C831EA400C48BF34EA9A
:10162000430C03D5FFF7E6FDFFF780FFF0BCBDE8F4
:10163000008C2DE9804C9A46934670B491E83800AE
:1016400007C810F0804F08BF13F0804F03D100F09F
:1016500005F8FFF76BFFF0BCBDE8008C20F07F477A
:1016600080EA030023F07F4C07EB0C03A3F57C53C7
:1016700000F00040A3F1FE0392F0000F00F0B380F1
:1016800095F0000F00F077802DE901494FEA1140F5
:101690004FEA144621EA004800FB06FC24EA06470C
:1016A00008FB06F607FB08F800FB07F718EB0648EF
:1016B0004CEB164C4FEA124B18EB07484FEA154615
:1016C0004CEB174022EA0B4E0BFB06FC25EA0647C3
:1016D0000EFB06F607FB0EFE0BFB07F71EEB064E96
:1016E0004CEB164C4FF000061EEB074E4CEB174B25
:1016F00018EB0B0840F1000018EB0E0B58EB00083C
:1017000040F100008F1A4FF000013CBFC943661B37
:1017100014BFB5EB040C00213CBFC943F61B4FEAD4
:1017200017444EEA8E0E27EA04454FEA1C4704FB95
:1017300007622CEA074C05FB07F70CFB05F604FBD8
:101740000CFC16EB074642EB174216EB0C4642EB3D
:101750001C421BEB060658EB0202414146EA9E067C
:1017600001D5BDE80189B619524141EB0101A3F150
:101770000103BDE801894FEA14454FEA114724EA05
:10178000054621EA074C05FB07F406FB07F70CFBAF
:1017900006F105FB0CFC11EB074144EB17444FEA43
:1017A000124711EB0C4144EB1C4422EA074C05FBA9
:1017B00007F206FB07F70CFB06F605FB0CFC16EB25
:1017C000074642EB174216EB0C4642EB1C456A18E3
:1017D00054F1000148BF7047B619524141EB010175
:1017E000A3F10103704795F0000F37D04FEA114283
:1017F0004FEA144721EA024624EA074C02FB07F1AC
:1018000006FB07F70CFB06F402FB0CFC14EB074489
:1018100041EB17414FEA154714EB0C4441EB1C41D7
:1018200025EA074C02FB07F506FB07F70CFB06F65B
:1018300002FB0CFC16EB074645EB174516EB0C4676
:1018400045EB1C42121951F1000148BF7047B6190F
:10185000524141EB0101A3F1010370474FEA1445E6
:101860004FEA114724EA054621EA074C05FB07F138
:1018700006FB07F70CFB06F24FF0000605FB0CFC1D
:1018800012EB074241EB174112EB0C4251EB1C41AA
:1018900048BF7047921841EB0101A3F10103704763
:1018A00010B50146806B026C12F0500F05D0026C2F
:1018B000D20626D500F054FB10BD016C41F4007136
:1018C000016401688A6812F0405F17D1027EAAB9EC
:1018D000CA6A12F4700F02D08A6852050ED44A68A0
:1018E00022F020024A60016C21F480710164016CD5
:1018F000C90403D4016C41F00101016400F02EFB26
:1019000010BD806BC26CBDE810400846104710B592
:10191000806B40210164416C41F00401416400F09E
:101920001FFB10BD10B5806B00F019FB10BD00004F
:10193000464910B54A6822F440324A604A68436812
:101940001A434A6001684A6822F480724A6001685A
:101950004A68036942EA03224A6001684A6822F041
:1019600040724A6001684A6883681A434A600168A5
:101970008A6822F400628A6001688A68C3681A4330
:101980008A60816A6FF07062D14201688A6822F0D1
:1019900070628A6001688A680CD0836A1A438A6020
:1019A00001688A6822F040528A6001688A68C36AC6
:1019B0001A4301E022F040528A6001688A6822F0EE
:1019C00002028A6001688A68037E42EA43028A60F2
:1019D00090F82010002901684A680FD042F4006294
:1019E0004A6001684A6822F460424A6001684A68B5
:1019F000174C436A04EB43331A4301E022F40062BC
:101A00004A600168CA6A22F47002CA620168CA6A3E
:101A1000838B104C04EB03531A43CA6201688A6833
:101A200022F400728A6001688A6890F8303042EAD5
:101A300043228A6001688A6822F480628A600168B1
:101A40008A68406942EA8020886010BD0023014016
:101A500000E0FFFF0000F0FFFEE70000014800F09B
:101A6000F5BB00005003002070B51B481C4C1C49FE
:101A700000681A4D1A4B603CB839A84202D9174A7F
:101A8000543A03E0984203D9144A583A126804E0E1
:101A9000A04201D94A6800E00A6812F0200F16D06F
:101AA0002022A84202D90D484C3803E0984203D9BD
:101AB0000A485038026004E0A04201D9CA6000E040
:101AC0008A60084A10685168926800F0C5F8BDE85D
:101AD0007040014800F0BABB240200205864024064
:101AE000B8600240D0010020014800F0AFBB000008
:101AF000EC040020014800F0A9BB00004C050020C8
:101B000001681823CAB2103AB2FBF3F2054B6FF327
:101B10000901032A9B5CC36500D9091D816508463C
:101B200070470000D8D7020810B5014600208B6925
:101B30008A6A4FF0C07453B1B3F5005F15D072B12B
:101B4000012A0CD0022A0AD0032A09D104E01AB1D2
:101B5000012A06D0022A03D1C96AC90100D5012091
:101B600010BDC96AA142FAD010BD002AF7D0012ADF
:101B7000F2D0022AF3D0032AF3D010BD30B50468A6
:101B8000256825F480252560046863608368402B00
:101B9000036803D099600068C26030BD9A60006835
:101BA000C16030BD08B50020064C8DF80000002350
:101BB0001A466946206820F00FFB642020F0D1FA15
:101BC000F5E7000014000020704772B6FEE7000041
:101BD0002DE9F04186B014216846FEF7E9FD1B4867
:101BE0000024016841F001010160016801F0010178
:101BF0000591016841F0020101600068144F00F096
:101C00000200059001220821384600F0A0FDDFF80F
:101C100044804FF4004600223146404600F097FDD4
:101C2000082000900125CDE9015469463846039407
:101C300000F090FC0096CDE90154694640460394BB
:101C400000F088FC06B0BDE8F081000030380240AA
:101C500000040240000002402DE9F0435F4C894639
:101C60002DED048B00254FEA19432178160C83B023
:101C7000984697B2012904D0022904D0032908D13B
:101C800003E01D4602E03D4600E03546B5F57A6FBB
:101C90007ED261F31F600090CDE901920C2269466B
:101CA0004F4802F091FA1FFA89F000EE100AF0EEA8
:101CB000080AB8EE400A20EE200ADFED4A0A207832
:101CC00020EE200AF2EE060A60EE208A9FED469B87
:101CD000012804D0022813D0032822D03BE000EED4
:101CE000108AB8EE400A10EE100A29F0BDF853EC45
:101CF000192B28F0CFFF41EC100B94ED021B20E0D4
:101D000000EE107AB8EE400A10EE100A29F0ACF896
:101D100053EC192B28F0BEFF41EC100B94ED041B83
:101D20000FE000EE106AB8EE400A10EE100A29F03B
:101D30009BF853EC192B28F0ADFF41EC100B94ED00
:101D4000061B51EC100B53EC112B28F099FE28F0D8
:101D500051FC08EE100A2648B0EE680A006821F02F
:101D6000D6F82448B0EE480A006821F0D0F8B5F55E
:101D7000006500D56D42A9B240F26C72002091421C
:101D80000CD96178491CC9B26170A070082900E0C3
:101D90001BE012D360702078401C0BE0122911D296
:101DA000A178491CC9B2A1706070082905D3A07040
:101DB0002078401EC0B209F02BFB03B0BDEC048BB1
:101DC000BDE8F0836070A070F7E703B0491CBDEC7C
:101DD000048BC8B2BDE8F04309F01ABB78000020BC
:101DE000A404002000008039000000000000A04092
:101DF000980000209C00002078B50024009490F802
:101E00003C20012A19D0012280F83C200A680723CF
:101E10000568092A13D9EE680A3A02EB4202934098
:101E20009E43EE600B788A680A3B03EB43039A40BB
:101E30000368DD682A43DA6010E0022078BD2E696D
:101E400002EB420293409E432E610B788A6803EBBB
:101E500043039A4003681D692A431A614A681F2395
:101E6000072A13D205686E6B521E02EB8202934062
:101E70009E436E630A8893B20A79521E02EB820275
:101E800093400268556B2B43536327E005680D2A86
:101E900012D22E6BD21F02EB820293409E432E631E
:101EA0000B790A88DB1F92B203EB83039A40036825
:101EB0001D6B2A431A6311E0EE6A0D3A02EB8202AF
:101EC00093409E43EE620B790A880D3B92B203EB7E
:101ED00083039A400368DD6A2A43DA621B4B056874
:101EE000194A9D420AD10D68122D07D1556825F473
:101EF00000055560556845F48005556005689D42AC
:101F00001DD1134D0B68AB4201D0112B17D1536873
:101F100023F480035360536843F40003536009685B
:101F2000A9420CD10B490C4A0968B1FBF2F101EB53
:101F30008101490000E0491E00910029FBD180F891
:101F40003C40002078BD00000023014000200140FB
:101F500012000010A000002040420F0070477047A0
:101F6000704770B504004FF0000503D0206C0026C8
:101F700010B107E0012070BD204600F01DF8666436
:101F800084F83C60206CC00610D4206C20F488508B
:101F900040F0020020642046FFF7CAFC6664206C13
:101FA00020F0020040F00100206400E0012584F8E8
:101FB0003C60284670BD000070B586B0064614210E
:101FC0006846FEF7F5FB24493068884241D1234832
:101FD0000025016841F48071016000681F4900F428
:101FE000807014390590086840F0010008600868A6
:101FF00000F001000590086840F0020008600868E1
:10200000032400F002000590E0208DE831006946CD
:10201000134800F09FFA01208DE83100694611480D
:1020200000F098FA114C1048C4E900050015A560AD
:10203000C4E90350400060618000C4E906052562E0
:102040002046656200F0D2F908B1FFF7BEFDB46327
:10205000A66306B070BD0000002001404438024075
:1020600000000240000402401064024024020020EC
:10207000F8B5044600200E46009094F83C10012963
:1020800007D0012184F83C1021688B68DB0702D05F
:1020900011E00220F8BD8B6843F001038B603649E4
:1020A000364B0968B1FBF3F101EB410100E0491E39
:1020B00000910029FBD121688B68DB0503D58B6873
:1020C00023F480738B6021688B68DB0749D0236C15
:1020D00040F20165AB4343F48073236449684905CA
:1020E00005D5216C21F4005141F480512164216C0B
:1020F000C90404D5616C21F00601616400E06064EC
:1021000084F83C00A16B1F481D4DC863A16B1E489D
:102110000864A16B1D48C86421686FF02200086044
:102120002068416841F0806141602068816841F425
:10213000807181602168134632464C31A06B00F0FB
:10214000BFF96868C006206802D01149884210D1E2
:10215000816811F0405F0CD1816841F0804181605D
:1021600007E0206C40F010002064606C40F001003B
:1021700060640020F8BD0000A000002040420F0075
:1021800000230140A1180008251900080F190008B4
:10219000002001402DE9F0410446876D00F0DCFA93
:1021A000064694F835000025022806D08020606598
:1021B00084F834500120BDE8F0812068016821F0E6
:1021C000160101602068416921F080014161206CA5
:1021D00008B9A06C20B12068016821F008010160F5
:1021E0002068016821F0010101600CE000F0B4FA00
:1021F000801B052807D920206065032084F835005E
:1022000084F83450D7E720680068C007EED194F80E
:102210005C103F208840B860012084F8350084F8C5
:1022200034500020C7E790F83510022903D08021F0
:10223000416501207047052180F83510006801686C
:1022400021F0010101600020704700002DE9F843F2
:1022500004464FF00009CDF8009063484FF4165142
:10226000A56D0068B0FBF1F72E6894F85C100820AB
:1022700000FA01F131420FD021680A6852070BD5EC
:102280000A6822F004020A6094F85C108840A86092
:10229000606D40F00100606594F85C104FF001083B
:1022A00008FA01F0304208D021684969090604D5CE
:1022B000A860606D40F00200606594F85C10042036
:1022C0008840304208D021680968890704D5A86091
:1022D000606D40F00400606594F85C101020884048
:1022E000304218D021680968090714D5A860206811
:1022F0000168490304D50068000308D5A16C07E014
:102300000168C90503D4016821F008010160216C4E
:1023100009B12046884794F85C102020884030425C
:1023200031D021680968C9062DD5A86094F8350018
:1023300005282068016806D0490347D500680003D6
:102340001DD4616C1CE021F0160101602068416918
:1023500021F080014161206C08B9A06C20B1206897
:10236000016821F00801016094F85C103F2088406A
:10237000A86084F8358084F83490216D1FE0E16B0B
:1023800009B120468847606D00282BD0606DC007DA
:1023900014D0052084F835002068016821F001017F
:1023A00001600098401C0090B84203D82068006883
:1023B000C007F6D184F8358084F83490E16C0029A8
:1023C00010D001B02046BDE8F04308470168C905B8
:1023D000D5D4016821F01001016084F8358084F8BB
:1023E0003490CCE7BDE8F883A00000202DE9F0414F
:1023F000044600F0B1F906465CB1022084F83500CD
:10240000002584F834502068016821F00101016042
:102410000DE00120BDE8F08100F09EF9801B052849
:1024200005D920206065032084F83500F2E7206894
:102430000068C007F0D12268116820480140D4E943
:1024400001031843D4E9033633431843636918433F
:10245000A3691843E3691843236A18430843616A70
:10246000042903D1D4E90B131943084310602068F1
:102470004069666A20F0070130460E4301270428B0
:102480000CD1A06A0643E06A40B12046FFF74CFB3E
:1024900020B14020606584F83570BAE72068466155
:1024A0002046FFF72DFB94F85C203F21914081608E
:1024B000656584F835700020ACE700003F8010F0BF
:1024C0002DE9F0410446866D90F83400002501287E
:1024D0000DD0012084F8340094F835700020012FCD
:1024E00007D084F8340002252846BDE8F081022098
:1024F000FBE7022784F8357060652046FFF73EFB56
:1025000094F85C103F208840B0602068016841F07A
:1025100016010160206C20B12068016841F00801BB
:1025200001602068016841F001010160DCE7000002
:1025300070B5044600F010F90546601C02D004484E
:102540000078044400F008F9401BA042FAD370BDA3
:10255000640000202DE9F84FDFF8B8A10022012423
:1025600003254FF00F090AF1040BAAF1040E00BF76
:102570000B6804FA02F63340B34273D10F7907F0C7
:102580000307012F01D0022F16D187684FEA4208B6
:1025900005FA08FC27EA0C07D1F80CC00CFA08FC75
:1025A0004CEA070CC0F808C04768B7430E79C6F379
:1025B000001696403E4346600E79F643B6070DD0AE
:1025C000C768560005FA06FC27EA0C07D1F808C0D0
:1025D0000CFA06FC4CEA070CC0F80CC00E7906F0A9
:1025E0000306022E10D1D60800EB8608D8F820602A
:1025F00057074FEAD76C09FA0CF7BE430F6907FA81
:102600000CF73743C8F8207006684FEA420C05FA09
:102610000CF7BE430F7907F0030707FA0CF73743AF
:1026200007604E6816F4403F6DD03B4E376847F464
:1026300080473760366822F0030706F4804600962C
:10264000364E07EB060CDCF8086897073F0F09FACF
:1026500007F826EA0806DFF8C880404503D14FF0A6
:1026600000081EE04FE0DFF8BC80404502D14FF08B
:10267000010816E0DFF8B080404502D14FF00208B3
:102680000FE0DFF8A880404502D14FF0030808E0D2
:10269000DFF89C80404502D14FF0040801E04FF084
:1026A000070808FA07F848EA0608CCF80888DAF8B4
:1026B00000605746D1F804C09E435FEACC2C00D599
:1026C0001E433E60DBF800605F46D1F804C09E43C5
:1026D0005FEA8C2C00D51E433E60DEF80060774632
:1026E000D1F804C09E435FEA8C3C00D51E433E6097
:1026F000084F083F3E68D1F804C09E435FEACC3CD7
:1027000000D51E433E60521C102AFFF431AFBDE8D5
:10271000F88F0000083C014044380240003001407E
:10272000000002400004024000080240000C024089
:10273000001002400069084000D001207047426943
:1027400021EA02030A4043EA0241816170470AB16B
:10275000816170470904FBE7014880687047000009
:102760006400002070B5040025D094F83D000025D9
:1027700020B984F83C50204600F0B8F8242084F8B2
:102780003D002068016821F00101016020680168B6
:1027900041F4004101602068016821F400410160BA
:1027A00000F000FB4D4A6168914201D84C4900E0BD
:1027B0004C49884201D2012070BD4B492368B0FBCF
:1027C000F1F15E6826F03F060E435E606368934257
:1027D00006D94FF4967359434FF47A73B1FBF3F172
:1027E0002368491C1E6A26F03F063143196261685E
:1027F000914210D84900401EB0FBF1F2521CC2F3C6
:102800000B02042A01D2042022E0B0FBF1F0401CAC
:10281000C0F30B001CE0A268F2B301EBC10303EBB1
:102820000116431EB3FBF6F35B1C43F480431B0508
:1028300049D092B301EBC10202EB0111401EB0FB83
:10284000F1F0401CC0F30B0040F4804040F4004025
:102850002168CA694CF6FF739A431043C861D4E9F2
:10286000071001432068026822F0C0021143016092
:10287000D4E9030101432068826848F2FF339A4398
:1028800011438160D4E9050108432168CA6822F038
:10289000FF021043C86001E00EE016E02068016806
:1028A00041F0010101602564202084F83D0025638A
:1028B00084F83E50002070BD01EB4106431EB3FB7F
:1028C000F6F35B1CB3E70120C2E701EB4101401EB8
:1028D000B0FBF1F0401CC0F30B00B7E7A08601008D
:1028E00080841E0000093D0040420F0010B586B0F4
:1028F000044614216846FDF75BFF134920688842AF
:1029000020D112480021026842F0020202600068F1
:1029100000F002000590C02000901220CDE90101D6
:10292000032003900420049069460948FFF712FE33
:1029300006481030016841F400110160006800F49D
:102940000010059006B010BD005400403038024021
:102950000004024002488168027811448160704797
:10296000640000200B4810B5016841F4007101605B
:10297000016841F480610160016841F48071016087
:10298000032000F099F80F2000F006F800F04AF854
:10299000002010BD003C024030B505461C4887B001
:1029A0000024016841F480210160006806A900F458
:1029B0008020009001A800F0D5F900F003FA154935
:1029C000154AB0FBF1F11548491E026040F2E732AA
:1029D000C0E90324C0E90114846100F0ABFE0400E7
:1029E00012D10E4800F018FF04000DD11A2000F09B
:1029F00035F8102D07D2002229461A2000F03CF8A5
:102A00000748056000E0012407B0204630BD000003
:102A10004438024040420F0000480140AC0500200D
:102A2000680000200C4882B0016841F480410160D8
:102A3000006800F4804000900748001F016841F0E2
:102A4000805101600068002200F0805000900F214A
:102A5000901E02B000F010B844380240002809DB94
:102A600000F01F02012191404009800000F1E020A8
:102A7000C0F8001170470000F0B40E4B1B680C4604
:102A8000C3F30223C3F10705042D00D90425191D42
:102A9000072901D2002300E0DB1E012606FA05F11A
:102AA000491E214099409E40761E16403143F0BC9D
:102AB00002F0E2BE0CED00E0064900F007020868F3
:102AC0004FF6FF03184040EA0220034A1043086013
:102AD000704700000CED00E00000FA052DE9F84316
:102AE000044600684FF00109C1074FF0000601D10C
:102AF000400729D5DFF82081C8F86860FFF72CFE71
:102B00000746464D05E000BFFFF726FEC01B022822
:102B100059D828680001F7D4A068217B800140EAD9
:102B20000170616808433D4984310860C8F86890C5
:102B3000FFF712FE074604E0FFF70EFEC01B022857
:102B400041D828680001F7D52078800752D533484E
:102B50004030016841F0805101600068304D00F064
:102B600080500090286840F480702860FFF7F4FDE2
:102B7000074604E0FFF7F0FDC01B022823D82868B1
:102B8000C005F7D5254D7035286810F4407020D069
:102B9000218A01F4407181421BD02868214920F428
:102BA0004070C1F800900E6028602868C00710D0FF
:102BB000FFF7D2FD064641F2883707E0FFF7CCFD6C
:102BC000801BB84202D90320BDE8F883286880073B
:102BD000F4D521691148C1F301220830032A12D02B
:102BE000016821F4F81101602868218AC1F30B0102
:102BF000084328602078000703D50B49207DC1F8E1
:102C0000E0010020E0E70268084B22F4F8121940C6
:102C10000A430260E8E70000000047420038024033
:102C200000700040400E474200104742FFFCFF0F7B
:102C30002DE9F0470E46050065D0DFF81481D8F87D
:102C40000000F7B200F00700B04207D288F8007029
:102C5000D8F8000000F00700B04254D128683D4C7D
:102C6000810712D5400703D5206840F4E05020606A
:102C70002878000703D5206840F460402060206871
:102C8000A96820F0F000084320602878C0072DD004
:102C9000304968680839012812D0022813D0032867
:102CA00011D00968890700292DDA216821F0030174
:102CB00001432160FFF750FD814641F2883A0EE062
:102CC00009688903EFE709688901ECE7FFF744FD2C
:102CD000A0EB0901514502D90320BDE8F087206827
:102CE000696800F00C00B0EB810FEFD1D8F800104C
:102CF000404601F00701B14207D90770006800F0B3
:102D00000700B04201D00120E7E72878400705D549
:102D10002068E96820F4E050084320602878000724
:102D200006D52068296920F4604040EAC10020608F
:102D300000F058F82168084AC1F30311515CC840FB
:102D40000649086006480068FFF726FE0020C4E731
:102D5000003C024008380240E0D70208A0000020F2
:102D6000680000200F2202600C4A136803F003037E
:102D70004360136803F0F0038360136803F4E053C7
:102D8000C36012684FF4E05303EAD20202610448C0
:102D9000006800F007000860704700000838024033
:102DA000003C02400448054900680968044AC1F330
:102DB0008221515CC8407047A000002008380240C2
:102DC000F0D702080448054900680968044AC1F3BD
:102DD0004231515CC8407047A000002008380240D2
:102DE000F0D70208154810B5006810F00C0214481E
:102DF00013D01449042A0FD0082A0ED10F4C241FD7
:102E00002268236802F03F025B0207D52068C0F306
:102E10008810A0FB010106E0084610BD2168C1F33F
:102E20008811A1FB00010023FDF70CFB2168C1F311
:102E30000141491C4900B0FBF1F010BD08380240C7
:102E40000024F40040787D012DE9F84F04006ED095
:102E50002078DFF84C93C007A9F104054AD009F1A6
:102E600004000168C1F38101012908D00068C0F3A2
:102E7000810002280AD1D9F80000400206D528684E
:102E8000800337D560680028E1D033E06068B0F592
:102E9000803F10D0B0F5A02F286810D020F48030EB
:102EA0002860286820F4802028606068A8B1FFF7B7
:102EB00053FC06460DE0286840F48030F4E740F407
:102EC00080202860F7E700BFFFF746FC801B6428DE
:102ED00073D828688003F7D50CE0FFF73DFC064661
:102EE00005E000BFFFF738FC801B6428F0D8286895
:102EF0008003F7D42078DFF8AC8280074FF0000A17
:102F00003ED5A748001D016811F00C0F08D00068DD
:102F1000C0F3810002280BD1D9F80000400207D489
:102F20002868800716D5E068012800D112E033E157
:102F3000E068B8B10120C8F80000FFF70DFC0646B4
:102F400005E000BFFFF708FC801B0228C0D82868F6
:102F50008007F7D52868216920F0F80040EAC10011
:102F600028600DE0C8F800A0FFF7F6FB064604E075
:102F7000FFF7F2FB801B02281FD828688007F7D4D0
:102F80002078000722D5864F87486169703771B174
:102F900001210160FFF7E0FB064604E0FFF7DCFBE0
:102FA000801B022809D838688007F7D50EE0C0F8E2
:102FB00000A0FFF7D1FB064605E082E0FFF7CCFB5F
:102FC000801B02287DD838688007F7D42078400716
:102FD00068D5DFF8CCB100270BF13C0BDBF8000023
:102FE000C0000BD4DBF8001041F08051CBF800108A
:102FF000DBF80000012700F0805000906B4E306835
:10300000C00510D4306840F480703060FFF7A4FB36
:10301000009005E0FFF7A0FB0099401A022850D865
:103020003068C005F6D55E4EA0686C3601280FD01A
:103030000528306810D020F001003060306820F0A2
:1030400004003060A068B8B1FFF786FB00900FE085
:10305000306840F00100F4E740F004003060F7E72A
:10306000FFF77AFB0099411A41F28830814266D815
:1030700030688007F4D50EE0FFF76EFB009007E0A4
:10308000FFF76AFB0099411A41F28830814256D815
:1030900030688007F4D42FB1DBF8001021F08051A4
:1030A000CBF80010A069C8B33D49091D0968C1F3F8
:1030B000810102294AD00228504607D0C8F8600092
:1030C00000E03CE0FFF748FB04463BE04746C8F819
:1030D0006000FFF741FB064605E000BFFFF73CFB41
:1030E000801B02282BD828688001F7D4D4E9070177
:1030F0000843A16A2E4A490802EB0141626A41EA8B
:103100008211084394F82C1040EA0161C9F80010BC
:1031100001203866FFF720FB044606E03EE000BFD2
:10312000FFF71AFB001B022809D828688001F7D591
:1031300034E000BFFFF710FB001B022802D9032078
:10314000BDE8F88F28688001F4D427E00128F7D083
:10315000D9F80000E26900F4800191421CD1226A92
:1031600000F03F01914217D147F6C071626A0140F9
:10317000B1EB821F10D1A26A4FF0FF3300F440314F
:1031800003EB5202B1EB024F06D194F82C1000F081
:103190007060B0EB016F01D00120D1E70020CFE7D4
:1031A0000438024000004742800E47420070004051
:1031B0000000FFFF10B5040002D0607F10B106E0F0
:1031C000012010BD00202077204600F041F80220A9
:1031D00060772068C168C943C90632D5CA214162F7
:1031E000216853204862204601F08AFD20BB2068F8
:1031F0008168164A114081602168886862681043BE
:10320000D4E904231A43104388602168E068086108
:1032100020680169228941EA02410161204601F0EA
:1032200093FD48B921680A6C22F480220A6421685F
:103230000A6CA3691A430A642268FF21516208B12B
:1032400010BD00200121617710BD0000BFFF8FFF7E
:1032500010B586B0044618216846FDF7A9FA094959
:10326000206888420CD10220009000020490684639
:10327000FFF734FC08B1FEF7A8FC03490120086001
:1032800006B010BD002800403C0E474270B5044611
:103290000B482168C860FFF75FFA05464FF47A765D
:1032A00007E000BFFFF758FA401BB04201D90320E6
:1032B00070BD2068C0688006F4D5002070BD000095
:1032C0005F3F0100704770B5040009D0606A0025B7
:1032D00040B125616561A56294F8510040B10CE0F0
:1032E000012070BD6068B0F5827FF4D0E561F2E73F
:1032F00084F85050204600F045F8022084F8510030
:103300002068016821F040010160A088218900F453
:10331000827001F404410843A18901F4006108436B
:10332000217C01F002010843217D01F001010843E5
:10333000218B01F400710843217F01F0380108431B
:1033400094F8201001F080010843218D01F4005110
:10335000084321680860A069042101EA104094F83C
:10336000241001F010010843216848602068C169F9
:1033700021F40061C1616565012084F851000020DD
:1033800070BD000070B586B0064614216846FDF792
:103390000FFA20493068884239D11F48002501685A
:1033A00041F480410160006800F4804005901A48B3
:1033B0001038016841F0020101600068694600F0C0
:1033C000020005904FF4204000900220CDE9010555
:1033D00003200390052004901048FFF7BBF8114C20
:1033E0000F48C4E900054020C4E90205000120613E
:1033F000400060618000C4E90605256220466562E0
:10340000FEF7F4FF08B1FEF7E0FBB464A66306B074
:1034100070BD000000380040403802400004024007
:1034200070600240500300202DE9F84F9846164680
:103430008A460446FFF790F9814694F85100012826
:103440001ED1BAF1000F73D0002E71D094F8500045
:10345000012815D0012784F85070032084F851000A
:1034600000256565C4F830A0A686E686A563A58715
:10347000E58765642564A068B0F5004F03D00CE0D3
:103480000220BDE8F88F2068016821F0400101604A
:103490002068016841F480410160206801684906A4
:1034A00003D4016841F040010160E068B0F5006FAD
:1034B000606803D048B3012E27D047E008B1012E41
:1034C0001FD1206B21680088C86006E020688168F1
:1034D000890709D5216B0988C160206B801C206396
:1034E000E08E401EE0860CE0FFF736F9A0EB090104
:1034F000414503D3B8F1FF3F03D035E0B8F1000FE9
:1035000032D0E08E0028E1D123E0206B21680078E2
:10351000087306E02068816889070AD5216B09785D
:103520000173206B401C2063E08E401EE0860DE09E
:103530002BE0FFF711F9A0EB0901414503D3B8F1E6
:10354000FF3F03D010E0B8F1000F0DD0E08E00284F
:10355000E0D14A464146204601F054FC08B1202003
:103560006065A06830B109E084F8517084F850506B
:10357000032086E72068C1688068009084F8517055
:1035800004F8505F60680028F3D0012079E700005C
:1035900070B5044690F8510001281CD1C9B1C2B1E0
:1035A00094F85000012816D0012084F85000032020
:1035B00084F85100002565652163A286E286A56333
:1035C00065642564A587E587A068B0F5004F04D041
:1035D0000DE0012070BD022070BD2068016821F05F
:1035E000400101602068016841F480410160A16CE4
:1035F00017480864A16C1748C863A16C1648C864D2
:10360000A06C0565E38E2268216B0C32A06CFEF77E
:1036100057FF30B1606D40F01000606584F8505085
:10362000D7E720680168490603D4016841F04001EA
:10363000016084F850502068416841F020014160E9
:103640002068416841F002014160002070BD000027
:10365000954D00089F4D0008734D00087047704756
:103660007047704710B590F83C20012A22D0012203
:1036700080F83C20CA688C6822F4407222434C686F
:1036800022F4806222430C6822F4006222430C6917
:1036900022F4805222434C6922F400522243C96929
:1036A000002322F480420A4301684A6480F83C30D7
:1036B000002010BD022010BD70B590F83C20012AFA
:1036C0002CD0012480F83C40022280F83D20036881
:1036D0005A689D6822F070060A6832435A60104B9F
:1036E00002689A420ED0B2F1804F0BD00D4B9A4235
:1036F00008D00D4B9A4205D00C4B9A4202D00C4B8D
:103700009A4204D1496825F080031943916080F8FA
:103710003D40002180F83C10084670BD022070BD7D
:10372000000001400004004000080040000C004080
:103730000040014010B5040003D094F83D0010B1E2
:1037400007E0012010BD002084F83C00204600F076
:103750001FF8022084F83D00211D206801F062FC62
:10376000012084F8460084F83E0084F83F0084F885
:10377000400084F8410084F8420084F8430084F853
:10378000440084F8450084F83D00002010BD00008E
:1037900008B50068B0F1804F08D10548016841F0D4
:1037A00001010160006800F00100009008BD000008
:1037B0004038024090F83D10012901D001207047A7
:1037C000022180F83D1000680E4988420ED0B0F109
:1037D000804F0BD00C49884208D00C49884205D054
:1037E0000B49884202D00B49884204D1816801F01C
:1037F0000701062903D0016841F0010101600020A2
:103800007047000000000140000400400008004034
:10381000000C00400040014090F83D10012901D00B
:1038200001207047022180F83D100168CA6842F00B
:103830000102CA6000680E4988420ED0B0F1804F84
:103840000BD00C49884208D00B49884205D00B495F
:10385000884202D00A49884204D1816801F00701F8
:10386000062903D0016841F0010101600020704782
:10387000000001400004004000080040000C00402F
:103880000040014070472DE9F04104460068C668D9
:1038900005694FF00007A90713D5B10711D5F91E27
:1038A000016101202077206880698007204602D0CE
:1038B000FFF7E8FF04E000F0C1F8204600F07EF9D1
:1038C0002777680716D5700714D521686FF00400B4
:1038D0000861022020772068806910F4407F20462C
:1038E00002D0FFF7CFFF04E000F0A8F8204600F078
:1038F00065F92777280715D5300713D521686FF0AC
:1039000008000861042020772068C06980072046ED
:1039100002D0FFF7B7FF04E000F090F8204600F077
:103920004DF92777E80616D5F00614D521686FF013
:1039300010000861082020772068C06910F4407FDB
:10394000204602D0FFF79EFF04E000F077F8204603
:1039500000F034F92777E80708D0F00706D021688F
:103960006FF001000861204600F082F9280608D5B2
:10397000300606D521686FF0800008612046FFF709
:103980006FFE680608D5700606D521686FF0400006
:103990000861204600F0A1F9A8060AD5B00608D5AE
:1039A00021686FF0200008612046BDE8F041FFF774
:1039B00058BEBDE8F081000010B586B00446142161
:1039C0006846FCF7F5FE2368174C002117480222D1
:1039D000A34211D1036843F001030360006800F0C3
:1039E0000100059050020090CDE901210120CDE9B0
:1039F000031069460E4812E00E4CA34211D1036831
:103A000043F002030360006800F0020005906015B7
:103A10000090CDE90121CDE9031269460648FEF781
:103A200099FD06B010BD0000000001403038024092
:103A3000000002400008004000040240704770B5DA
:103A4000044690F83C0000260D4601280FD00120C6
:103A500084F83C006AB1042A1DD0082A2FD00C2A11
:103A60003FD00126002084F83C00304670BD022083
:103A700070BD206801F040FB2068816941F00801B9
:103A800081612068816921F0040181612068816978
:103A90002A69114311E0206801F056FB2068816912
:103AA00041F4006181612068816921F48061816154
:103AB000206881692A6941EA02218161D2E7206890
:103AC00001F06EFB2068C16941F00801C161206806
:103AD000C16921F00401C1612068C1692A691143EB
:103AE00011E0206801F088FB2068C16941F40061A1
:103AF000C1612068C16921F48061C1612068C16928
:103B00002A6941EA0221C161ACE710B5040003D083
:103B100094F83D0010B107E0012010BD002084F8AA
:103B20003C00204600F01EF8022084F83D00211DD4
:103B3000206801F077FA012084F8460084F83E00FE
:103B400084F83F0084F8400084F8410084F8420083
:103B500084F8430084F8440084F8450084F83D006C
:103B6000002010BD08B500681149884212D11148E3
:103B7000016841F0010101600068002200F00100CD
:103B800000900F211A20FEF777FFBDE808401A20A9
:103B9000FEF764BF0849884209D10648001F016842
:103BA00041F004010160006800F00400009008BDCD
:103BB0000000014044380240000800407047000007
:103BC00010B50446022249B104290ED0082913D0A9
:103BD00094F84100012816D0012010BD94F83E0051
:103BE0000128F9D184F83E200FE094F83F00012825
:103BF000F2D184F83F2008E094F840000128EBD18E
:103C000084F8402001E084F841200122206801F07E
:103C10005BFA12492068884203D1426C42F40042A8
:103C20004264206888420ED0B0F1804F0BD00C491E
:103C3000884208D00B49884205D00B49884202D0FF
:103C40000A49884204D1816801F00701062903D09E
:103C5000016841F001010160002010BD0000014039
:103C60000004004000080040000C004000400140FB
:103C700000680349884201D1FEF76CBE704700001E
:103C80000048014070B5044690F83C00012812D06D
:103C9000012584F83C50022084F83D00204601F0C4
:103CA000CDFA01004FF0000007D084F83D5084F8B1
:103CB0003C00012070BD022070BD2168CA6822F05E
:103CC0004002CA602168CA6822F48042CA6084F84F
:103CD0003D5084F83C00002070BD7047704710B51F
:103CE00004460068406994F84110C0F3C0102129CF
:103CF00011D180B12068143050E8001F21F08001FC
:103D000040E80012002AF5D1A06B08B1FEF742FA94
:103D1000204601F0D3FB2068406994F84210C0F3BC
:103D20008010222911D180B12068143050E8001F82
:103D300021F0400140E80012002AF5D1E06B08B103
:103D4000FEF728FA204601F092FB002010BD7047D4
:103D5000F8B5016804460868CA684B6910F00F0F8F
:103D60004FF0000559D003F0010602F49077374375
:103D700065D0C10705D0D10503D5616C41F00101C3
:103D80006164410705D5D90703D0616C41F0020198
:103D90006164810705D5D90703D0616C41F0040146
:103DA0006164010707D502F02001314303D0616C43
:103DB00041F008016164616C00293AD0800604D5A5
:103DC000900602D5204601F087FB20684069616CAF
:103DD000C0F38010090700D460B3204601F047FB10
:103DE00020684069400621D52068143050E8001F43
:103DF00021F0400140E80012002AF5D1E06BA8B1A3
:103E00006E490165E06BFEF70EFA002811D0E06BF9
:103E1000016D01B0BDE8F040084783060FD5930659
:103E20000DD52046BDE8F84001F056BB2046FFF70F
:103E30008EFFF8BD2046FFF78AFF6564F8BD266B4C
:103E40002023012E7DD1C6067BD5D60679D50868FC
:103E50004868009048694FF00206400641D5E16B82
:103E6000086840680004000CE8D0A28D8242E5D9C1
:103E7000E085C869B0F5807F2DD020680C3050E80F
:103E8000001F21F4807140E80012002AF5D120685B
:103E9000143050E8001F21F0010140E80012002A10
:103EA000F5D12068143050E8001F21F0400140E8AF
:103EB0000012002AF5D184F84230256320680C30C6
:103EC00050E8001F21F0100140E80012002AF5D14F
:103ED000E06BFEF75FF96663A08DE18D401A81B259
:103EE0002AE0A08DE18D401A81B2E08D0028A5D096
:103EF0000029A3D022680C3252E8000F20F4907001
:103F000042E80007002FF5D12068143050E8002F58
:103F100022F0010240E80027002FF5D184F842305A
:103F2000256320680C3050E8002F22F0100240E892
:103F30000023002BF5D166632046FFF7CFFEF8BDC6
:103F4000FFE705062BD5150629D594F84100212851
:103F5000F5D1A068B0F5805F01D12069B0B1206AC9
:103F6000411C2162216800784860E08C401E0004FA
:103F7000000CE084E3D12068C16821F08001C160B9
:103F80002068C16841F04001C160D8E7206A00881C
:103F9000C0F308004860206A801C2062E5E7400604
:103FA000CDD55006CBD5CA68204622F04002CA6063
:103FB00084F8413000F044F9C1E7000025530008BF
:103FC00070B5040004D094F84100002510B106E05B
:103FD000012070BD84F84050204600F023F82420D2
:103FE00084F841002068C16821F40051C160204676
:103FF00001F0D4FA2068016921F490410161206840
:10400000416921F02A0141612068C16841F40051F1
:10401000C1606564202084F8410084F84200656333
:10402000002070BD2DE9F04186B006461421684697
:10403000FCF7BEFB2F493068884258D12E48002437
:10404000016841F020010160006800F02000059047
:1040500029481438016841F001010160006869468F
:1040600000F0010005904FF4C05000900220CDE90F
:10407000010403200390082004902048FEF76AFA08
:10408000204D1F484FF4806887052860C5E90174FA
:10409000C5E903486C61AC61EC612C6228466C6236
:1040A000FEF7A4F908B1FDF790FDF563AE63154D79
:1040B000134860357830E5E802074020A5E8110193
:1040C000104845F814496030AC61EC612C626C62B8
:1040D000FEF78CF908B1FDF778FDB56300220521E4
:1040E0004720AE63FEF7C8FC4720FEF7B7FC06B0DA
:1040F000BDE8F08100140140443802400000024055
:1041000028640240EC04002090F84230202B01D0BB
:104110000220704721B11AB10023036301F0C4BA31
:1041200001207047704770472DE9F843044690F826
:104130004100984616460D46202802D00220BDE8D0
:10414000F88385B17EB100206064212084F84100AD
:10415000FEF702FBA6848146E684A0682027B0F51E
:10416000805F02D003E00120E9E7206910B12E460C
:1041700000250EE000260CE08021204601F0DCFA4C
:10418000A8B9C6B116F8010B21684860E08C401E42
:10419000E084E08C4B464FF00002CDF80080002810
:1041A000EAD14FF04001204601F0C6FA40B184F850
:1041B00041700320C3E735F8020BC0F30800E3E7C2
:1041C00084F841700020BAE770B5044690F84100C9
:1041D000202801D0022070BD49B342B32162A284DD
:1041E000E28400206064212384F84130A56B114BE8
:1041F000EB63A56B104B2B64A56B104BEB64A36BAF
:104200001865256813462A1DA06BFEF759F9216829
:104210006FF0400008602068143050E8001F41F043
:10422000800140E80012002AF5D1002070BD012075
:1042300070BD000023540008655400083553000881
:1042400070477047FEE70000284D294E294F4FF078
:104250005508294C4FF0AA094FF0030A4FF4806B20
:1042600025F0F8FA192225492048FFF74DFF286864
:10427000C16841F01001C1600D2121A001F04AF890
:1042800008201EF0FDFD306008201EF0F9FD3860AA
:1042900084F8008084F8019084F802A0FDF798FC6F
:1042A000032007F0B5F8002259461948FEF74FFAE7
:1042B0000422211D1748FDF7DBFE1748FFF77AFAA5
:1042C00008211648FFF77CFC00F0E2F813F02CFC04
:1042D00019F0B2FE24F0DCFB26F07AF8002025F07D
:1042E000EBF94FF4FA701DF03CFFB9E7A40400208D
:1042F000980000209C000020D001002088040020AD
:10430000706F7765722D7069636F0D0A0000000091
:1043100000040240DC010020F8030020B00300206C
:104320002DE9F0410027494CDFF8248101253E4664
:1043300010B12570667001E02078C8B301214046B5
:10434000FEF7F8F998B102214046FEF7F3F970B193
:1043500004214046FEF7EEF948B108214046FEF739
:10436000E9F920B110214046FEF7E4F900BB032033
:104370001DF0F7FE01214046FEF7DCF9002859D078
:1043800002214046FEF7D6F9002855D004214046C8
:10439000FEF7D0F9F0B308214046FEF7CBF9D0B3D1
:1043A00010214046FEF7C6F9B0B36078A8B3267076
:1043B000607890B301214046FEF7BCF968B3022152
:1043C0004046FEF7B7F940B304214046FEF7B2F984
:1043D00018B308214046FEF7ADF9F0B11021404670
:1043E000FEF7A8F9C8B103201DF0BBFE012140462D
:1043F000FEF7A0F988B102214046FEF79BF960B1B3
:1044000004214046FEF796F938B108214046FEF7F0
:1044100091F903E012E014E015E008E038B1102152
:104420004046FEF787F910B1257067786670384608
:10443000BDE8F0816570BAE7022000E003206070FB
:10444000B5E70420FBE70520F9E700007000002035
:104450000000024008B500200C4C8DF80000002040
:10446000FFF75EFF8DF8000006280AD2DFE800F0B3
:1044700009030303030301230022694620681DF09A
:1044800009FF01201DF06DFEE9E700001400002087
:1044900000B587B014216846FCF78AF90A48002164
:1044A000026842F001020260006800F0010005901D
:1044B0001F20CDE900010120029069460348FEF764
:1044C00049F807B000BD000030380240000002404B
:1044D0002DE9F04104461D4616460F462A2000F0FD
:1044E0009DF9204600F08AF9304600F087F92B202C
:1044F00000F094F9384600F081F9284600F07EF982
:10450000BDE8F0412C2000F089B9000070B55D1ABB
:10451000141A641C6D1C503350316C439BB289B229
:10452000049EFFF7D5FF0D4D4FF40060E86028684A
:10453000016841F400610160A2B231462846FFF7EC
:1045400027F80748006841680029FCD10020E8608E
:104550002868016821F40061016070BDF802002044
:10456000500300202DE9F04780461F4603F14F001D
:1045700083B21646501E82B20C4601F1500081B241
:104580004046DDF82090FFF7A3FF0AE0454604E02F
:10459000484600F033F96D1CADB2B542F8D3641C47
:1045A000A4B2BC42F2D3BDE8F0870000F0B587B0FA
:1045B00014216846FCF7FCF81848016841F0020134
:1045C0000160016801F002010591016841F00201FA
:1045D000016000684FF4805600F00200059001244D
:1045E0000F4FCDE900640325694603953846FDF772
:1045F000B1FF012231463846FEF7A9F82E02CDE977
:104600000064084C694603952046FDF7A3FF01228C
:1046100031462046FEF79BF807B0F0BD3038024027
:10462000000402400000024070B5FFF7BFFF002207
:104630004FF480716748FEF78AF8674D4FF4805455
:10464000002221462846FEF782F86420FDF770FF1D
:10465000012221462846FEF77AF86420FDF768FF1C
:10466000112000F0DBF87820FDF762FF362000F023
:10467000D5F8C02000F0E8F83A2000F0CFF8052087
:1046800000F0E2F8B22000F0C9F80C2000F0DCF8ED
:104690000C2000F0D9F8002000F0D6F8332000F00C
:1046A000D3F8332000F0D0F8B72000F0B7F8352069
:1046B00000F0CAF8BB2000F0B1F8192000F0C4F8EF
:1046C000C02000F0ABF82C2000F0BEF8C22000F0B3
:1046D000A5F8012000F0B8F8C32000F09FF81220E0
:1046E00000F0B2F8C42000F099F8202000F0ACF8F7
:1046F000C62000F093F80F2000F0A6F8D02000F0BC
:104700008DF8A42000F0A0F8A12000F09DF8E02092
:1047100000F084F8D02000F097F8042000F094F81E
:104720000D2000F091F8112000F08EF8132000F019
:104730008BF82B2000F088F83F2000F085F85420FB
:1047400000F082F84C2000F07FF8182000F07CF890
:104750000D2000F079F80B2000F076F81F2000F013
:1047600073F8232000F070F8E12000F057F8D02013
:1047700000F06AF8042000F067F80C2000F064F8FC
:10478000112000F061F8132000F05EF82C2000F0FA
:104790005BF83F2000F058F8442000F055F8512015
:1047A00000F052F82F2000F04FF81F2000F04CF8D6
:1047B0001F2000F049F8202000F046F8232000F0E8
:1047C00043F8212000F02AF8BDE87040292000F0CD
:1047D00025B800000000024000040240411F5F298C
:1047E00009D84FF4967110FB01F06421B0FBF1F091
:1047F00001490968C8637047B003002008B5010A81
:104800008DF800108DF8010001230222694602484C
:10481000FEF70AFE08BD0000F802002070B5094D41
:1048200006464FF40074002221462846FDF78FFF0C
:10483000304600F009F821462846BDE870400122C4
:10484000FDF785BF0000024001B501231A46694605
:104850000148FEF7E9FD08BDF80200201CF08AFDC2
:1048600001201DF07EFCF9E77FB500212A48009168
:1048700001910291274A0391026001244FF4803292
:104880000461C0E90121017680F820101203C262A0
:1048900004254FF0C062C5618262C16080F830407B
:1048A0004461FDF75EFB08B1FDF78FF90520CDE906
:1048B00000040624694618480294FDF79DFA08B1E1
:1048C000FDF783F90220CDE9004069461248FDF763
:1048D00093FA08B1FDF779F90720009003200190C1
:1048E00069460D48FDF788FA08B1FDF76EF9082012
:1048F000CDE9000569460848FDF77EFA08B1FDF7E5
:1049000064F9054848300068016841F01001016011
:104910007FBD000000200140DC010020194808B5DF
:10492000016841F400110160016801F40011009177
:10493000016841F4800101600068002200F48000F9
:10494000009005210F20FEF797F80F20FEF786F85C
:10495000002205213820FEF78FF83820FEF77EF878
:10496000002205213920FEF787F83920FEF776F876
:10497000002205214520FEF77FF8BDE808404520CC
:10498000FEF76CB83038024010B500F02DFF044A35
:10499000002104481DF0B2FC0349086010BD00006E
:1049A00064AF0208294F0008000000202DE9F04103
:1049B00086B014216846FBF7FBFE1F4800240168FF
:1049C00041F004010160016801F0040105910168F2
:1049D00041F001010160016801F0010105910168E8
:1049E00041F0020101600068144F00F002004FF432
:1049F00000550590002229463846FDF7A8FEDFF84D
:104A00004080EE10002231464046FDF7A0FE0095A2
:104A10000125CDE90154694638460394FDF79AFD16
:104A20000096CDE90154694640460394FDF792FD96
:104A300006B0BDE8F08100003038024000080240B6
:104A4000000402400D4810B50B4901600C4941605B
:104A500000214FF480428160C0E90312416181610D
:104A6000C1610162FDF77EFE002803D0BDE8104061
:104A7000FDF7ABB810BD00000054004084020020D8
:104A8000A08601000B4810B50949016000217F2272
:104A9000C0E90112FF22C0E9032141618161FEF7F3
:104AA00089FB002803D0BDE81040FDF78EB810BD8B
:104AB00000280040D8020020104810B50E490160BF
:104AC0004FF482714160002102228160C0E903122B
:104AD000012242615202C0E9062101624162816203
:104AE0000A21C162FEF7EFFB002803D0BDE81040A9
:104AF000FDF76BB810BD000000380040F802002040
:104B000010B592B000240F941C2108A81094FBF754
:104B10004FFE20216846FBF74BFE20481E490160EE
:104B20006321C0E901144FF49671C0E90314446194
:104B30008461FEF7EAFF08B1FDF747F80F940FA96B
:104B400016481094FEF7B8FD08B1FDF73EF8602056
:104B5000CDE908040A940B940C940D94082208A93A
:104B60000E480E94FEF76BFF08B1FDF72EF8009487
:104B70004FF40050CDE90440029401940394694637
:104B800006480794FEF76EFD08B1FDF71EF80348CE
:104B9000FEF712FF12B010BD00000140B00300206C
:104BA00010B588B014216846FBF702FE00241548B2
:104BB00005944FF08041069401600921C0E9011479
:104BC00040F2E731C0E9031480218161FEF7B2FDB4
:104BD00008B1FCF7FAFF009469460A480194FFF710
:104BE00051F808B1FCF7F1FF2020CDE9050405A933
:104BF0000448FEF761FD002801D0FCF7E6FF08B08D
:104C000010BD0000F803002010B58AB000240794FE
:104C10001C2168460894FBF7CBFD16481449016037
:104C20006321C0E90114FA21C0E903148461FEF78D
:104C30006CFF08B1FCF7C9FF079407A90D48089459
:104C4000FEF73AFD08B1FCF7C0FF6020CDE9000493
:104C500002940C22694607480494FEF7F0FE08B15E
:104C6000FCF7B3FF0348FEF7A7FE0AB010BD000033
:104C700000080040400400200C4810B50A490160BB
:104C80000B494160002181600C22C160C0E904121F
:104C90008161C161FFF794F9002803D0BDE810409D
:104CA000FCF793BF10BD000000140140A4040020D5
:104CB00060E31600FEE7FEE718210148FBF778BD28
:104CC000F405002070B5074C207D002809D0256828
:104CD000286800B18047A868006819F085FE0020A8
:104CE000607570BDF405002004490A7D052A04D2D0
:104CF00041F82200087D401C08757047F40500202B
:104D00002DE9F041044600680025C168490618D421
:104D1000C16841F08001C160FDF71EFD06464FF4F9
:104D20007A78042707E000BFFDF716FD801B404599
:104D300001D9677701252068C068400601D4002D9D
:104D4000F2D02846BDE8F08170B504460068002521
:104D5000C16821F08001C16020688068800606D4A7
:104D60002046FEF793FA10B104206077012528460B
:104D700070BD10B5806B01684A6822F003024A607A
:104D8000416D41F010014165012180F85110FEF79D
:104D900099FA10BD10B5806BFEF761FC10BD38B5F7
:104DA0000546846BFDF7D8FC024628680068C005FC
:104DB00023D42068416821F02001416020684168C7
:104DC00021F0020141606421204600F01BF818B177
:104DD000606D40F020006065A068002118B920686F
:104DE000C26880680090E186012084F85100606DFF
:104DF00018B12046FEF766FA38BD2046FEF72EFCB5
:104E000038BD0000F8B515460E460B460092044624
:104E10000122022100F02CF8A0B9134813490068C0
:104E2000B0FBF1F04FF47A71484300906068B0F540
:104E3000827F0DD13346002280212046009500F06C
:104E400017F870B1606D40F0200060650320F8BD78
:104E5000009830B1401E009020688068C043000672
:104E6000F6D50020F8BD0000A000002000366E013D
:104E70002DE9F8431E46914688460446089DFDF7F5
:104E80006BFC401B351AFDF767FC07462548006898
:104E9000C0F3CB30684338E0701C37D0FDF75CFCC2
:104EA000C01BA84203D215B1009860B32CE0206863
:104EB000416821F0E00141606068B0F5827F0BD16C
:104EC000A068B0F5004F02D0B0F5806F04D1206823
:104ED000016821F040010160A06AB0F5005F09D1CE
:104EE0002068016821F4005101602068016841F4E4
:104EF00000510160012084F85100002084F8500026
:104F00000320BDE8F8830025401E009020688168DA
:104F100038EA010004D000214945BDD10020F0E766
:104F20000121F9E7A0000020064D4FF400544FF492
:104F3000FA7621462846FDF702FC30461DF011F9AD
:104F4000F7E700000008024010B54FF0E0200069CC
:104F500025F046F9012803D0BDE8104024F006BE34
:104F600010BD000030B593B030216846FBF720FC3F
:104F700014210CA8FBF71CFC1D480024016841F01B
:104F800080510160006800F080501190194801685C
:104F900041F4404101600068102100F4404011904C
:104FA0000A2000900120CDE903010225CDE9050585
:104FB0000820CDE907406420CDE9090504200B90C5
:104FC0006846FDF741FF08B172B6FEE70F20CDE954
:104FD0000C054FF48050CDE90E4003210CA810942D
:104FE000FDF726FE002801D072B6FEE713B030BDF3
:104FF00040380240007000400248016841F47001EE
:105000000160704788ED00E010B50448FEF73BFCF6
:10501000BDE810400248FEF736BC0000B003002097
:10502000AC050020F0B50268204B214C9F03214DB8
:10503000214E984207D0B84205D0A04203D0A842E2
:1050400001D0B04204D122F0700C4A6842EA0C024E
:10505000984210D0B8420ED0A0420CD0A8420AD03C
:10506000B04208D0154CA04205D0154CA04202D049
:10507000144CA04203D122F44074CA6822434C6904
:1050800022F08002224302608A68C2620A68826259
:10509000984201D109690163012141610169C90790
:1050A00003D0016921F001010161F0BD0000014060
:1050B0000004004000080040000C00400040014097
:1050C000004401400048014010B501F01F030121D8
:1050D000046A99408C430462016A9A401143016258
:1050E00010BD10B5846842EA032224F47F440A43C9
:1050F0002243826010BD000030B5036A026A22F0CC
:10510000010202624268846924F073050C682C4332
:1051100023F002058B682B430A4DA8420BD123F0E4
:105120000805CB6822F440722B434D6923F0040339
:1051300015438A692A434260846149684163036276
:1051400030BD00000000014030B5026A036A23F060
:1051500010030362436884690D6824F4E64444EA5A
:1051600005248D6822F0200242EA05120B4DA84268
:105170000ED1CD6822F0800242EA05124D6923F477
:10518000406343EA85038D6922F0400243EA8503C8
:105190004360846149688163026230BD0000014060
:1051A00030B5036A026A22F4807202624268C469FE
:1051B00023F4007324F073050C682C438D6843EAD4
:1051C00005230C4DA8420ED1CD6823F4006343EAB9
:1051D00005234D6922F4405242EA05128D6923F4F9
:1051E000806342EA05124260C4614968C163036298
:1051F00030BD00000000014030B5046A026A22F4AC
:10520000805202624268C3690D6823F4E64343EAB0
:1052100005238D6824F4005444EA0534064DA84261
:1052200004D14D6922F4804242EA85124260C36192
:1052300049680164046230BD0000014070B5036834
:1052400000249A6822F070054A682A4322F0070574
:105250000A682A439A604A6812F00F0F31D112117E
:10526000082A2ED2DFE802F02E2E2E2E0B21270444
:105270000B69D1E902210068FFF733FF22E00A68D9
:10528000052A10D00268136A156A25F00105156217
:1052900002689569096925F0F00545EA01119161F7
:1052A000006803620EE0012070BD0A698968006829
:1052B00000F00AF806E00A698968006800F015F84D
:1052C00000E00124204670BD10B5036A046A24F092
:1052D00001040462846924F0F00444EA021423F017
:1052E0000A020A438461026210BD10B5036A046AAF
:1052F00024F010040462846923F0A00324F47044B1
:1053000044EA023243EA01118261016210BD0120C8
:105310001BF06CBF0A46014601230148FEF704BF9B
:10532000A404002010B5806B0021C185C184FEF764
:105330000EFD10BD70B5846B2068406994F8411073
:10534000C0F3C0100025212904D118B1E5842046FE
:1053500000F0B4F82068406994F84210C0F380105F
:10536000222904D118B1E585204600F080F8606C50
:1053700040F0100060642046FEF7E9FC70BD10B5F7
:105380000146806B096809684FF00002C9052ED4F8
:10539000C28501680C3151E8003F23F4807341E875
:1053A0000034002CF5D10168143151E8003F23F09E
:1053B000010341E80034002CF5D10168143151E8B3
:1053C000003F23F0400341E80034002CF5D12021B8
:1053D00080F84210016B012909D101680C3151E8B4
:1053E000003F23F0100341E80034002CF5D1426364
:1053F000016B012902D0FEF795FE10BD818DFEF7ED
:105400006DFC10BD10B5806B01214163016B01295A
:1054100002D0FEF788FE10BD818D4908FEF75EFCC4
:1054200010BD10B50146806B09680968C90516D41E
:105430000021C1840168143151E8002F22F080025C
:1054400041E80023002BF5D101680C3151E8002F11
:1054500042F0400241E80023002BF5D110BDFEF7D9
:10546000EFFE10BD10B5806BFEF7EBFE10BD0168BE
:105470000C3151E8002F22F4907241E80023002BF8
:10548000F5D10168143151E8002F22F0010241E802
:105490000023002BF5D1016B012909D101680C31E2
:1054A00051E8002F22F0100241E80023002BF5D133
:1054B000202180F8421000210163704701680C31FF
:1054C00051E8002F22F0C00241E80023002BF5D163
:1054D000202180F84110704708B590F84210222929
:1054E00001D0022008BD82684FF480539A4201D156
:1054F000016921B1816A9A421BD04AB10AE002686F
:10550000816A5268C2F308020A80816A891C08E035
:10551000026972B10268526802F07F020A70816A01
:10552000491C8162C18D491E0904090CC18503D043
:105530001BE002685268F1E70168CA6822F02002A5
:10554000CA600168CA6822F48072CA6001684A6948
:1055500022F001024A61202180F8421000214163BB
:10556000026B012A03D0FEF7DDFD002008BD0163B8
:1055700001680C3151E8002F22F0100241E80023AD
:10558000002BF5D101680A68D20602D50A6849687D
:105590000091818DFEF7A2FBE7E7000070B504469D
:1055A00000680169E26821F44051114301612169F9
:1055B000A068E26908436169114308432168CA6829
:1055C00049F20C639A430243CA6020684169A269A8
:1055D00021F440711143416131492068884202D071
:1055E0003049884202D1FDF7EDFB01E0FDF7DAFB1F
:1055F000E2690023192164253226B2F5004F626862
:1056000028D0A0FB0101930F9200FAF71BFF01467F
:10561000B0FBF5F06FF01802504301EB800006EB91
:105620000010B0FBF5F000F0F002B1FBF5F002EB7A
:105630000012B1FBF5F06FF01803584301EB800046
:1056400006EB0010B0FBF5F000F00F0021681044ED
:10565000886070BDA0FB010192185B41FAF7F2FE71
:105660000146B0FBF5F00201B1FBF5F06FF0180355
:10567000584301EB800006EBC000B0FBF5F000F0F2
:10568000F80002EB4002B1FBF5F0584301EB80005B
:1056900006EBC000B0FBF5F000F00700D6E7000015
:1056A000001001400014014038B581620446828533
:1056B000002013466064222284F84220E56B1B4AD6
:1056C000EA63E56B1A4A2A64E56B1A4AEA64E26BFC
:1056D00010650A462168E06B091DFCF7F1FE2068A1
:1056E000016840680090206948B120680C3050E89B
:1056F000001F41F4807140E80012002AF5D12068B3
:10570000143050E8001F41F0010140E80012002A67
:10571000F5D12068143050E8001F41F0400140E806
:105720000012002AF5D1002038BD00007F53000888
:1057300005540008355300082DE9F84398461746EC
:105740000D460446089E24E0701C22D0FDF704F8A4
:10575000A0EB0800B0421AD8CEB12068C168490752
:1057600017D5802D15D0402D13D00168C9430907E6
:105770000FD401680025406800902046FFF777FEAF
:105780000820606484F840500120BDE8F8830320BD
:10579000FBE72068006835EA000004D00020B8422A
:1057A000D2D00020F1E70120F9E700000B4810B546
:1057B00000680168C943C9060AD46FF0100101608E
:1057C0000648FEF78CFA192205490448FEF79CFCAE
:1057D000BDE810400148FEF7BBBA0000A404002059
:1057E00088040020FEE7000010B5002201210420FB
:1057F0001CF024FD0E4C0F4A002120610E481CF0C5
:105800007DFD0C4A2060243200210C481CF076FDFE
:10581000084A60604832002109481CF06FFD054AC3
:10582000A0606C32002107481CF068FDE06010BDEC
:105830000400002088AF020849420008A51B0008A8
:10584000554400085D48000803B4019841000098E1
:1058500050EAC12018BF04204A0D18BF40F00100D3
:1058600040F2FF72B2EB515F08BF40F00200012826
:1058700008BF052002B070470907090E002804DBA5
:1058800000F1E02080F80014704700F00F0000F1F4
:10589000E02080F8141D704770B5044600256FF0B5
:1058A0002F0608E02068411C2160007805EB850187
:1058B00006EB410145182068007800F061F80028E7
:1058C000F0D1284670BD70B514460D461BB911467F
:1058D0000CF0F6FB034603FB05F0142C0ED0E11F81
:1058E00003290AD8072C0DD0082C0DD0092C0DD077
:1058F0000A2C0DD0002100EB810070BD590801FB7E
:10590000050070BD0221F6E70421F4E71021F2E75B
:105910004FF48071EFE7000010B516482DED028BB3
:105920000178491CC9B201700A2907D3002101700E
:10593000406816F014FD002018F096FD0E4800682F
:105940001DF082FA51EC100B24F054FE08EE100A00
:105950000A4800681DF078FA51EC100B24F04AFE5A
:10596000F0EE480ABDEC028B00EE100ABDE81040D4
:105970001FF00ABF2C0000209C000020980000208F
:105980003038092801D8012070470020704730388E
:105990000A2801D201207047002070472DE9FC5FE2
:1059A0009B460CAB8A468146DDE9116093E81210F4
:1059B000DDE90F575FEA80784FF030031AD45EB10B
:1059C0005FEAC07808D000F00C0858EA0C0803D051
:1059D000761E01E00B55641CBC4204D2202CF9D386
:1059E00001E00B55641C5FEAC07803D0B44201D2D9
:1059F000202CF6D35FEAC06825D55FEA40580AD468
:105A00004CB1BC4201D0B44205D1641E03D0102D6C
:105A100003D1641E04E0102D02D0022D0AD00EE046
:105A2000850603D4202C1ED2782506E0202C1AD21D
:105A3000582502E0202C16D262250D55641C202C1E
:105A400011D20B55641C202C0DD2BCF1000F01D0DB
:105A50002D2306E0430701D52B2302E0030702D5DF
:105A600020230B55641CCDE900BAC8461546814673
:105A70008B46AA46800714D1274607E02A46DDE96F
:105A800000316D1C2020C446E0477F1CB742F5D38F
:105A900007E02A466D1C641EDDE900311BF8040096
:105AA000C047002CF5D15FEA897006D409E02A4688
:105AB000DDE900316D1C2020C047A5EB0A00B04293
:105AC000F5D32846BDE8FC9F2DE9F04F8FB09946ED
:105AD0008B46DDE91818DDE91C63DDE91A479246BB
:105AE0008646002209B923F01003580507AD00D5FA
:105AF000C9B1B1FBF4F004FB1010C0B20A2801D206
:105B0000303009E05FEA836C02D54FF0410C01E0D0
:105B10004FF0610C60440A38B1FBF4F1A854521CF8
:105B200009B1202AE5D3CDF80880CDE90563CDE998
:105B30000052CDE903474B46524659467046FFF79F
:105B40002DFF0FB0BDE8F08F2DE9FF4F8FB01CACDB
:105B5000DDE9239594E8030820AC94E8C004002410
:105B600050EA010201D125F010056A050DF11C086B
:105B700002D550EA010217D032463B46FAF762FCE2
:105B8000D2B20A2A01D2303206E0AB0601D5412357
:105B900000E061231A440A3A08F80420641C50EA21
:105BA000010201D0202CE7D3CDE90084CDF808B064
:105BB000CDE90595CDE9036A0FAF97E80F00FFF730
:105BC000EDFE13B0BDE8F08F9A4200D288547047C2
:105BD000704770B50D46040011D08DB100F067F824
:105BE00000280BD0616800690AF0F2FA0646E16B02
:105BF00028468847E1680844E060304670BDFEE70B
:105C0000FEE72DE9FF4114460E4605460A461F46AB
:105C100021466846DDF8288009F009F800281AD0E6
:105C2000019861682268411A009808FB0151821AA4
:105C3000551831683844441A684608F0E6FF0021D8
:105C400007E0625C6B5C1A44FF2A00D9FF226254B1
:105C5000491C8142F5D3BDE8FF8110B502004FF029
:105C600000000CD04B1E194200D0FEE70A44521E21
:105C70009A43B2F5803F02D20C2A01D9104610BDDA
:105C80000C2010BD08444A1E401E9043114200D013
:105C9000FEE7704710B5402013F0A8FB040005D0C4
:105CA0004022002113F0D3FC204610BDFEE72DE971
:105CB000FC410D4604002AD055B304F1240080466F
:105CC00018F057FA009008B30769616838460AF07F
:105CD0007FFA064629463846626813F0FDFB04F158
:105CE000300013F0A8FA019098B10422694613F02D
:105CF000F3FB2046009906F053F8042201A913F0A3
:105D0000EBFB2146304662680AF072FA07E0FEE7D4
:105D1000FEE74046009918F0F6F900200090009840
:105D2000BDE8FC812DE9F0410F4601210025044624
:105D30002E46C16309E01A4919F0E2FB08B16D1C57
:105D400002E0E06B401CE063761C57F8260010B1BF
:105D500001780029EFD1A06BA8421FD0206B00264C
:105D600010B110F069FD2663606B10B110F064FD96
:105D70006663280113F03AFB206338B1680013F022
:105D800035FB606318B1216B11B102E0FEE7FEE75D
:105D900000256A00002113F05AFCA563BDE8F081DC
:105DA0001CFD000810B5044690F85400E26BC107D2
:105DB000616C04D121B14B1C18D0491E6164A9B992
:105DC0000AB1C10712D02146144813F0D9FA00F0E5
:105DD00027F8216909B120468847616909B1204641
:105DE00088472046BDE8104010F026BD216C49428E
:105DF0006163002A10D0C10702D1A16B49426163DF
:105E0000411C61F3000084F85400E16A606A616239
:105E1000E062206B2263E06310BD00008C4F002025
:105E200010B50A4C012084F8A40004F1AC0013F072
:105E3000DDF90028D4F8A80003D0BDE810401BF01D
:105E400033BBBDE810401BF01DBB0000E04E00203E
:105E50002DE9F0413D4D95F8A50038B15FF0000007
:105E600085F8A5003948AC30074664E00120F7E723
:105E7000206D1BF0A5F9616B084460631BF0A6F967
:105E80002065002085F8A40094F8540095F8A5102A
:105E9000C0F340028A4254D061F3410084F85400B8
:105EA00041071ED4616B002941DB000709D4A169B9
:105EB00039B120468847616A01446162E16A084459
:105EC000E06220461EF0B8F8E16809B12046884734
:105ED00094F8540040F0040084F8540020461DF06B
:105EE000CBFF606B002822DB216B884200DD616301
:105EF000216A20468847A16A0646B1420DD0A662B3
:105F0000626812B131462068904795F8A40088B9BC
:105F1000A2682AB131462046904795F8A40048B9B6
:105F2000D4E90C0181420CDB2046FFF73BFF95F8DA
:105F3000A40030B1384613F059F9040098D1BDE8F7
:105F4000F0812146384613F063F9F6E7E04E002071
:105F500070B5044640680D4608B1FFF7F9FF2268A6
:105F6000002A04D029462046BDE87040104770BD85
:105F700070B50D6806460C46286838B1296AC90212
:105F800004D5206021463046FFF7F2FF2146304617
:105F90002560BDE87040FFF7DBBF08F005BC08F0E6
:105FA00049BC000010B5416C96B0044601B3684688
:105FB00007F022FF2146684607F0B8FF0F49684600
:105FC00007F09EFF6846616C07F092FF01220021F6
:105FD000684607F0A5FF0A49684607F093FF09499C
:105FE000684607F07EFF684607F0C2FF16B010BD96
:105FF00016B0BDE810401CF0CBBE0000152E020804
:10600000BDDE0008172E020810B50446406882085D
:106010000AD0496821F00301091D08446060204648
:1060200000F042F8204610BDFEE74068103120F035
:106030000300884201D301207047002070472DE9FA
:10604000FC47054648680C4620F0030001AA694653
:106050001BF064FEDDE9007005EBC71101EB800960
:106060008046D9F83C0060B164B1C4E9020504F18E
:106070000806C46030460421FFF704FE864202D0C1
:10608000FEE7FEE7FEE7C9F83C400120296900FA77
:1060900007F21143296105EB870100FA08F04A690C
:1060A00002434A61BDE8FC8710B5044600F087F85A
:1060B000046010BD2DE9FC4706464FF000000D00BE
:1060C00000900746019042D00C46E9460DF10408C5
:1060D000802907D3084622F053F9411F0120884048
:1060E000401E04444246494620461BF017FE009CD1
:1060F0000A2C2CDA06EB8400019A40694FF0FF313C
:1061000001FA02F210400CD1641C3069A140084031
:106110001DD022F02DF90446009006EB8000406966
:1061200078B122F025F9034606EBC411019001EB8A
:106130008000C76B5FB1786820F00300A84201D2ED
:10614000FEE7FEE739463046009A1DF0D1FE38469C
:10615000BDE8FC8710B50446FFF7A6FF416841F093
:1061600002014160606840F00100606010BD10B540
:10617000044600F024F8416821F0020141606068A3
:1061800020F00100606010BD70B506460D4608465F
:1061900000F015F8040010D02079C0070BD0686813
:1061A00080080BD02146304600F03CF821462846B6
:1061B000FFF72AFF0546284670BDFEE7FEE7426866
:1061C00000F1080122F00300001F0844910800D1EB
:1061D000FEE7704770B506460C004FF000001ED079
:1061E000F2B120791546C0071BD011462046FFF7B3
:1061F0001CFF78B12946204600F025F805462046C8
:10620000FFF752FF6868294640F002006860304698
:10621000FFF715FF2046FFF7AAFF04F1080070BD45
:10622000FEE7FEE77CB5054648680C4620F0030013
:1062300001AA69461BF072FDDDE9002321462846CC
:106240001DF056FE7CBD2DE9F0410D46044600F1DF
:106250000801281F0E18606806F1080720F00300E7
:10626000401BA0F1040838460421FFF70BFD8742CC
:1062700000D0FEE7606820F0030108EB0500001D78
:10628000814200D0FEE7307900F0030040EA0800C8
:10629000706020F003000C2800D2FEE7207900F0A7
:1062A0000300284360603046FFF754FF3046BDE8E6
:1062B000F08138B5044611F09FFB054611F0D7FB7D
:1062C0000028204605D0616C216416F048F80120B2
:1062D00038BD0FF007FE002820461ED00FF0B2FC9C
:1062E000D4E9100181420CD06064206C00906A46B1
:1062F0002021204617F0E3F80128E9D1204616F0C6
:106300002EF8284611F0C2FB0428E0D1204614F0F4
:1063100078FC002110F017FED9E70FF041FED6E718
:10632000002802D0C01C20F00300704710F084BA8F
:10633000C01C13F05BB82DE9F04104460068154617
:106340001346476A0E4600222046B84701280FD15F
:106350000020BDE8F0812946204600F013F800280F
:10636000F7D020682B460022476A31462046B847BE
:106370000228F0D020682A46314603692046BDE84D
:10638000F041184770B5044600680E46026A204680
:106390009047050010D020683246294643692046C0
:1063A0009847284609F00FFFA269314690472846D2
:1063B00009F000FF012070BD002070BD2DE9F04FF5
:1063C0000C4685B00546002114F03FFB58B321462A
:1063D000284600F08DFA2146284600F069F8002191
:1063E000284615F02BFA83460021284615F074FA4A
:1063F00004900021284615F0F8F801281BD000274A
:106400000021284615F0DCFB80460021284615F0C7
:1064100070F96FF040490646C8450ED1688D0005F9
:106420000BD401200AE005B02046BDE8F04F202241
:10643000002113F00CB90127E2E70020804628462E
:1064400014F0A1FB824628460021822215F06EFA44
:10645000C2B22369A1682068CDE90031CDE9020705
:106460005B464146504605F0F1FFA0614E4504D120
:10647000688D400501D4012600E00026284614F06E
:1064800071FB074628460021832215F04FFAC2B25D
:10649000606900256368E1688DE82B003146384665
:1064A000049B05F0D3FFE06105B0BDE8F08F00006C
:1064B0002DE9F34F81B00C46019805F053FA060020
:1064C0004FF000081ED1019814F0F0FB05F04AFAD5
:1064D000070074D0019805F049FA8146019805F04B
:1064E00049FA80468500281D12F080FF06462A469C
:1064F00007EB890112F0F0FF6FF0604146F82810B9
:106500004FF00108019814F03EFB8346304600F03E
:106510001DFF2061800012F069FF2060206980006B
:1065200012F064FF0025DFF82CA1A06038E056F8D7
:106530002510DFF82491514531D100271FE039465D
:10654000019814F082FA4549009015F010FCA8B9A2
:10655000009805F00FFA012810D1009805F006FA0E
:10656000A8420BD1009815F0B5FB4946484501DA21
:10657000084602E0009815F0ADFB81467F1C0198AB
:1065800014F0A2FAB842DAD8B9F1000F03DBA1681F
:1065900041F8259003E0A168002041F825006D1C1A
:1065A0002069A842C3D8DFF8AC90002509F10109A1
:1065B000C9F1000352462F4628469A4614E046E0A9
:1065C00056F82010494503DB6B1803EB0A050AE077
:1065D000914204D1A16851F820100F4403E0A36850
:1065E0000F4443F82010401C21698142E8D8002163
:1065F000019815F023F92169C1F1010200FB02B0F5
:10660000C01B00D50020002114E000BF56F8212057
:106610004A450EDB02EB0A0300FB03F205EBD577DC
:1066200002EB670292FBF5F2A768ED1A801A47F8B1
:106630002120491C22698A4201D9002DE6D1B8F1F6
:10664000000F04D03046BDE8FE4F10F0F5B8BDE8AD
:10665000FE8F00009AFFFF1F010000E0010006000E
:106660002DE9FC5F054614F071FC8346A86808B16B
:106670000021C1610021284615F015FA0190002182
:10668000284615F083F98246284614F06FFF01462C
:1066900001982E4C014401EB0A07284614F014FA25
:1066A0008046002639E0A868DFF8A09028490068F5
:1066B00050F82600009015F05AFB68BB009815F0C2
:1066C000AFFEE0BB0021009814F074FFB8B30128BE
:1066D00036D0022834D0032832D00021009815F09B
:1066E0007EFA60B90098143008F080FA019900EB46
:1066F00001090021009815F035F848448146002131
:10670000009815F014F84844A04205DB00210098D9
:1067100015F00DF800EB0904761C4645C3D3A868B4
:1067200010B1CBF10001C1616FF06040C44203D0F1
:1067300004EB0A00B84200DA3846BDE8FC9FFFE7E8
:106740000098A969006A401A401CD7E7010000E0E0
:10675000010004002DE9FE4F054614F0F1FB029004
:10676000A86808B1002181610021284615F06CF964
:1067700000900021284615F038F98346284614F089
:1067800003FF00EB0B010098DFF85C9101EB0008C0
:106790004C46284614F098F907460021284614F084
:1067A00018FF01284FF0000645D082E0A868CA46CD
:1067B0004E49006850F82600019015F0D8FAC8BB81
:1067C000019815F02DFE20B10198E9694069081A79
:1067D00014E00021019814F0EDFE58B1032809D00F
:1067E000062807D0082805D00021019815F0F4F9F3
:1067F00030B112E00199E8694969401A401C0BE088
:106800000198143008F001FA009900EB010A002108
:10681000019814F095FF504482460021019814F02D
:106820008FFF5044A04205DB0021019814F088FF3F
:1068300000EB0A04761CBE42B8D34C453FD05C4402
:106840003DE0A868CA462949006850F82600019032
:1068500015F08DFA60BB019815F0E2FDE0BB002158
:10686000019814F0A7FEB8B3012836D0042834D01C
:10687000072832D00021019815F0AEF958B90198D7
:10688000143008F0C2F900EB0B0A0021019814F053
:1068900060FF504482460021019814F05AFF504492
:1068A000A04205DB0021019814F053FF00EB0A041D
:1068B000761CBE42C5D34C4501D000980444A8685C
:1068C00010B10299494281614C45404602D044458D
:1068D00000DD2046BDE8FE8FFFE701986969C069C9
:1068E000401A401CD6E70000010000E0010004004F
:1068F0002DE9F34F81B00C46019805F0EAFB060044
:106900004FF000081ED1019814F0D0F905F0E1FB1A
:10691000070072D0019805F054FC8146019805F0FB
:1069200054FC80468500281D12F060FD06462A466C
:1069300007EB890112F0D0FD6FF0604146F8281096
:106940004FF00108304600F001FD6061800012F058
:106950004DFD60606069800012F048FD0025DFF8A1
:1069600038A1E0603AE056F82500DFF83091504554
:1069700033D10027DFF828B11FE03946019814F021
:1069800064F85946009015F0F2F9A8B9009805F09E
:106990001CFC012810D1009805F013FCA8420BD173
:1069A000009814F033F94946484501DA084602E0F8
:1069B000009814F02BF981467F1C019814F084F89C
:1069C000B842DAD8B9F1000F03DBE16841F825904D
:1069D00003E0E168002041F825006D1C6069A842D1
:1069E000C1D8DFF8B490002509F10109C9F100030D
:1069F00052462F4628469A4614E04AE056F82010A0
:106A0000494503DB6B1803EB0A050AE0914204D108
:106A1000E16851F820100F4403E0E3680F4443F8A5
:106A20002010401C61698142E8D80021019814F0CF
:106A300053FF8346019814F095F801466069C0F150
:106A400001020BFB0210C01B00D50020002113E047
:106A500056F821204A450EDB02EB0A0300FB03F245
:106A600005EBD57702EB670292FBF5F2E768ED1ACA
:106A7000801A47F82120491C62698A4201D9002DF9
:106A8000E6D1B8F1000F04D03046BDE8FE4F0FF05C
:106A9000D3BEBDE8FE8F00009AFFFF1F010000E09B
:106AA0000100060070B5044600216E2214F03EFF7E
:106AB000D8B9204600216C2214F038FF4FF48075BD
:106AC000A84212D1204600216D2214F02FFFA842C7
:106AD0000BD120460021712214F028FF28B920464E
:106AE0000021722214F022FF08B1022070BD20465E
:106AF0000021602214F01AFFC0B2FF280DD12046F9
:106B00000021732214F012FF38B9204600216722B9
:106B100014F00CFF10F0FF00E8D0012070BD2DE94B
:106B2000F041044606A81D46174690E84C0002298D
:106B30000FD003290BD12946384619F0D7FC05465A
:106B4000304608F062F8401B216808442060BDE828
:106B5000F0812946384619F0C9FC0546304608F050
:106B600054F800EBD071491005EBD570A1EB600033
:106B7000EAE700002DE9FF4F95B0C878269CC007D2
:106B80000D46002801D0FE4800E0FE48099001D0E3
:106B9000FD4800E0FD480F9001D1FB4800E0FB48B4
:106BA000109001D0FA4800E0FA48039001D0FA486A
:106BB00000E0FA48069001D1F54800E0F54805905C
:106BC00001D1F54800E0F5484FF01409049069E060
:106BD000D4E901124FF0000BA1EB020358465946CD
:106BE0004FF00C0E0FE000BF01EB4102266909EBEC
:106BF000C20C16F80CC05FEACC7C08D00EEBC202C7
:106C0000B2589B1A491C8F42EED8002144E04FF045
:106C1000100C0CEBC202B2581044F3E701EB410632
:106C2000276909EBC60A17F80A20D20733D1E8B35F
:106C30004FF0100C93FBF0F20CEBC60CCDF848C0F3
:106C400057F80C804FF0080C08FB02F804220CEBFC
:106C5000C60C02EBC60257F80CC0BA58CDF820C0DB
:106C6000C44500DDC446624503DC089A424500DDA8
:106C70004246424504D04FF0010C47F80AC0E346B3
:106C8000D4F810C00EEBC6064CF806202769129EF9
:106C9000BE59801B9B1A491C62698A42BED8BBF14F
:106CA000000F02D06769002F92D100E028E0002198
:106CB000159814F0A0FC012823D00021002088465C
:106CC0000D900E900EA90DA8CDE900012878E3687B
:106CD000626824991BF075FBE87810EA080F05D06C
:106CE000159813F050FF0D9908440D9017991598B9
:106CF00013F0ABFE0646DFF8A8926FF0704B3AE156
:106D0000FEE70121DAE7A749304615F030F8002800
:106D10007AD10021304614F0E3FCE8B3002738466E
:106D200061690FE0226900EB400352F83320B24260
:106D300007D100EB40020C20216900EBC2000F5884
:106D400002E0401C8142EDD8E878C007708D04D085
:106D500020F4806040F4006003E020F4006040F420
:106D60008060708506F114000F9982468847B8420A
:106D700024D0304615F0F3FA70691190B069129082
:106D8000F0691390306A1490099A3946504690473A
:106D900011AA2E21304600E00CE016F090FB3046A0
:106DA00013F084FF3246272116F089FB304615F098
:106DB000D6FA03E0708D20F4406070856878012871
:106DC00023D0022804D0059A00213046904727E0BE
:106DD000109906F1140088472168059A491C21F092
:106DE0000101081A00EBD0704FEA600A002130461A
:106DF00090470746049A002130469047381A00EB26
:106E0000D0710AEB61000BE0ADE0109906F11400BF
:106E100088472168049A0F1A002130469047381A93
:106E20000790E87810EA080F06D00F9906F11400D1
:106E300088470D99081A0D90304600216A2214F0F7
:106E400075FD0746304600216B2214F06FFD824627
:106E5000304614F03FFF0C90304613F0D7FE014649
:106E6000C7F3417001280DD127F0C040484509DC27
:106E7000B0F1805F01DBABEB00000C9A5043642261
:106E800090FBF2F7CAF3417001280CD12AF0C04000
:106E9000484508DCB0F1805F01DBABEB0000484304
:106EA000642190FBF1FA71692298401A0744B16994
:106EB0002398411A01EB0A000190E878C00706D038
:106EC000039A0021304690470D99084400E0079846
:106ED00000EB070AE878C00701D0079805E0039A9D
:106EE0000021304690470D990844019947185AEA05
:106EF000070019D0304615F032FA716901EB0A002B
:106F00007061F16901EB0A00F061B0693844B06169
:106F1000306A38443062304615F021FA00233A4690
:106F20005146304615F0C4FAE87810EA080F14D13B
:106F30000F9906F1140088472599039A08440E9981
:106F400047180021304690470744069A00213046F2
:106F500090470D993844084404E00E992598084458
:106F60000D99081A0D90E87817AAC0F380011598BA
:106F700004F08EFF0646002E19D0DDE9170113E05C
:106F8000E7EE0008DDEE00080BEC0008EDEB000872
:106F90004DB7010871B701085FB701083BB7010899
:106FA000FEFFFF1F0100060088427FF4ACAE19B05F
:106FB000BDE8F08F2DE9F04F91B00E0005463AD0B4
:106FC000AE61286808B10FF037FC06EB46010620D9
:106FD00000EB410012F00AFA286018B3022101EB1D
:106FE00046010144E960042101EB86010144C5E941
:106FF000010101210024012E15D03001103012F0C2
:1070000019FAA346B100CDE9051B8246C1F101077B
:1070100000EBC600891000F108095C46CDF834B0D9
:10702000099196E0FEE7B4220270E8680480E868FF
:107030004180A868048011B0BDE8F08F4FF00008CF
:10704000002F05DC0699032000EB4100074408E00F
:10705000DDE905010A1A052101EB4201401E0F443A
:1070600005900698401C069005A800F0DAF870B16B
:10707000059809AB82100DA943F8282000F0030001
:1070800041F8280008F10108B8F1040FD8DBB8F185
:10709000040F64D10C99099888420AD14AF8240057
:1070A00049F824B0DDE90D010144DDE90F02104487
:1070B00018E00A99884218D04AF8240049F824B008
:1070C00069680D9808556968000108550998641C9D
:1070D000401E4AF8240049F824B0DDE90E010144BD
:1070E0001098001D084469682CE00B994AF82400A8
:1070F000884249F824B0DDE90D01084411D06968DF
:1071000008556968000108550998641C401E4AF832
:10711000240049F824B0DDE90F010844083069680B
:1071200010E00F990844696808556968000108551E
:107130000998641C401E4AF8240049F824B01098AD
:1071400069680C300BF1010B08556968000108559E
:10715000641C05A800F065F800287FF46FAF0AEB07
:10716000840140F2D320464351F8041CB0128142FE
:1071700005D109EB840151F8041C814219D0A6EB1A
:107180008021B1F5007F03DC494341F3CF3106E0B4
:10719000C1F58061494341F3CF31C1F10F014AF894
:1071A000240049F824006868015568680901015500
:1071B000641CA01E0DE000BF59F820204AF82420CE
:1071C0005AF8202049F8242069680A5C0A55401EB4
:1071D000641C0028F0DAEB680021084619801AE0E8
:1071E000EA6822F81100AB683AF8202023F8112051
:1071F0000AE0AB685AF8202033F81160964200DAB2
:10720000324623F81120401C59F820208A4201D12F
:10721000A042EEDB491CA042E2DB50460FF00CFB23
:1072200009E703C8814201DC012070470020704754
:10723000012070477CB504460FF070F806462046E2
:107240000FF068F80546304613F030FD0446302D47
:1072500023D00B2D4DD110F0CFFB10B1007A0128B7
:1072600047D06946304613F083FD94F8300010F0A3
:107270000C0F30461BD013F086FC0546002120463B
:1072800014F0CBF90128009805EBD5710CD000EB78
:10729000610000BF90FBF5F512E0E16A02B0002248
:1072A000BDE8704018F0A4BEC0EB6100F2E713F037
:1072B00059FC019900EBD07201EB620191FBF0F5F2
:1072C000002D00DA0025E06A0026A84200D0012641
:1072D00010F092FB08B1012200E00022294620466E
:1072E00018F086FE002E04D000222021204616F041
:1072F000E6F87CBD30B5002822DA8B1A002B00DCC2
:10730000531A64225343C0F30901B3FBF1F1C0F3F4
:107310000953C0F38922C0F3095000EB800003EB4E
:1073200083034000B1EB430F01D20C4600E004465A
:1073300002EB8205B4EB450F03D202EB8200400062
:1073400030BDB1EB430FFBD2084630BD01460020F3
:107350006FF0604200E0401C51F820309342FAD1B7
:1073600070471FB5044690F8640000F001008842A1
:1073700025D094F8640011B140F0010001E020F044
:10738000010084F8640004F15001684607F0BAFB7C
:10739000E06A0099426911440091019980690844AA
:1073A0000190E06A0299406908440290E06A0399FA
:1073B0008069084403906946204614F0EBFF1FBD26
:1073C00008B50846114609F096FC0090BDF800008B
:1073D0009DF8021040EA014008BD00002DE9FC5F65
:1073E000088C0C46C0F307208F6C09F0A5FC814681
:1073F000208D636A81B2CA00B2FBF9F0072202EB6A
:10740000C002D6081A0C01FB02FA02FB00F599B281
:107410000E23364800960AF04DFC060007D0206A7D
:10742000D6F81080000C000704D5386A18E0002058
:10743000BDE8FC9F207C012801D080B115E001A8A7
:107440000090534642460C21386804F0A3F810B966
:107450000199514509D030460AF06DFCE7E7E06834
:1074600052460169404612F037F8208CC0F30720DD
:107470000E2837D008EB0A00A0F1010B08EB05003D
:10748000A0F1010A012000FA09F0401E002100F0DD
:10749000FF0E0B4624E000BF9BF800004A46C840A0
:1074A00010EA0E000FD080460AE000BFC2F1080CBF
:1074B00000FA0CFC4CEA080C4A440CF0FF08D2B26B
:1074C000082AF3D340468AF8000001EB0900C1B254
:1074D000082902D30021ABF1010BAAF1010A5B1CC0
:1074E000AB42D9D3FE610120E662A1E7D84F00206C
:1074F0002DE9FC478F6C086A0E46D7F800A0C0F350
:1075000007254FF48079072D0DD0082D0DD0092DBA
:107510000DD00A2D0DD0002189008846C0F3C0404F
:1075200048B1386A28E00221F6E70421F4E7102187
:10753000F2E74946F0E7307C012801D0D8B115E0E8
:10754000084611F053FF040009D001A800904346FB
:1075500022460C21504604F01DF820B900E0FEE759
:107560000199414505D020460FF066F90020BDE89D
:10757000FC877C6001E0F06804693463072D09D062
:10758000082D09D0092D09D00A2D09D000207063DB
:107590000120ECE70220FAE70420F8E71020F6E7E4
:1075A0004846F4E72DE9F0430024DDE90759D617F2
:1075B000072808D0082810D0092819D00A2821D077
:1075C0000020BDE8F08302EB567405EBE40502F001
:1075D00007020120C2F1070416E002EB96740220B4
:1075E00005EBA40502F003020624A4EB42040BE021
:1075F00002EBD274042005EB640502F00102A0EB5B
:10760000820401E00820154401228240521E1FFA24
:1076100082FC0026C0F1080211E02F7809EB8608F1
:10762000E74007EA0C0701EB8707241A3F6864B2BA
:10763000C8F80070002C01DA14466D1C761C9E42BE
:10764000EBDB0120BDE710B10268D2691047FEE70D
:1076500070B505460EF05EFE044628460EF0B4FEF8
:10766000352C07D1D0F8F802002803D0BDE87040CF
:1076700019F01ABF70BD000038B5054609480078FA
:1076800058B10092888983B2088982B2888884B20E
:107690000888214680B2FCF739FF2846BDE838400B
:1076A00009F062BDCC0100202DE9F0410446C0691B
:1076B0000E4610B10020BDE8F081012200213046C5
:1076C0000AF038FE05004FF0FF3716D030460BF0B9
:1076D0009BFA90B10220A86405F13800E561C4E985
:1076E0000160204603F0E8FBE16903208864002084
:1076F000E0610AF0BFFD0120DDE73846DBE74143EA
:1077000002EBA121414303EBA121414388127047C1
:107710007CB5044617F096FC94F8A01004F12C05F3
:1077200041F0010184F8A010F8B101281DD0022811
:107730001DD110F061F9694610F07CF90322694609
:10774000204616F093FA0021204613F05AFF012834
:107750000ED00026204605F05BFE014694F84C0052
:107760000E40B04206D0012205E0C4F89C507CBD1A
:107770000126EFE7002204F1380089B3009902B333
:10778000D4F884209142F0DBE26F91423ADC626FE0
:10779000E16F009B891A01EBD17102EB6102D11AF2
:1077A000002900DC991AD4F88460D4F88C20921B4C
:1077B00002EBD27206EB6206F21A002A4ADC9A1B2E
:1077C00048E0D4F88C209142CFDC626F914219DB03
:1077D000DDE700BF44F89C5F207920F0020006E05E
:1077E00007E000BF44F89C0F207940F002002071B0
:1077F0007CBD01994AB1D4F890209142B5DCA26FCA
:1078000091420ADAC4F89C007CBDD4F888209142E9
:10781000ABDBD4F880209142F4DCD4F88020A16F57
:10782000521A02EBD27201EB62020199511A00293D
:1078300001DC0199891AD4F89030D4F888209B1A79
:1078400003EBD37302EB6303019A9A1A002A01DC5B
:10785000019AD21A8A42C5DABCE72DE9FF4FB7B0C8
:10786000154637981F460C468268DDF81081469E03
:107870001DA807F0DCF900287DD01DA807F0C5F988
:107880001C9005A82C22002111F0E1FE1C9811F09B
:10789000ADFD03900B9000202190229023900123B6
:1078A0004246294624A80DF049FD24A82190002F26
:1078B00007DD00233A4621462DA80DF03FFD2DA8F7
:1078C000229010A805900D90BDF81401ADF8290084
:1078D0009DF816018DF82B008DF828602068C119DD
:1078E0002868814200DD08461890A068A968C01B7E
:1078F000884200DB08461A906068C11968688142B6
:1079000000DD08461990E068C11BE868814200DA92
:1079100008461B9018A807F078F961686A689142D8
:1079200001DC012100E000218946E168EA6891421A
:1079300001DB012100E000218A4621682A6891428A
:1079400001DC012600E00026A168AA68914201DB63
:10795000012200E00022904606EA080101EA09013E
:107960004FF0010B11EA0A0F03D0322801DA4FF071
:10797000000B012000E030E18DF8300019EA0B0F18
:107980000CD0189810901A9812906068119068683E
:1079900005A9401E139037980CF027F91AEA0B0F2F
:1079A0000CD0189810901A981290E86805A9401CFD
:1079B0001190E068139037980CF017F92968A868BF
:1079C000814205DB96B1B8F1000F02D0206812E0C9
:1079D00066B120681090286805A9401E1290199879
:1079E00011901B98139037980CF0FFF8B8F1000F26
:1079F0000CD0A868401C1090A068129019981190A3
:107A00001B98139005A937980CF0EFF81D98BBF15F
:107A1000000F109006D018981F9A411E8A423EDA35
:107A200010463DE01F98129068686168401AB8429D
:107A300000DA3846814600252EE060684619E06885
:107A4000A0EB05081E98B04202DD2099414522DBDB
:107A5000FF211C9A039811F0FAFD1C980090334600
:107A600021A8109A03990DF04FFB8DF830001E9855
:107A7000B04205DC119605A9139637980CF0B5F8BD
:107A80002099414507DBCDF8448005A9CDF84C800D
:107A900037980CF0AAF86D1C4D45CEDB92E0401EE5
:107AA000129010A807F0B1F8051E39DD56EA09005A
:107AB00019D01E9C14E011942A46FF2113940398B8
:107AC00011F0C5FD0095234621A8109A03990DF0E9
:107AD0001BFB8DF8300005A937980CF086F8641C64
:107AE0001998A042E7DC56EA0A0619D01B9C13E05D
:107AF00011942A46FF211394039811F0A8FD0095D4
:107B0000234621A8109A03990DF0FEFA8DF8300053
:107B100005A937980CF069F82098641CA042E7DAB0
:107B200012991D98491C884201DD014601E0129915
:107B3000491C10911A99491C884201DC1A98401C72
:107B400010901F98129010A807F05FF8051E39DDFD
:107B500058EA090019D01E9C14E011942A46FF210E
:107B60001394039811F073FD0095234621A8109AF1
:107B700003990DF0C9FA8DF8300005A937980CF07B
:107B800034F8641C1998A042E7DC58EA0A0019D0BE
:107B90001B9C13E011942A46FF211394039811F0C3
:107BA00056FD0095234621A8109A03990DF0ACFAD2
:107BB0008DF8300005A937980CF017F82098641C50
:107BC000A042E7DA24A80DF0DDFA002F02DD2DA88F
:107BD0000DF0D8FA03980EF02FFE3BB0BDE8F08F01
:107BE0002DE9FF4794B015460C46824604A82C2286
:107BF0000021209E11F02BFDCDF810D0BDF85C00C7
:107C0000ADF825009DF85E008DF827008DF8246002
:107C100060686968884201DC012700E00027E068AD
:107C2000E968884201DB012600E000262068296817
:107C3000884201DC012100E000218946A168AA6890
:107C4000914201DB012100E000210090A068029038
:107C50006068019068688846401E03901FB104A9BF
:107C600050460BF0C2FFE868401C0190E0680390AA
:107C70001EB104A950460BF0B8FF20680090286898
:107C8000401E02900FB1686800E0606801900EB17C
:107C9000E86800E0E0680390B9F1000F03D004A9A0
:107CA00050460BF0A2FFA868401C0090A06802900C
:107CB000B8F1000F03D004A950460BF096FF18B09E
:107CC000BDE8F0872DE9F04F8B46A2F57F41A1B0CA
:107CD00091460646FF3942D0F46A208D804698428C
:107CE00004D02385608D40F0080060854FF4802A21
:107CF0005146204613F01CFF07465146204613F01C
:107D00003BFF054638460EF08CFD0746304603F033
:107D1000AEFF80697A1909FB0200014605EBD570B8
:107D2000A1EB60001D9038446D1E28441F90F06A3E
:107D300041691C91C0691E9068460BF017FD6A46A8
:107D40005146204614F07DF91CAA694658460BF0AE
:107D5000F7FAA4F82880608D20F00800608521B033
:107D6000BDE8F08F2DE9F04F0E46A2F57F41A5B09A
:107D700090460546FF395CD0EC6A278D9F4204D0BF
:107D80002385608D40F00800608503A80AF0AEFCF2
:107D90004FF4802903AA4946204614F094F8494636
:107DA000204613F0E9FE1190284603F060FF05001D
:107DB0003FD00B980EF035FD119AA969131808FBF6
:107DC000031119911146199A01EBD171A2EB6101CE
:107DD000119A19911144401E08441B906069189033
:107DE000E0691A9018AA06F118011FA806F01FFFF3
:107DF000D0B118360DF17C0C96E80F00804689460C
:107E000092469B469CE80F0086E80F002846183EE5
:107E100010F022FB0A9005F1140203A930460AF083
:107E200034FC183686E8000F2785608D20F00800A6
:107E3000608525B0BDE8F08F7FB50446D0F8A85224
:107E400004E000BF0AF01EFA0AF060F9A86B0028EF
:107E5000F8D1204609F012FA18B12648006921F03D
:107E6000E8FD01202063A16BC90702D0A16B89073F
:107E700000D400206063606B08B1012600E000269A
:107E8000A06A20B3286821696A460569D4F800030E
:107E9000084400906169D4F8040308440190216902
:107EA000D4F80803084402906169D4F80C0308442C
:107EB00003903A21204609F083FAA36A2A466946CC
:107EC000204698476A463B21204609F079FA204629
:107ED00009F0D4F900280BD094F83900012801D119
:107EE000002E05D0616AE069814200D1206A60629B
:107EF0007FBD0000E04E002038B540680C46010C04
:107F0000491E83B200220091114620465B1E06F0F6
:107F1000E0FF38BD2DE9F047B8B005460EF0FEF998
:107F2000044628460EF031FA8246E06A10F094FAD0
:107F3000054694F86400C00771D004A80BF016FC45
:107F40004FF4C02904AA4946204614F07AF804F1F7
:107F50005001684606F0D6FDE06A00994269114476
:107F60000091019980696A4608440190E06A02998B
:107F7000406908440290E06A0399806908440390CC
:107F800004A950460BF0DCF94946204613F0A5FB46
:107F900006464946204613F07EFC8719494620468E
:107FA00013F0C1FC4FF000081E490644CDF8D48000
:107FB000CDF8D880206E0968284488470246206E94
:107FC000411935A811F088FA0098582238440090D9
:107FD0000198414630440190E06A13F0A7FC054641
:107FE00020A80AF083FB20AA4946204613F06BFF25
:107FF0009DF83000022805D829462B9808F08CFE01
:1080000000280CD135A827909DF8CC006A4640F096
:1080100040008DF8CC0020A950460AF036FB38B05D
:10802000BDE8F087241203082DE9F04FEDB00546B6
:1080300038300E465E9011F06BF900287ED105F1C4
:10804000140206F1180168A806F0F1FD002875D0A9
:10805000183668AC96E80F0083462091CDE964237A
:1080600094E80F0086E80F003DA8183E0AF06FFE66
:108070004FF4C0243DAA2146284613F07EFF21A8D4
:108080000BF074FB21AA2146284613F0DAFF2146A3
:10809000284613F09BFD00EBD07047102146284680
:1080A00013F094FD00EBD0704FEA600A5E9811F077
:1080B000B6F890E040223DA94EA811F00DFA7022CA
:1080C00021A9684611F008FAA089ADF86401A07BE7
:1080D0008DF86601A089ADF82100A07B8DF8230002
:1080E000A08AC00502D5D4E900010BE0A2686FF0B8
:1080F000004082426BD066AB2846216908F0EAFA5C
:10810000DDE966016A6902EB0008A86900EB010974
:1081100027B1BAF1000F01D0012000E000206690E5
:10812000A8EB07005F9008EB07006190A9EB0A003D
:10813000609009EB0A006290207D00E056E0810724
:108140001CD0C00701D0686900E04046CDE9550960
:10815000207D800701D5E86900E04046CDE9570958
:108160000020519003904EA930460AF0B4FD669865
:1081700020B15FAA694630460BF0E2F8207D10F08E
:108180000C0F1ED0CDF85481207D400701D5A86981
:1081900000E04846CDE95608207D000701D5286A51
:1081A00000E0484658900120519003904EA9304677
:1081B0000AF091FD669820B15FAA694630460BF03F
:1081C000BFF83F98401C3F902398401C23902146C5
:1081D0005E9811F021F804007FF46CAFDDE96423B0
:1081E0002099C6F818B01C3686E80E006DB0BDE8C0
:1081F000F08F2DE9F04F884601F11802A5B0044632
:1082000000F114011AA806F012FD002872D008F13E
:10821000180114AD91E80D00D8F82410179185E8E5
:108220000D001AAE08F1180096E82E0080E80E0046
:1082300000212046C8F8245013F043FA05460021D7
:10824000204613F016FB28441E900021204613F010
:1082500058FB0544204612F096FC1390204612F07D
:1082600081FC129002A80AF072FD02AA00212046A9
:1082700013F083FE20460021322213F057FB00F05A
:10828000FF090021204613F01CFA824620460021F7
:10829000342213F04BFBC6B2204612F089FD239026
:1082A000204612F047FEA16EB9B3A1692944A1EBA3
:1082B000000B60690990E0690B90B4F86800002534
:1082C00007B2B9F1020F26D9BAF1000F23DDB007CA
:1082D00005D50021204613F014FB00B90125F00755
:1082E00019D020460021112213F020FB98B97F1EDF
:1082F0003FB210E055E0A16E1298491E6843B0FBF2
:10830000F1F058440A900C9002A9049540460AF0F6
:10831000E2FC6D1C2DB2BD42EDDBE06EC0B36169C5
:108320001E98002701442398B9F1020FA1EB000B1E
:10833000A0690A90206A0C90B4F86C0005B225D9A7
:10834000BAF1000F22DD700705D50021204613F099
:1083500090FA00B90127300718D5204600211322D2
:1083600013F0E4FA90B96D1E2DB20FE01398E16E90
:108370007843491EB0FBF1F0584409900B9002A9D4
:10838000049740460AF0A7FC7F1C3FB2AF42EDDBEA
:1083900014AD08F1180195E81D0081E80D00C8F83A
:1083A000244025B0BDE8F08F2DE9F047A0B0064687
:1083B0000DF0B0FF054630460DF0B0FF0446172D16
:1083C0002DD01A2D28D1206C002825D0E06B002854
:1083D00022D0A06C00281FD0E06C00281CD03046B2
:1083E0000DF0D3FFA16D054601F0030001287BD0FD
:1083F000890779D002280FD168460AF077F96A46D2
:108400000021204613F05FFDE06A079004F114029A
:10841000694628460AF039F920B0BDE8F0873046B1
:108420000DF0C4FF054600780228F5D0A06D4FF08E
:108430000106C143890755D000F00301022951D03C
:10844000C0F3840008F09BFCF0BB204600214422CE
:1084500013F06CFAC0B2FF2844D1606CA0BBA06CD2
:108460003102884207D1E06C884204D1002204F135
:108470001401686830E007A920460FF0C3F82046D1
:1084800012F0C4FB0746204613F024FC0146B4F862
:108490004820B4F84C0092B2009207AB80B2CDE90C
:1084A000010300233A4603A80EF06FFD03996069AB
:1084B000084403900499A0690844049005996069F0
:1084C00008440590069901E00CE00DE0A069002247
:1084D0000844069003A9686806F0C9FB10B1206B38
:1084E000002899D02E7097E701A809F0DFFF01AAB4
:1084F0000021204613F08DFCD5E90880D5E90667F8
:10850000814611A920460FF07DF8A06C0D90E06C1B
:108510000E90606C0C9094F85800C109BDF85000A2
:1085200061F30C30ADF85000B4F85800010B9DF821
:10853000510061F303008DF85100206B1B90E06A3D
:108540000890A269206C1044401E00906169E06BA5
:108550000B1816A882465B1E06F0BBFC20460021C5
:108560000C2213F0E3F91A90B4F85800C0F3032278
:108570000A2A10D2A06B0090514604F11400636BDC
:1085800006F09EF90DF1580C9CE80F000DF1700CEF
:108590008CE80F0007E00C2A0ED016AC94E80F0010
:1085A0001CAC84E80F001CAA01A9284609F02AFF88
:1085B000183585E8C0032FE705F1180104F114020E
:1085C000084606F034FBD4E90D12504606F074FC60
:1085D000E8691799411A206C091A491C91FBF0F2BD
:1085E0004243A8691699411AE06B091A491C91FB8C
:1085F000F0F14143504606F05FFC18350DF1700C68
:1086000095E80F008CE80F00BDF85000183D40F4CD
:108610000050ADF85000C6E72DE9F04FADF5117DE3
:1086200005460DF07BFE044628460DF0AEFE8F9009
:1086300001A9204612F0B8FA00216822204613F062
:1086400075F9054600216922204613F06FF90246AC
:10865000294601A806F0DEFA01A806F0D6FA09902C
:1086600001A806F0C3FA0790D4E90C10401A5FEA9B
:10867000000801D14FF0010894F870000027C0F302
:10868000C200012805D0022806D00799099888421F
:1086900001DB012700E00027204606F0DDFD1290F7
:1086A0000021204613F0DFF85D900021204613F0F2
:1086B000FBF85C900021204613F01DF95B9000212F
:1086C000204613F0A3F8059004F13C0001A90090A6
:1086D00006F0FDF9E16B5D986FF001050144E1637F
:1086E000616C5C98091A6164216C5B980144216497
:1086F000A16C0598091AA164009877B106F076FA82
:10870000042818DA0798A16900EBD07005EB600027
:1087100008442064001DA0640DE006F076FA0428E9
:1087200009DA0998616900EBD07005EB6000084434
:10873000E063001D6064009806F067FA0546009843
:1087400006F054FA2FB1A94604F14405C548009E2D
:1087500005E08146C44804F1400604F148050D9047
:10876000E26E501C14D0616E206BA36E091A181AA9
:1087700001FB09F100FB09F091FBF8F190FBF8F027
:10878000401A5043C21700EB126001EB202006E0B4
:10879000A16B206B081A00FB09F090FBF8F0E26D6A
:1087A0008346501C14D0616D206BA36D091A181AF2
:1087B00001FB09F100FB09F091FBF8F190FBF8F0E7
:1087C000401A5043C21700EB126001EB202006E074
:1087D000D4E90B10081A00FB09F090FBF8F0824670
:1087E00020460021272213F0A1F8C0B20FB10128C2
:1087F00000D0002094F84C10814208D030462E461C
:1088000001210546CAF1000ACBF1000B00E000216E
:1088100047B1326802EB0A002860326802EB0B00B5
:10882000306008E02A68A2EB0A00401C30602A6829
:10883000A2EB0B002860129840B3206B404200FB73
:1088400009F090FBF8F097B129B133682A46181A5D
:108850003146401C03E033683246294618442B68F1
:1088600011E00B6010601FE0136008601CE021B194
:108870002B682A463146184404E02B683246181A01
:108880002946401C33688342EEDDEAE70D990098E3
:108890008847012808DC00221F21204614F00FFE23
:1088A0000DF5117DBDE8F08F7AA8009906F00FF95B
:1088B00022A80AF05BFF22AA4FF40031204613F0F1
:1088C000C0FB204600210C2213F030F80546079922
:1088D0000998884200DB0846B5EB600F00DD4510C3
:1088E000DDF8A480009806F090F90446009806F0A0
:1088F0007DF98442009802DA06F087F901E006F07B
:1089000075F9B8EB600F01DD4FEA60089DF8B7001C
:10891000002400F0070017B1022802D002E001286D
:1089200000D101242E9800B101245D9801264FF05A
:108930000009002810DB5C9800280DDB5B980028FC
:108940000ADB0598002807DBA84505DA2A4601A9B5
:108950007AA806F08CF998B34E4694B3702222A9F7
:108960005EA8F7F7EBFE8DF8C0918DF8B3918DF806
:10897000D0918DF898917AAA5EA98F980AF0E0FCC0
:108980008DF8F490702222A93EA8F7F7D7FE8DF853
:1089900050910DF5F47A8DF840918DF864919AE834
:1089A0000F000DF5FE7A8AE80F00ECB197B101993E
:1089B0005D9808447F9003995C98081A819011E0B3
:1089C00000E04CE054F0010049D08DF8D0908DF8D3
:1089D000E090D5E702995B9808448090DDE90410A7
:1089E000081A8290CDF814917FAA10218F980AF06E
:1089F00041F907467FAA3EA90AF0A2FC83A80AF023
:108A00009BFC4EB101AE96E80F008AAE86E82F00BF
:108A100083A938460AF058FC4CB17AAC94E80F00B0
:108A20008AAC84E80F0183A938460AF04DFC07A8F8
:108A300009F03CFD7FAA07A90E978F980AF09EF8CF
:108A4000702222A93EA8F7F779FE8DF818918DF8CB
:108A500033917AAA3EA98F980AF072FC20E77AAA8D
:108A600022A9F8E70BEC0008EDEB00082DE9F04334
:108A7000BDB005460DF052FC044628460DF085FCBD
:108A800081460021204612F0BCFD01280BD00025B4
:108A9000204604F0BDFC064694F84C103540A9422F
:108AA00003D0012502E00125F2E70025204616F05B
:108AB000D4FA074620467EB112F0A8F8804637B1B6
:108AC000E06A002803DA1DB104E038900EE00DB131
:108AD000E06BFAE7606CF8E713F0FCF880460FB340
:108AE000E06A00281EDAF5B11FE0399068460AF006
:108AF0003DFE6A464FF44031204613F0A2FA334659
:108B0000424638A9204619F095FC04F1840038A9A2
:108B1000074605F0EEFF204616F094FA022806D02C
:108B20003A462AE00DB1A06CDFE7206CDDE7702249
:108B300069461CA810F0D0FC3A46694648460AF03F
:108B4000FFFB2EB115B1606C389004E0E06BFBE7E1
:108B5000D5B1206C39903346424638A9204619F0E9
:108B600069FC04F1740038A9044605F0C2FF7022C4
:108B70001CA9684610F0B0FC2246694648460AF037
:108B8000DFFB3DB0BDE8F083A06CE3E72DE9F04FDB
:108B9000ADB004460DF0C2FB054612F087F806465C
:108BA0000EA809F0A3FD0EAA0021304613F08BF9A0
:108BB00020460DF0EAFB00F1180104460FC98B4670
:108BC000CDE90723824604F1180106F1140223A817
:108BD0002B9106F02CF8002860D023AF97E80F0007
:108BE00004F1180787E80F0027A9304603F0F1FACF
:108BF00068690190A8690290E8690390289801AA21
:108C0000049010462B9906F012F8C8B1D4E90881F7
:108C1000F4E906670DF1040C89469CE80F0084E82E
:108C20000F002846183C0FF017FC159005F11402B0
:108C30000EA9204609F029FD04F1180080E8C003C0
:108C4000686901902A980290E8690390286A01AA4D
:108C5000049010462B9905F0EAFFC8B1D4E90881C9
:108C6000F4E906670DF1040C89469CE80F0084E8DE
:108C70000F002846183C0FF0EFFB159005F1140289
:108C80000EA9204609F001FD04F1180080E8C00398
:108C9000DDE90723C4E90823C4E906AB2DB0BDE82C
:108CA000F08F00002DE9F0438BB00646DDE9129805
:108CB0001D4617460C46484617F097FC002872D10F
:108CC00000234A4601A928460DF0DBFCBDF80C0044
:108CD000002868D0BDF80A10002964D0BDF90E3014
:108CE0003A681A441144491E07920991D5E90312C2
:108CF000891A7A681144BDF91020091A891A0844A2
:108D0000401E0A900891002207A8B16806F006F8F4
:108D100030B1B1680022E06806F000F8002842D1C6
:108D20000198002580B39DF812000021401E0828FC
:108D300021D20095BDF80C30BDF80A20A06909F0D9
:108D40009AF9010017D1A06908B108F0F4FFBDF845
:108D50000C20BDF80A1001FB02F0402800D252009E
:108D60000E231248009508F0A5FF01000DD0BDF8B4
:108D70000C00C880A16101A80DF07EFC206008B144
:108D80009DF81200207102E000E0FEE7257107A8BF
:108D9000A06001A8002320611A4621463046C04742
:108DA00001A80DF040FD0BB0BDE8F083C04F0020DE
:108DB000F0B58FB01D4616460C0007464CD0207902
:108DC000092849D2DFE800F0051919481948484830
:108DD0001900684608F0F3FDE07D8DF82800A08AB0
:108DE000ADF82000A07D8DF8220001200990694691
:108DF0003846E2680BF0EDF82EE0A3680DF12C0C7C
:108E00000FCB8CE80F000BA805F0FFFE0E2109F038
:108E100057F90B99401E08440D9068462C220021FA
:108E200010F015FCA08AADF81500A07D8DF8170094
:108E3000E07D8DF814002068016906910BA9089166
:108E40000089694680B20990A068009002208DF8E0
:108E50001C0038460AF0C9FE002E09D0002D07D0AC
:108E60000FB02A4631463846BDE8F0400BF02EBE22
:108E70000FB0F0BD2DE9F34F086B0C46401E4310B8
:108E800000F00100C518C969606A8FB0814201DA3B
:108E90000A4600E00246009200DD0846A0F101000B
:108EA0000290206A6946A0EB05000190206A1844F0
:108EB00003900F988268084605F0B9FE002838D064
:108EC000A06B18B1606B08B1012600E000262C21D0
:108ED00004A810F0FCFBCDF810D0A08DADF8250053
:108EE00094F82E008DF8270094F83C006D468DF81C
:108EF0002400D6B1684605F088FE0646039F019817
:108F00000390D4E90D100844009991FBF0F200FBA6
:108F1000121A304610F06AFA4FF0020B0C958DF8D9
:108F20002CB081460A90019D35E004A90F980AF003
:108F30005CFE11B0BDE8F08F3246FF21484610F0CC
:108F400086FB002150460B465A4617E0D4F834C041
:108F5000844506DBACEB000C0FFA8CFC61446044EA
:108F600008E0D4F83880C444844501DA002001E0E8
:108F700009F80130401C8DF82C20491CB142E5DB7A
:108F800004A90F980AF031FE0198401C0190039843
:108F9000401C6D1C0390BD42CEDD48460DF04CFCDC
:108FA000C7E700002DE9F34F8A46096ADAF828007E
:108FB000D9B00AF11C040AF12406814205DA2146DF
:108FC000684614F0FFFF314604E03146684614F06D
:108FD000F9FF2146DDE90057684614F0F3FFDDE9AB
:108FE0000046A4EB0508A6EB0709B8F1000001DC78
:108FF000C8F10000B9F1000101DCC9F100018842AB
:1090000001DD012000E000200190DAF8301058B1B5
:10901000B9F1000001DCC9F100004201B8F1000023
:109020000DDCC8F100000AE0B8F1000001DCC8F175
:1090300000004201B9F1000001DCC9F1000092FB1F
:10904000F0F0924A105C48433F30C0114FEA600B89
:1090500000F0010202EB0B010691A54201DA29465C
:1090600000E02146A1EB00010A9101DD294600E064
:10907000214601440C91B74201DA394600E03146FD
:10908000A1EB00010B9101DD394600E031460844B7
:109090000D9059980AA98268084605F0C8FD002875
:1090A0007DD014210EA8F7F783FB1EA80E902CA8E4
:1090B0000F9001990020002972D0B8F1000F13DD44
:1090C000A6EB0B01CDE900102346A7EB0B022946C6
:1090D0001EA80CF09FF8069801213044CDE900014C
:1090E000069823463A1812E0069923463144CDE902
:1090F0000010069829463A181EA80CF08BF801219A
:10910000A6EB0B002346A7EB0B02CDE90001294695
:109110002CA80CF07FF89AF83D004FF0020BC00627
:109120001AD4032107EB0800CDE90001A5EB0903E0
:109130003A4629463AA80CF06DF806EB0801CDE94D
:10914000001BA4EB09033246214648A80CF062F844
:109150003AA8109048A811900AA805F056FD0446B8
:1091600015F0DEF808F01EF805460AA805F043FDE4
:10917000A84203D20AA805F03EFD0546A8462846A7
:1091800010F034F981460D9F0B980D900025424652
:10919000FF21484610F05BFA2C2113A801E071E092
:1091A00014E010F094FA0AA91391BAF82C20ADF843
:1091B00061209AF82E008DF863009AF83C008DF833
:1091C0006000CDF864901B910B9E3AE0CDE9006001
:1091D00006983A46231829181EA80CF01BF80120FF
:1091E000CDE90060A4EB0B033A46A5EB0B018FE73A
:1091F000009409EB05010A9A33460EA808910BF07A
:1092000083FF8DF8680018B92146089810F05FFABE
:1092100025442919414503D20D98401C0D900FE0BB
:109220008DF868B013A959980AF0DFFC0D98002555
:10923000401C0B900D904246FF21484610F007FA63
:10924000761CBE42D4DD0D990B98884207D0481E8B
:109250000D908DF868B013A959980AF0C6FC4846DD
:109260000DF0EAFA1EA80BF08DFF2CA80BF08AFF78
:109270009AF83D00C00605D43AA80BF083FF48A831
:109280000BF080FF5BB0BDE8F08F0000A812030870
:109290002DE9F04F8346086B0C46401E411000F04C
:1092A00001004218E06991B0821A084400920290CD
:1092B000216AA06A814200DA08460190216AA06A08
:1092C000814200DD0846401E039069460846DBF8EF
:1092D000082005F0ACFC00283BD0A06B18B1606BF7
:1092E00008B1012600E000262C2104A810F0EFF9B7
:1092F000CDF810D0A08DADF8250094F82E008DF893
:10930000270094F83C006D468DF82400EEB16846C5
:1093100005F07BFC0F90039F019803900F9810F0CD
:1093200065F880460A9002200C958DF82C00D4E94F
:109330000D10084401994FF0000991FBF0F200FB79
:1093400012150E464FF0010A25E004A958460AF00E
:109350004CFC11B0BDE8F08FFF2140460F9A10F091
:1093600076F9606BA84202DA8DF82C9001E08DF856
:109370002CA0D4E90D100844A84200DC002504A963
:1093800058466D1C0AF031FC0198401C019003986E
:10939000401C761C0390BE42DEDD40460DF04CFAC8
:1093A000D7E72DE9FF4705460CF0B8FFC46A284609
:1093B0000CF0EBFFE26A054600F118016846143232
:1093C00005F035FC002834D0D5E90881F5E90667B9
:1093D00089469DE80F0085E80F0094F84C00183D81
:1093E000800628D5A26C206C824208D12123294610
:1093F0002046FEF767FC20462123A26C13E02023C1
:1094000029462046FEF75EFC204620232946A26C12
:10941000FEF7A8FC204601232946226CFEF752FCE9
:10942000226C204601232946FEF79CFC183585E86E
:10943000C003BDE8FF87204620232946A26CFEF723
:1094400041FC20462023A26CEDE700002DE9F04FFF
:10945000F7B005460CF062FF0446806B00287DD013
:1094600028460CF092FF7290608D40F008016185F3
:1094700020466CA911F098FB0025278D2585608D6D
:109480002E4640F0080161853BA80AF06FF957A805
:1094900009F02CF94FF4A0293BAA4946204612F0C6
:1094A000D0FD57AA4946204612F00DFD608D0021DF
:1094B00020F0080060852046278512F01FFA75907D
:1094C0000021204612F0A5F974900021204612F0E8
:1094D000CDF973900021204612F0E9F982460DE1A2
:1094E000761CE06A90A150F8260016F009F80028D2
:1094F000F6D0606B30F81500C1067CD44FF0000840
:10950000C10501D54FF00108400602D548F08000A2
:1095100012E0206CA84210D1B80601D548F020080E
:10952000B80701D548F00208780701D548F00408CB
:10953000380702D548F008008046206B00EB051183
:1095400003A805F0CDFA03996C98049A014403919D
:109550006D99114404910599084400E0D6E0059006
:109560006D990698B8F1000F084406907ED0A4F8D3
:109570002880608D40F0080161850AA80AF0F6F89D
:1095800026A809F0B3F80AAA4946204612F059FD68
:1095900026AA4946204612F096FC2785608D20F0C9
:1095A000080161859DF871000C95C10636D520F043
:1095B0001F000F308DF8710063697399039A194485
:1095C0008A4203D120F004008DF87100E269059908
:1095D000A2EB0A00814205D19DF8710020F008003D
:1095E0008DF87100A269759804991044814207D1E1
:1095F0009DF8710000E07FE020F002008DF871001E
:10960000226A74980699101A814207D19DF8710058
:109610004108490061F304008DF8710003A805F0CA
:10962000E5FA07905FEA886008D5606B30F81500AE
:10963000400503D504990798081A049003AA0AA9BB
:10964000729809F07DFE2E9871903598709034993B
:109650000191E06A50F826B06CA805F0D6FA9DF8A2
:10966000E3200199CDE90010029200E051E0DDE92C
:109670007032594608A816F0DDFE03A805F0C5FAB9
:109680000899401A039900EBD07001EB6000039039
:1096900003A805F0ABFA0999401A049900EBD070C1
:1096A00001EB60000490089903980844059009991B
:1096B0000498084406905FEA88600FD5606B30F824
:1096C000150040050AD50798049900EBD070A1EB6E
:1096D000600104910699A1EB600006909DF8E400FA
:1096E000CDF8B4B040F040008DF8E40003AA26A9FC
:1096F0002895729808F0C9FF6D1C761CA06BA842D3
:109700003FF6EFAE608D20F00800608577B0BDE8D1
:10971000F08F70223BA90AA80FF0DEFE542257A951
:1097200026A80FF0D9FE3DE70A0000002DE9F04F12
:10973000F9B005460CF0F2FD044628460CF025FE73
:1097400071900021204611F0BFFF05460021122232
:10975000204612F0EBF8284477900021132220468F
:1097600012F0E4F800EB050B03A808F0BFFF03AA12
:109770004FF40031204612F0A6FB206B40B1814629
:1097800094F84C00002700F00F00012807D007E0F4
:1097900080222DA920460CF075FB2DA8EFE70127AC
:1097A00020460021272212F0C1F8C0B2012800D1C2
:1097B0000127606B4FF0000800285CD00EF00CF918
:1097C0008246022818D04DA9606B0DF04DFD01288E
:1097D00022D04FF0FF363546A069691E73900844C9
:1097E00075906069711E72900844CDF80080749085
:1097F000B7B10722779B16E011989DF857206FF0BC
:1098000060418DE80700129B0B9A50A8616B16F01F
:1098100011FEDDE95065DFE74E9886B2050CDBE707
:10982000CBF10003082272A904F1140005F048F8F6
:10983000BAF1020F49D04DA808F038FE4FF4003AB3
:109840004DAA5146204612F0E4FA05EBD5704210BD
:1098500006EBD67041105DA814F0B9FB20466E22CD
:10986000514612F063F85890606B549072AA4DA95B
:10987000719808F0C7FD18A808F038FF18AA002151
:10988000204612F020FB26989DF8AB206FF0604137
:109890008DE8070049466FA8279B209A16F0CAFD5D
:1098A00060696F996B900844401E6D90A069709933
:1098B0006C900844401E6E90606B70B1CDF80080D3
:1098C00087B1CBF1000308220EE0606B0A9072AA08
:1098D00003A9719808F0D9FECDE700230922CDF83D
:1098E000008001E0779B07226BA904F1140004F0CB
:1098F000E7FFCDF87C90206B28B99DF8AC0040F0D4
:1099000040008DF8AC006BAA18A9719808F0BDFE54
:1099100079B0BDE8F08F2DE9F04FABB005460CF003
:10992000FDFC044628460CF030FD05461FA92046E4
:1099300011F0F6F8204602F0A4F9064603A808F054
:10994000D5FEE06A0A90606D1390A06D149094F8B3
:109950005C0000F00700032808D01FA805F046F9B6
:10996000B0F5806F02DB04F1380017908DF8576076
:1099700003AA0021204612F0A6FA9DF856004FF0E7
:10998000010808B98DF85680606C0C90A06C0D90A1
:109990000C994FF6FF70814226D00D99814223D059
:1099A0004FF48029274658224946204611F0BEFF31
:1099B00002464946384613F093FF0090BDF8000078
:1099C000ADF83B009DF802008DF83D0020461C22BA
:1099D000494611F0ABFF0090BDF80000ADF83E0025
:1099E0009DF802008DF8400094F85C006FF0604B29
:1099F00000F00700022801D0032817D19DF8560077
:109A0000022801D0032811D11199CDE9001B02963B
:109A1000129B0B9A27A8E16A16F00CFD1FA805F00F
:109A2000F4F82799884201DA8DF8568005F118027A
:109A30001FA919A805F0FBF800287ED094F85C0057
:109A4000400709D1204611F075FA424200211FA8B3
:109A500005F032FA206A229094F85C0000F00700CA
:109A600002281BD0032819D01FAA03A9284608F0F2
:109A70000CFED5E907800DF1640C81469CE80F00CF
:109A800005F1180CD5F824A0AF698CE80F0094F804
:109A90005C0000F00700032818D051E0D5E90782E8
:109AA0000DF1640C91469CE80F0005F1180CD5F8F7
:109AB00024A0AF698CE80F001FAA03A9284608F06C
:109AC000E4FD05F1180080E88007D2E71199CDE99F
:109AD000001B0296129B0B9A29A8E16A16F0AAFCB9
:109AE0001FA805F092F82999884212DA202211461F
:109AF0000B980CF064FE616D299A00EB4000114454
:109B000008441390A06D14901FAA03A9284608F0DA
:109B1000BCFD1FA805F06AF82A99884210DA606D2A
:109B200013900B980CF07DFEA16D2A9A1144084405
:109B300014901FAA03A9284600E004E008F0A5FD40
:109B4000183585E880072BB0BDE8F08F2DE9F0438C
:109B5000A7B007460CF0DEFB054638460CF0DEFBEE
:109B600004464FF480261A2D7DD01D2D7CD1384619
:109B70000CF00BFC054603A808F0B8FD03AA31461B
:109B8000204612F0A0F922A9204602F022FB22AAC8
:109B900005F1180118A805F04AF8002864D02046FD
:109BA00002F06CF88146204612F094F806464846CA
:109BB0000EF052FC01461198CDE9000601220292F6
:109BC00020A8129B0B9A16F035FC204611F01EF8C7
:109BD00007460021204611F0B1FFC268D9F81810DD
:109BE00002EBD27201EB6201A269064607EBD7785D
:109BF00002EB68000F1A484611F008F8F168401AA5
:109C0000002802DDB90391FBF0F70B98A26902EB83
:109C10006801C068219A121A7A4301EBA23100EB65
:109C2000D070A1EB60080021204611F050FD0746DE
:109C300020460021122211F079FE0646204600211E
:109C4000132211F073FE6169F2191144CDE91C1859
:109C5000E169081AC01B21991E9008EB01001F90B2
:109C60009DF8570001E020E01CE040F001001835AD
:109C70008DF8570095E8D1000DF1600C80469CE806
:109C80000F0085E80F004846183D0EF0E5FB0A90EE
:109C90001CAA03A9284608F0F8FCC5F818801C3552
:109CA00085E8D00027B0BDE8F08338460CF06DFBA6
:109CB00005461CA9204602F08CFA684609F056FDBC
:109CC0006A463146204612F0BCF91CAA694628466D
:109CD00009F036FBE6E72DE9F043C7B005460CF086
:109CE0001DFB044628460CF050FB814642A9204645
:109CF00010F016FF05A809F039FD05AA4FF4003150
:109D0000204612F09EF942AA05A9484609F018FB20
:109D1000204610F07BFF054604F1140004F075FFA7
:109D2000461BE06A411C05D07043C11700EB11606F
:109D3000071208E0204611F035FC10F0010F01D0A9
:109D4000374600E0002720460021272211F0EEFDD3
:109D5000C0B2012800D1F71B60690090A069019092
:109D6000E0690290206A03900098002D384400902A
:109D700001DD6D1E00E0002528444FF440370290BD
:109D80003946204611F081FD06463946204611F03D
:109D90009AFD05463946204611F0BFFD80463946FA
:109DA000204611F042FD01460098019A801B009068
:109DB000029828440290A2EB0800019003980844FE
:109DC000039023A809F0D2FC23AA3946204612F0BA
:109DD00038F96A4623A9484609F0B2FA47B0BDE807
:109DE000F0832DE9F04FADF5137D05460CF096FAA2
:109DF000044628460CF0C9FA814600F1180204F125
:109E0000140105A804F013FF00287ED009F1180002
:109E100005AE90E80E00D9F82400CDE90A12CDE98C
:109E20000C3096E82E0009F1180080E80E0020465C
:109E300000213022C9F8245011F078FD8B900021C8
:109E4000204611F06DFD90900021204611F0F0FCAD
:109E500091900021204611F01BFD8F90002120469B
:109E600011F034FD8E90208D002514902585608D95
:109E700040F0080161852FA809F078FC4FF4A02676
:109E80002FAA3146204612F0DCF86BA808F02EFC11
:109E90006BAA3146204612F016F814982085608D82
:109EA000002620F008012046618511F04FF8014698
:109EB000A26990981044411A8B980E950844401E50
:109EC000CDE91050204611F03BF88D90002120463E
:109ED00011F09DFB012800D000208246002092E175
:109EE000A16B51F8280011998C90491C401E084420
:109EF000119008980F9181427DDCBAF1000F0BD0D0
:109F0000E1698E98091A8D9800E08AE1091A8B9808
:109F1000081A401E0E9008E061698F9801448D98E0
:109F2000091A8B980844401E1090002565E1606B6B
:109F30004FF0000B50F8260008B190F800B0BAF1CD
:109F4000000F0AD00E98401E1090E06B109950F848
:109F50002500081A401C0E9009E01098401C0E9035
:109F6000E06B0E9950F825000844401E1090002721
:109F700018E0616BF01951F82000C0B10078C007FB
:109F800015D0E9190422E06B02EB8101BAF1000F50
:109F9000405803D00E99081A0E9002E01099084418
:109FA00010907F1CE06A7919401E8142E1D311991B
:109FB000069881427CDB0E982B900F982C9010987D
:109FC000CDE92D019DF8050141070BD562698F9BF5
:109FD0002B991A44914205DD409A02EBD272A1EB13
:109FE00062012B9181070DD5A36990992C9A194490
:109FF0008A4207DD00E00BE1409901EBD171A2EB51
:10A0000061012C91010710D5E3698E992D9A591A97
:10A01000491E8A4209DA409901F0010201EBD1712F
:10A0200002EB61012D9A11442D91C00710D0226AD4
:10A0300091982E99101A401E814209DA409800F03A
:10A04000010100EBD07001EB60002E9908442E90C6
:10A05000626C0020424554D1216CA94251D1218D1E
:10A060004A0602D48A0600D520208A0701D540F08E
:10A0700002004A0701D540F00400090701D540F06D
:10A080000800F0B32085608D40F0080161854BA881
:10A0900009F06CFB16A808F029FB4BAA4FF4A0218D
:10A0A000204611F0CEFF16AA4FF4A021204600E072
:10A0B00092E011F008FF14982085608D20F00801CF
:10A0C0006185CDE94D85CDE918852BAA4BA9484678
:10A0D00009F036F9606B50F8260000287CD04FF468
:10A0E000A021204611F0D4FB02904FF4A02120467D
:10A0F00011F0ECFB85904FF4A021204611F010FCEC
:10A1000000E033E084904FF4A021204611F090FB52
:10A110000146002000900E9A029810446790109A11
:10A120008598101A69900F9A849810446890119835
:10A13000401A6A90CBF340005FEA000B01D0012087
:10A14000009067A804F061FD009A2499CDE9001001
:10A150000292606B259B739A50F8261087A80831ED
:10A1600016F068F9BBF1000F0BD01CE070222FA98C
:10A170004BA80FF0B1F954226BA916A80FF0ACF957
:10A180009FE78C980F9A00EBD070889902EB6002E1
:10A1900001EBD1714010A2EB610200EB61000F995D
:10A1A000689208446A900EAA05A980A804F03FFDB1
:10A1B00090B10DF5007B09F118009BE80E1080E8C6
:10A1C0000E00C9F824C0606B67AA16A950F82600D3
:10A1D00008301D90484600E00BE008F056FA0DF1FB
:10A1E000140B09F118009BE80E1080E80E00C9F866
:10A1F00024C03E443D44761C6D1CE06AA8423FF6F4
:10A2000096AE08F10100216B804641453FF668AEED
:10A210000AAD09F1180495E80F0084E80700C9F8B1
:10A2200024300DF5137DBDE8F08F2DE9F0479AB08D
:10A2300005460CF073F8044628460CF0A6F8824652
:10A24000E06A0EF009F9007800284FD1206B002851
:10A250004CD00078002849D004A808F047FA04AA96
:10A260004FF40021204611F02EFE94F870000007F4
:10A2700005D59DF85B0040F001008DF85B000021E2
:10A28000204611F008FB81460021204611F021FBF9
:10A2900080460021204611F046FB0746002120465B
:10A2A00011F0C9FA06460021204611F016FA0546BB
:10A2B00004F11401684604F025FC009809EB05013F
:10A2C00008440090029808EB0501401A029001989A
:10A2D00079190844019003987119401A0390206B72
:10A2E0000B906A4604A9504608F0CFF91AB0BDE8B1
:10A2F000F08730B5A5B00C46054620AA1CA910F081
:10A300002BFE1CA804F077FC20B920A804F073FCF5
:10A3100000281CD0694628461BF0A4F9012816D154
:10A320001CA804F068FC30B1002002901CAA694609
:10A33000204609F005F820A804F05DFC002806D0AE
:10A340000120029020AA6946204608F0F9FF25B0B6
:10A3500030BD2DE9F04F884601F11802B9B004462E
:10A3600000F1140120A804F062FC00286FD008F16D
:10A37000180020AE90E80E00D8F824002991019032
:10A38000CDE92B2396E82E0008F1180080E80E0096
:10A3900000212046C8F8245011F06BFA064600212F
:10A3A000204611F0AEFA8146204610F0ECFB2890D2
:10A3B000204610F0D7FB259004F12C002A900EF0D7
:10A3C00019FF05460021204611F041FA226F289915
:10A3D000C2F1010303FB0010B0FBF2FA4FF4A0211D
:10A3E000204611F034FA8346C5F1010202FB0BA0AE
:10A3F000B0FBF5F7012F00DA01270021204611F00C
:10A4000060F90546204610F0D3FC301A28443490F9
:10A41000204610F08FFDA9EB00002844339002A8DD
:10A4200009F0A4F902AA4FF4A021204611F009FE78
:10A430009DF83700099920F007008DF83700FF20BC
:10A440008DF82800206A00260844319069E075E004
:10A450002899401EA1EB0A017143B1FBF0F1349839
:10A460000844616900EB01090020CDE904062A983F
:10A470000EF0BCFE52E0287CC0074BD194F874006B
:10A48000000701D4E96800E000217A1E4A443092B6
:10A49000CDF8B89007EB0B02484602EB0009209B71
:10A4A000309A9A4233DB229A904239DC2889ADF8FF
:10A4B0002900A87A8DF82B008819216FDDF894C047
:10A4C000B0FBF1F201FB1201686850F82120287CF2
:10A4D000C0F3001304EB8303586CDB6C121A02FB0D
:10A4E0000CF2181A92FBF0F0ACEB00023398A3695F
:10A4F000104418442F90686850F821006FF0004114
:10A50000884204D02EAA02A9404608F019FF0498F8
:10A51000401C049029462A980EF07AFE0500AAD124
:10A52000761C206FB04293D8DDE92B2308F1180088
:10A530002999019C80E80E00C8F8244039B0BDE894
:10A54000F08F2DE9F04F01F11802884600F1140157
:10A55000CDB0044691460F4644A804F068FB00289D
:10A560007DD008F1180144AE91E80D00D8F8241010
:10A570000990CDE938219A4696E82E0008F1180096
:10A5800080E80E00C8F82450206F022867D300210D
:10A59000204611F096F805460021204611F069F991
:10A5A00046190021204611F0ACF90544204610F070
:10A5B000EAFA0890204610F0D5FA0690204610F0EE
:10A5C000F7FB61693144081A3D90204610F0B2FC57
:10A5D000A1694A462944081A4290394649A804F01C
:10A5E00026FB00283BD028A808F0B1FB28AA4FF48E
:10A5F000A021204611F0C1FC0CA809F0B7F84FF4D7
:10A6000000350CAA2946204611F01BFD294620469C
:10A6100011F0DCFA00EBD07046102946204611F00C
:10A620006EF800EBD0704110894634984E4500DA40
:10A63000314600EBD070B1EB600F05DD9DF8DD0019
:10A6400040F010008DF8DD003498012805D19DF808
:10A65000DD0040F010008DF8DD00216F00E033E1F7
:10A660000898814201DB012000E00020439004F1C2
:10A670002C0005460B900EF0BDFD401E2A900E905A
:10A6800028460EF0CCFD13E1287CC00706D02A989E
:10A69000401E2A900E98401E0E9005E12889ADF8C4
:10A6A000CC00A87A8DF8CE002889ADF85100A87AA0
:10A6B0008DF8530000202B900F9094F87400000741
:10A6C00001D4E86800E000203A903D982F90319046
:10A6D0003A9848906968834651F82000297CC1F374
:10A6E000001104EB81020699536CC01A4843D16CE7
:10A6F000C91A90FBF1F00699091A429800270844FC
:10A70000329003900590A5E031982F9032983090C8
:10A71000711C2F9A0AEB010082427EDC0898216F9F
:10A720007843491EB0FBF1F13D98069B08443190F7
:10A730003A98226F3844B0FBF2F102FB110B6968C2
:10A7400051F82B00297CC1F3001104EB8102516CFC
:10A75000D26C401A5843511A90FBF1F0191A4298E2
:10A760000844329009983199801B401E81426EDB6B
:10A77000002F6CD04398A0B36968489851F8202006
:10A780006FF00040824262D051F82B1081425ED0BF
:10A7900032990598814200DB084605900398814272
:10A7A00000DC0846039031992F9888424FD03298A8
:10A7B0003B90481E31902F9003983090059832902E
:10A7C00032993098884201D1481C329028A94046DD
:10A7D00008F081FA3198401C31903B980390059025
:10A7E00035E0FFE72F983099801B3E902F9830443A
:10A7F0004090A1EB09003F9001EB0900419068688F
:10A80000489950F821206FF000418A420CD050F84E
:10A810002B106FF00040814200E01FE004D028A917
:10A8200040462B9708F057FA8EB1B9F1000F0ED0C1
:10A830006968489851F820106FF00040814206D0B6
:10A84000781E0F903EAA0CA9404608F079FD7F1CA7
:10A85000CDF820B1206FB8423FF656AF4398E8B923
:10A86000206FB8421AD169686FF0004051F82B1080
:10A87000814213D031983299801B3E9031987F1ECF
:10A8800030444090A1EB09003F9001EB09000F9785
:10A8900041903EAA0CA9404608F052FD0E98401E79
:10A8A0000E902A98401E2A9029460B980EF0B4FC70
:10A8B00005007FF4E9AEDDE9383008F11801099AA6
:10A8C00081E80C04C8F824004DB0BDE8F08F00000A
:10A8D0002DE9F04F8A4601F11802C9B0054600F192
:10A8E00014013CA804F0A3F900287DD00AF1180156
:10A8F00033AC91E80D00DAF82410369184E80D00AD
:10A900003CAE0AF1180096E81E0080E80E00002117
:10A910002846CAF8244010F0D4FE044600212846F8
:10A9200010F0A7FF06460021284610F0EAFF074670
:10A93000284610F028F94190284610F013F940906D
:10A94000284610F035FA0146686932191044401A59
:10A950004290284610F0EEFA0146AA6938191044D0
:10A96000401A43901FA808F0F2F91FAA4FF4A02143
:10A97000284611F002FB03A808F0F8FE4FF400345B
:10A9800003AA2146284611F05CFB2146284611F017
:10A990001DF900EBD0704FEA60092146284610F0FF
:10A9A000AEFE00EBD070401080462B994A46C14560
:10A9B00000DA104601EBD171B0EB610F05DD9DF8B7
:10A9C000B90040F010008DF8B9002B98012805D18E
:10A9D0009DF8B90040F010008DF8B90005F12C0089
:10A9E00037900EF01CFCE8E0EAE0207CC0077DD147
:10A9F0002089ADF8A800A07A8DF8AA002089ADF8CA
:10AA00002D00A07A8DF82F0095F87400000701D46E
:10AA1000E66800E0002642982690449628906068F8
:10AA2000B34650F826000A2826D0419800902068A6
:10AA3000002350F82670207CC0F3C00005EB800096
:10AA4000C26D416D38460EF009FD4299002308445D
:10AA5000289040980090217C6068C1F3001105EBBC
:10AA6000810150F82600CA6C496C0EF0F7FC409941
:10AA7000081A4399084401E0544828900026299078
:10AA800082E028982690299827902A6F0BEB0600E1
:10AA9000B0FBF2F102FB110760686FF0004150F863
:10AAA000270088427ED040990091217C0023C1F389
:10AAB000001105EB8101CA6C496C0EF0CFFC409986
:10AAC0000023091A43980844299041980090217C5A
:10AAD0002068C1F3C00105EB810150F82700CA6D61
:10AAE000496D0EF0BBFC4299084400E061E02890FB
:10AAF0005EB32699A1EB0900459001EB0900279967
:10AB00004790A1EB0800469001EB0800489061686F
:10AB1000449851F820206FF00040824214D051F840
:10AB20002710814210D01FA95046229608F0D3F872
:10AB3000B9F1000F08D0B8F1000F05D045AA03A95C
:10AB40005046069608F0FCFB4497286FB0421AD195
:10AB5000606850F827106FF00040814213D02898A9
:10AB600045AAA0EB09004590289803A948444790BE
:10AB70002998A0EB080046902998069640444890F2
:10AB8000504608F0DDFB761C286FB0423FF679AFE7
:10AB9000219833AF401C21900598401C059097E800
:10ABA0004D0000E00FE00AF1180181E80D00CAF83D
:10ABB0002460214637980EF02FFB04007FF415AF78
:10ABC00049B0BDE8F08F4497DDE70000010000E0E8
:10ABD0002DE9F84304460BF0A1FB804620460BF01C
:10ABE000E5FB0646C06C4068B0F5A02F62D1304648
:10ABF0000BF01AF8054630460BF00FF8044655EAFC
:10AC0000040057D0F06C00278668072E05DB402231
:10AC10003146404605F006F928B10DB185F820709F
:10AC20000CB184F828704FF400423146404605F0DC
:10AC3000F9F820B354B1404616F0A6FA0090BDF8DA
:10AC4000000020849DF8020084F8220075B166207F
:10AC500085F82000404616F097FA0090BDF80000F5
:10AC6000A5F821009DF8020085F82300404605F074
:10AC7000D7F8B04203D115B1B22085F820004FF4C7
:10AC800080423146404605F0CDF8002812D0002C15
:10AC900010D0FF2084F828004046203416F074FAC3
:10ACA0000090BDF8000020809DF80200A070606850
:10ACB000401C6060BDE8F8832DE9F0410F460400B8
:10ACC00005D004F1300080460EF090FA11E0FEE766
:10ACD000286861680669304605F07AFA05F07CFA62
:10ACE00018B9A269394630469047294640460EF0C9
:10ACF0008FFA0500ECD104F1240013F0E1F940468D
:10AD00000EF054FA0020E060BDE8F0812DE9F0413A
:10AD1000174604002DD069B304F12400804613F0D7
:10AD2000FDF9050027D02E69A269394630469047C3
:10AD3000E16B30468847E168091AE1603046616896
:10AD400005F046FA07462869E16A0844294650F8A2
:10AD5000046C404613F060FA384605F02BFA314691
:10AD600004F130000EF00CFB3046BDE8F0410BF072
:10AD700063BDFEE7FEE7BDE8F0810879052801D054
:10AD800006281ED1C86C826B2ABBC26B1ABBC26A72
:10AD90003AB9036B4FF48072934202D1436B9342F2
:10ADA00001D0012300E00023826E02B101221A4289
:10ADB00011D1008CC0F307201AB10E280BD0142833
:10ADC00009D091F85100642805D3642081F851001E
:10ADD000012081F850000020704710B50446007E25
:10ADE000400721D42089282820D029281ED04FF4BC
:10ADF0008041206810F0B4FF002816D02089133855
:10AE00001F2813D2DFE800F01012121210101010D9
:10AE10001010101010121210121212101010101226
:10AE20001212121010121000002010BD012010BDCF
:10AE300070B504460CF0E0FD40B1207E810701D5DD
:10AE4000012070BDC00701D0002070BD206885685A
:10AE500005B108350122214628460BF0F5FA0128F4
:10AE6000F3D1217E8907F0D4214600200FF0D7FDD1
:10AE70000128EAD1217E8907E7D40022214628460D
:10AE80000BF0E2FA0546012814D1207E800711D488
:10AE900020680FF00BFF06000CD02046FFF79DFF47
:10AEA00040B120462660FFF7C3FF0546012801D1C7
:10AEB000207E8107284670BDC26911790B292DD2E9
:10AEC000DFE801F02C060A0E1216241E1A212800B3
:10AED000D16C083209F0FABDD16C083209F079B8AA
:10AEE000D16C083209F0E6B8D16C083209F0F4BF31
:10AEF000D16C083209F0D0BFD16C083208F086BCA2
:10AF0000D16C0AF008B8D16C0AF0B8BCD16C083228
:10AF100009F0ECBFD16C08320AF0AEBA70470000FD
:10AF20002DE9FF4F89B00E46DDE916B41746002122
:10AF3000099810F048FE05460021099810F0DCFB46
:10AF40000146F07882070BD5C3076FF0404202D06C
:10AF5000954202D006E0914206D120F00200F07046
:10AF6000C00701D0714800E071488146F078C00701
:10AF700012D06F484FF0000AC4F804A0C4F808A02B
:10AF8000C4F814A0C4F800A0C4F80CA0C4F810A021
:10AF900080463946009798E06448EBE70098B8424D
:10AFA00006D04FF40011284610F0DAFE00287DD1BB
:10AFB0006049284610F0DBFE00287BD1002128469E
:10AFC00010F08EFB0690A8B36069401C6061A26817
:10AFD00002EB0B01A160217EC9075AD000EB4000B3
:10AFE000C100206913F05EF9079078B1606900EB49
:10AFF0004001079800EBC1004FF0000140F8185CD9
:10B00000F078C007284602D0042201E0FEE70622BD
:10B0100010F08CFC616901EB4102079901EBC20160
:10B0200041F8140CF0784FF00001C007284602D018
:10B03000052201E01EE0072210F078FC6169079A02
:10B0400001EB410102EBC10141F8100C6169079A63
:10B0500001EB410102EBC101069841F8080C61695E
:10B0600001EB4102079901EBC20141F804AC0798DA
:10B0700020610EE0284649468847F178890704D5C3
:10B08000A1680A180C998A4225DCA2685844104429
:10B09000A06028464146884701462068814202DD7B
:10B0A0002846414688472060E06801E013E001E05F
:10B0B000401CE060F078400702D54FF0FF3000E020
:10B0C000012000994118009105D409980FF0BDFCAA
:10B0D000051E7FF463AFA068002802DDA0EB0B0023
:10B0E000A060606908B10C9800E0A0686060CDB114
:10B0F0000098B84216D109996A468968096851F8DA
:10B100002050F078C0F38001099800F0C1FE4DB1E5
:10B11000284641468847206028464946884760605F
:10B120000120E06000980DB0BDE8F08FDBBC0108A5
:10B1300013AC0108010006002DE9F04F93B004465E
:10B1400000217D2210F0F2FB9DF81710421C62F3E3
:10B150000001820862F34101C00860F382018DF8AA
:10B160001710204600217E2210F0E0FB8DF814001D
:10B17000204600217F2210F0D9FB8DF815002046D3
:10B180000021802210F0D2FB8DF81600002120460D
:10B1900010F031FA012800D0002080469DF81700F9
:10B1A0004FF00001C00720460CD010F098FB8146FC
:10B1B0009DF817004FF00001C007204605D010F0A1
:10B1C00040FB04E010F03DFBF1E710F088FB079036
:10B1D0009DF81700C007204602D00FF0D4FC01E014
:10B1E0000FF0C0FC002106900F462046102210F000
:10B1F0009DFB05463946204610F05DFA0646394665
:10B20000204610F043FA800700D53544A069054474
:10B2100020460FF09BFE281A002108900E4620467B
:10B22000122210F083FB05463146204610F043FA07
:10B2300007463146204610F029FA400700D53D4424
:10B240006069054420460FF07BFE281A11909DF896
:10B2500017009DF81660C00701D008AD00E011ADE1
:10B260000021204610F0AFFC12900021204610F083
:10B2700043FA83469DF81700C10708D06FF040429B
:10B28000934502D1618D490509D5C10708D11299AD
:10B290006FF04042914203D1618D090500D4002630
:10B2A000B8F1000F08D0C00706D116B1012E02D0A8
:10B2B00002E0012600E000260027BA46109776B388
:10B2C0009DF81700400703D5A068028D521E13E0B9
:10B2D000002211E000200F9009A90798CDE9000194
:10B2E00005A92046069BFFF71BFE099A07EB0901FB
:10B2F00057180AF1010A0246A068008D904201DD4C
:10B30000002AE7DABAF1000F01D0A7EB09079DF890
:10B310001700C007204603D00FF024FC02E00AE02B
:10B320000FF031FC10A9CDE90051014653463A46D1
:10B33000304617F046F89DF81700410703D5A1687D
:10B340000E8D761E00E00026B8F1000F04D0C00775
:10B3500002D128683844286009AFA068008DB04247
:10B3600043DD002E41DB01200F900798CDE9000757
:10B37000324605A92046069BFFF7D2FD8246B8F16A
:10B38000000F07D09DF81700C00703D1286809995E
:10B39000401A286006AB93E8070002AB019283E8ED
:10B3A0008300119800905346324605A92046FBF7CA
:10B3B000E1FB56460D980BF03FFA00200D90B8F1D6
:10B3C000000F03D09DF81700C00708D0286809991E
:10B3D000109A014402EB090008442860BDE7109A66
:10B3E000296802EB0900081AF7E712996FF040404C
:10B3F000814201D0834502D1204611F0B5FB0022E5
:10B400003021204612F05BF813B0BDE8F08F000049
:10B4100070B504461248134E4FF40045032C01D971
:10B42000032414E034B1032C11D0022C11D0012CD0
:10B4300001D009E0012400220821F7F788F9002251
:10B4400029463046F7F783F90748047070BD01229A
:10B45000F2E700220821F7F77AF90122F0E700006D
:10B460000004024000000240780000202DE9F74F60
:10B470000546007F93464FF0000AC00760D14FF0A9
:10B480000108EC680026C1467CB9287FC0F3C000E3
:10B49000401E304254D1B9F1000F51D001992846D5
:10B4A00088474FF000080446C1460EB9261E47D013
:10B4B000B8F1000F06D0214628465A469047044668
:10B4C000B0423DD04FF00108002CDED0206810F0D3
:10B4D00069F80006D8D427681FE00121384610F02B
:10B4E0003FFCB0B12FB10121384610F039FC0028E3
:10B4F000CAD1E868A04223D0B0B1284600F00CFBC6
:10B500000246E8681121006811F0D9FF012817D11F
:10B5100006E038460FF0CAFB0746002FDDD1E8E70A
:10B52000E868006810F01BFF2846EC6000F0F4FAB1
:10B530000246E8681021006811F0C1FF012802D01E
:10B540005046BDE8FE8FE868006810F008FF2969E2
:10B5500009B1284688470120F3E770B5846C054699
:10B56000002C16D0206820B10BF088F920680BF071
:10B5700063F9E06908B106F0DEFB206A08B106F065
:10B58000DAFB60680BF058F920460BF055F9002003
:10B59000A86470BD2DE9F0411D46069C164607467D
:10B5A0000CB100202060002238460BF0EDFA002894
:10B5B00007D123462A4631463846BDE8F0410BF014
:10B5C000FCB9BDE8F08170B50146C06ACA6C12F0E2
:10B5D000060F1AD0C2F34102022A18D0012A13D151
:10B5E000D1E90E54AC4201DA04F5B4744A6B0E6B27
:10B5F0001346B24201DA03F5B472291901EBD17195
:10B6000049108E4206DA304470BD496B00E0096B88
:10B61000084470BD8A4201DD184470BD084470BD05
:10B620002DE9F34F93B0064669460FF0BDFA304658
:10B6300010F050FB099030460FF0E8FA0890002116
:10B64000304610F013F983460021304610F02FF9F0
:10B6500004460021304610F051F9054600213046DD
:10B6600010F0D7F880460021304610F03BF907462D
:10B670000021304610F0E8F807F0010107EBD7721F
:10B6800001EB620100F0010200EBD07002EB600000
:10B69000401C491C0D2900DB0D2189460D2800DBCB
:10B6A0000D2082460D2C00DB0D2427460D2D00DBDE
:10B6B0000D254046B8F10D0F00DB0D20804600241B
:10B6C00057E0306B00EB04110EA803F009FA0E9856
:10B6D000009A594658450EDCBBF10D0F00DB0D21D9
:10B6E000511A08440E900F98A8421ADC01980D2DAB
:10B6F00005DA294604E0A2EB0A010844F2E70D212D
:10B70000401A0F9908440F9009981099C01B801E89
:10B7100081420846009924DB08440D2F07DA394698
:10B7200006E001990246A1EB09001044EBE70D2168
:10B73000084410900898119AA0EB08000199801E07
:10B740008242114411DB4046B8F10D0F00DB0D20A1
:10B750000844119000220EA8149903F01EFB58B95A
:10B7600006E0014401EB0A00E3E701EB0900F0E722
:10B77000641CB06BA042A4D8B06BA04201D14FF6BC
:10B78000FF7415B02046BDE8F08F10F00F0000D117
:10B79000012070472DE9F0410E4604002CD066B31D
:10B7A00004F1300080460DF021FD58B10068616859
:10B7B0000569284604F00CFD0746226931462846F3
:10B7C0009047D8B1314604F1240012F0A7FC0500DF
:10B7D00017D02969E06A084450F8046C40460DF01F
:10B7E00005FD0246314640460DF09BFD6168286923
:10B7F000BDE8F04104F0ECBCFEE7FEE73846BDE8EA
:10B80000F0810020FBE72DE9F0474FF000080546E6
:10B810001C4616460F464046C3F8008006E0E96B1A
:10B82000226851F82010401C11442160B042F6D328
:10B83000002128460FF0EBFE0128284615D00FF016
:10B840007FFB2168081A20600021284610F020F8AC
:10B85000216808442060E96B51F826100844401E16
:10B86000A0600020C4F804801FE00FF069FB21688D
:10B8700008442060284610F02DFA81460021284611
:10B8800010F024F822680146A9EB0200401AA060DB
:10B89000E96B51F82610401A2060E2E7A96B626854
:10B8A00051F82010401C11446160B842F6D30021C9
:10B8B000284610F035F861680844606028460FF0AB
:10B8C00045FB6168081A6060A96B51F827100844AD
:10B8D000401EE060BDE8F0872DE9F05F89469346A1
:10B8E000824600210FF0BCFF0546002150460FF0B4
:10B8F000D8FF8046002150460FF0FAFF0446002191
:10B9000050460FF080FF0646504610F0E3F9411B09
:10B91000A1EB080750460FF079F9001B801B874206
:10B92000504605DA10F0D6F9411BA1EB080003E000
:10B930000FF06CF9001B801B00EBD0704010DAF8A0
:10B94000141042190A44C9F800200219DAF8181034
:10B95000BBF1000F0A44C9F8042001D0CBF8000065
:10B96000BDE8F09F002185220FF0E0BF0021862274
:10B970000FF0DCBF002187220FF0D8BF032901D2CE
:10B98000012300E00023C01A03EB430301EB830112
:10B99000891EC1EB41110C23B1FBF3F11144642268
:10B9A000B0FBF2F2014401EB9001891A4FF4C87226
:10B9B000B0FBF2F008440721B0FBF1F201FB1200EA
:10B9C000C0B2704710B50446806C002804D14420F2
:10B9D0000DF030FD08B1A06410BDFEE72DE9FC4775
:10B9E000A9B1856900220427688AC0F308030CE026
:10B9F000AE6802EB820456F8240007EB8404345B43
:10BA0000081A844206D8521C92B29342F0D8002001
:10BA1000BDE8FC8702EB82041221AB6801EB8401D4
:10BA20000026595C062702290BD04FF00C0961B1A2
:10BA3000274A08234FF0100C03290FD0012926D0E4
:10BA400043E007EB8401595A3EE009EB840107EB20
:10BA5000840259589A5A085C161836E0ADF804006A
:10BA60000092A8680CEB840103EB8408425A50F85A
:10BA70000810022301A815F075FE30B3A96851F82B
:10BA80000820801A07EB84024010895A1CE0ADF8A8
:10BA900004000092A8680CEB840103EB8408425A6E
:10BAA00050F80810022301A815F05CFE68B1A968DF
:10BAB00007EB840351F80820801A09EB8402401038
:10BAC0008A58C95A32F810000E183046A0E7000014
:10BAD000D98E02082DE9F0410D46044600F0C7F862
:10BAE000071E17D0B86900212E1A384610F020F82A
:10BAF0000AF097FE05460021384610F03DF800EBAD
:10BB0000D07106EB6101284491FBF0F0E16B8142BA
:10BB100000D8481EBDE8F08170B5064600252846CD
:10BB20000BE000BF0BF0B2FF012820460AD00BF05B
:10BB30006FFFB04200D1254620460BF06FFF040096
:10BB4000F0D1284670BD0000FEB5836980690025EC
:10BB50005B8AC4689B04A06826D4830F14D0012399
:10BB6000B3EB907F2CD1174826688DE80700A068BA
:10BB7000042320F04042314601A815F0F3FDF8B14E
:10BB8000801B801061681AE00F4826688DE8070066
:10BB9000A068022320F04042314601A815F0E2FDE2
:10BBA00070B1801B4010EDE76368805C595C39B16F
:10BBB00030B1637B2268491E11FB0321401E0D56E4
:10BBC0002846FEBD89D700089DD700082DE9FC5FF7
:10BBD0000E461D46174682464FF400310FF0F6FC24
:10BBE00000EBD07044103F1B5046FFF7ECFCBAF856
:10BBF0005C1001EB000909F15A0000B215F078FD64
:10BC000078434FEAE0380FFA89F015F071FD784378
:10BC1000C7134FF44039494650460FF021FE834682
:10BC2000494650460FF03DFE0190494650460FF000
:10BC30005FFE0090494650460FF0E5FD3268204413
:10BC40004244A2EB0B01091B29603268019942446E
:10BC500021441144A9607168CA190099511A091B3D
:10BC60006960716839440844E860BDE8FC9FC06AB7
:10BC7000002802D000210EF0E8BE704700210EF02F
:10BC8000E4BE70B590F85C100024C90600D501240C
:10BC9000054600210FF09DFF6FF0404188420CD116
:10BCA000002128460FF06AFD6FF06041884204D100
:10BCB000688D000501D444F00204204670BDB0F543
:10BCC000806F01D201207047800A70472DE9F04152
:10BCD00004460F46618D00200426C1F305120FE0D3
:10BCE000E36806EBC0055B59DD0108D523F07F430F
:10BCF000BB4204D1E16851F83000BDE8F081401C3E
:10BD00008242EDD84FF0806000EBB1204FEAB05096
:10BD1000608510F47C7F41D0C0F30510C100E0685D
:10BD200012F0C0FAE060C0B3608DC0F305156D1E5F
:10BD300016D06FF003025300E06802EBC5014158D2
:10BD40005FEAC11C0CD489010AD403EBC50C00EBDB
:10BD5000C50184446D1EDCE9000CC1E9000CEBD187
:10BD6000E068082100EBC5000DF09DFC0C200DF0F3
:10BD70003DFBE16841F8350013F03BFCE26806EB5F
:10BD8000C500115841F080711150E26867F3170146
:10BD90001150E06850F83500AFE700E0FEE7FEE73D
:10BDA0000969C06A0844001F704700007FB5164645
:10BDB0000A4690F83B5004462946104606F080F9A2
:10BDC000072D25D0082D25D0092D25D00A2D25D0C9
:10BDD0000021626AD268A2EB8101B1FBF0F4B442A7
:10BDE00000DD34460020134E00900290254601905D
:10BDF000681E03906A463221306905F0E1FA684610
:10BE000002F0F4FEA0420CDD6D1E002DF0DC0AE015
:10BE10000221DEE70421DCE71021DAE74FF480712C
:10BE2000D7E7002D02DC002004B070BD0398401C51
:10BE3000FAE70000E04E0020491E01D5401E0C31FB
:10BE40000C2901DB401C0C3901290DD0072091FB86
:10BE5000F0F200FB121000EBD07121F00101401A4A
:10BE6000C0F11F00C0B2704781070CD16421B0FB44
:10BE7000F1F201FB120149B94FF4C871B0FBF1F2C4
:10BE800001FB120010B100201C30EBE70120FBE7A2
:10BE9000136821B15B1E13600BD4806805E05B1C46
:10BEA00013608068018D8B4203DA006850F823002C
:10BEB0007047002070472DE9FC4115460E460446A8
:10BEC0000BF09AFD0BF0E2FD01280AD0032808D000
:10BED0004FF6FF7005B1286006B130600020BDE864
:10BEE000FC810BF089FD69460BF0A4FD4FF00008C2
:10BEF00055B320460FF024F800994718002120463A
:10BF00000FF085FB01280BD0606900213F1A204605
:10BF10000FF0BEFC3A1A00204146C5F8008010E040
:10BF2000002120460FF0D2FC0146E069401AC21BF6
:10BF3000F1E7E36B53F821301844824204DB491CDB
:10BF40002960E36A9942F4D3DEB120460EF0FEFF89
:10BF500001990844A169451A002120460FF0E0FC30
:10BF60002A1A00204146C6F8008007E0A36B53F868
:10BF700021301844824204DB491C3160236B994212
:10BF8000F4D30120ABE72DE9FF4F81B005460398BC
:10BF900080081E2800D91F20012787401FFA81F83A
:10BFA0006FEA080080B2009095F82A0001F47F093A
:10BFB000C0F3C00A4FF0FF3600244FF0040B1CE022
:10BFC000E96801EBC400426892013DD5BAF1000F67
:10BFD00012D10BEBC4028958C1F30741090449454A
:10BFE0000AD103685868384206D0DDE903121846C2
:10BFF00013F0DBFA01282FD0641C688DC0F3051004
:10C00000A042DDD820E0E96851F8340042683A42A5
:10C0100019D00BEBC4028A58C2F307410904494501
:10C0200011D11FFA82FA009A1AEA020F0BD1B24517
:10C0300009DDDDE9031213F0B8FA012803D15046F7
:10C04000C24508D00646641C688DC0F30510A042A6
:10C05000D9D8002E03DB012005B0BDE8F08F002009
:10C06000FAE72DE9F04742F300061D460F468146E8
:10C070005408761C15F037FBA7EB040800FB08F00A
:10C08000C711484615F034FB00FB08F0C011002F23
:10C0900006DD803F39120A1B324421442A6005E044
:10C0A000803739120A1B2144891B2A60A9600028A5
:10C0B00006DD80380012011B31442044696005E030
:10C0C00080300012011B2044801B6960E860BDE8DD
:10C0D000F087002184220FF029BC2DE9FF4F87B0A3
:10C0E0000746DDE917BA0D4609980AF09AFB00EBFE
:10C0F0000B0101EB0A000490FC6A0BEB0A006C4395
:10C10000A1460025039053E07B6B53F8241079B3CC
:10C11000FA6B0092002652F825E04FF0040C401E06
:10C120000FE0A21953F8222072B11278D2070BD077
:10C1300005EB0608009A0CEB8808761C52F808807C
:10C14000C64472198242ECD30878800711D5099849
:10C150000AF067FB00EB0B0104985144814206DDB5
:10C1600009980AF05EFB00EB0B0101EB0A0004905A
:10C170001CE0DDE915010144AEEB01001499CDE9A5
:10C18000001000220292786B50F82410DDE9092398
:10C1900005A8083114F04EF906990398084404994B
:10C1A000884200DC0846344435440490641C6D1C0D
:10C1B000F86A00EB0901A142A6D804980BB0BDE8CB
:10C1C000F08F002189220FF0B1BB00218A220FF0ED
:10C1D000ADBB2DE9FF410C46064600210FF0AEFC39
:10C1E00005464FF4802130460FF0A8FC074628464C
:10C1F0000AF017FB054638460AF013FB07460021F4
:10C2000030460FF0BFFC0146781900EBD07001EB0F
:10C21000600530460EF0FAFCB16900EBD07001EB1E
:10C22000600005EBD571A0EB610060602844E06020
:10C23000694630460EF0B8FC009820600298A06075
:10C24000BDE8FF81F0B585B00446FFF717FD060095
:10C250001DD04FF48027394620460FF06FFC05466D
:10C26000394620460FF07CFC044630460CF0F4F8CA
:10C27000014600206FF06042CDE9000202902346A3
:10C280002A4603A814F0D6F8039805B0F0BD0020A4
:10C29000FBE700002DE9F0411E461446054601F477
:10C2A0007F07FFF770FE012829D08D2C02D2184895
:10C2B000005D05E01748006BA0B1A4F18D01405C62
:10C2C00010F0010F0ED00FB1002700E06D68EDB146
:10C2D000298D3346394322462846FFF754FE01286C
:10C2E0000DD0F3E797B9012C01D0022C0ED12868AC
:10C2F0000AE0012C05D0C16929B101203160BDE8F7
:10C30000F0818169F8E700680028F2D10020F6E7A3
:10C3100094110308E04E00202DE9F04104460D463B
:10C32000638D00200422C3F305110AE0E66802EBE6
:10C33000C007F659B70103D526F07F46AE4202D0BA
:10C34000401C8142F2D8814204D0E16801EBC00078
:10C35000BDE8F0814FF0806000EBB3204FEAB050B1
:10C36000608510F47C7F2FD0C0F30510C100E06819
:10C3700011F098FFE060608DC0F30510401E0DD0F5
:10C380006FF00702E16802EBC00601EBC0030E4448
:10C39000401ED6E90016C3E90016F3D10821E06873
:10C3A0000DF081F90C200DF021F8E168086013F020
:10C3B00020F9E168486840F000704860E16865F382
:10C3C00017004860E068C3E7FEE72DE9F041051E6D
:10C3D00005D005F1300006460CF021FF0DE0FEE728
:10C3E00020686968006903F0F3FE074603F0F4FE75
:10C3F00038B1214630460CF00FFF0400F0D1BDE803
:10C40000F0813846FBE7000038B50F480D4614466A
:10C41000D0F8B0014FF0020190F82400C0074FF0AF
:10C42000120002D011F090FC01E011F0ADFC2246A8
:10C43000294604F0CDFC0090BDF800009DF80210E4
:10C4400040EA014038BD0000E04E00202DE9F047F1
:10C450004FF0000CDDE90964089DDDF82CA0E146F1
:10C460006F1EF1B9052A03D0062A01D0042A02D191
:10C470000023012D01D0002107E001225FF000011F
:10C480009C4456F82180491CC444A942F8D3ACEB23
:10C490000301072A21D2DFE802F004070B201B1357
:10C4A0000D00C4F8009018E0411A01EBD1710CE0C6
:10C4B000411A0BE0411A91FBF7F3C4F800900CE02D
:10C4C000411A91FBF5F303EBD3714910216004E0AD
:10C4D000421A691C92FBF1F3236000210BE000BFBC
:10C4E00054F8212056F821C0624404EB810C1A4410
:10C4F000491CCCF80420B942F2D304EB850106EBC9
:10C50000850251F8041C52F8042C114422688A1A3E
:10C51000BAF1000F0DD0002109E000BF54F821301E
:10C5200056F82170C31ADB1B44F82130491CA9427C
:10C53000F4D31046BDE8F0872DE9F0418CB00446F5
:10C540006946F9F73BFF08A8102200210DF07FF89B
:10C5500000210E46204612220FF0E8F9054631462A
:10C5600020460FF0A5F80746314620460FF088F820
:10C57000400700D53D4400212E460F46204610229C
:10C580000FF0D4F90546394620460FF091F8804661
:10C59000394620460FF074F8800700D54544204600
:10C5A0000EF0CEFC61693144081A0A9020460EF064
:10C5B000CDFCA1692944081A00250B9007E000680A
:10C5C00008AA694650F8250000F03AFF6D1CA068E3
:10C5D000018DA942F3D800980AF02EF901980AF0CB
:10C5E0002BF902980AF028F903980AF025F900219E
:10C5F00020460FF0E5FA0546002120460FF079F8B5
:10C600006FF040418D4201D0884202D1204610F0A7
:10C61000ABFA00223021204610F051FF0CB0BDE8EB
:10C62000F0812DE9F0470446C06A4FF4404103F021
:10C630003CF994F93610A08E0122FFF79FF90546C8
:10C64000A06B08B300264FF002084FF00309AF1D9E
:10C650004FF4004A15E0A06BA28E30F826109142EC
:10C660000ED108EB8601425694F936108A4207D162
:10C6700009EB860140565246C119E06A03F0DEFB21
:10C68000761CE06BB042E6D8A08E218E884210D195
:10C6900094F9360094F9321088420AD194F93300A3
:10C6A000AD1D4119E06ABDE8F0474FF4804203F048
:10C6B000C5BBBDE8F08710B502464B68127A097A0F
:10C6C00040684FF0FF348A4215D1012A01D05AB197
:10C6D0000EE0194612F014FF002809D002DD4FF0D9
:10C6E000010010BD204610BD984201D0FAD9F6E7EE
:10C6F0004FF0000010BDF5D9F1E770B5C5680446EC
:10C700001021284605F0BBFB10B1284605F013FBAD
:10C71000207A012804D16068BDE870400AF08CB826
:10C7200070BD00002DE9F04F0C46804687B00C210B
:10C7300020460CF0C8FF98F81060D8F80C7016B9B5
:10C740003869002824D00AF095FFDFF818A15FEAC5
:10C75000000908F1140B1ED0012E26D18DF80460BB
:10C76000009700226946DAF8200103F0A1FC0500D9
:10C7700013D003F028FD00F108010EC984E80E0073
:10C78000446900222946DAF8200103F04CFD2046D6
:10C7900007B0BDE8F08F012E07D102223946584676
:10C7A0000AF0C0F808B10020F2E72F4800900CF022
:10C7B0001DFD13E0286868B1686858B10022114671
:10C7C00058460AF0E1F92B68224641462846984728
:10C7D000012808D0294600980CF01AFD0500E9D17F
:10C7E000012E16D018E020890004000CF8D1208812
:10C7F000C0F30720142808D004F09EFAA18889B25B
:10C800004843C01DC0082081EAE7A0880004C00B8F
:10C81000F9E758460AF032F8B9F1000F1CD0012EA2
:10C820001AD1CDB18DF80460384612F07FFE05951F
:10C83000009094E8070002AB544683E8070000220A
:10C840006946DAF8200103F058FC010006D0002206
:10C85000D4F8200103F0E7FC284699E7009809F096
:10C86000EBFFA0E7E04E0020F04F002010B502469D
:10C870000B681279097900684FF0FF348A4215D1AC
:10C88000012A01D05AB10EE0194612F039FE0028F3
:10C8900009D002DD4FF0010010BD204610BD9842C6
:10C8A00001D0FAD9F6E74FF0000010BDF5D9F1E755
:10C8B0000179012902D1006809F0BEBF704700006C
:10C8C0002DE9F04F95B083461EA8894690E84005B3
:10C8D000B1F84810ADF8181099F84A008DF81A0010
:10C8E000106B0790506B0890244DD06A1C46174679
:10C8F00060B114B12068A84208D1CDE9006806AB48
:10C9000049465846D04715B0BDE8F08F98E80F006B
:10C910000DF1080C8CE80F0070684242306841420B
:10C9200002A802F0C9FA04B90DAC25606560A560E3
:10C93000E560224602A938460AF088FC054694E8DC
:10C940000F000DF1240C8CE80F00D6E9001209A8A5
:10C9500002F0B2FA012DD6D109AA414611A802F07F
:10C9600066F90028E5D011A909A8CDE9000106ABB8
:10C970003A4649465846D047DBE70000010000E050
:10C980002DE9FF4FADB0C86ADDE93A970E4638B9D8
:10C99000316B4FF48070814202D1716B814201D0C2
:10C9A000012000E000201A90B06E08B1012500E0DF
:10C9B0000025D46A2C2200212069169020891FFAB4
:10C9C00080FA2088C0F3072B07A80CF040FE96F8E9
:10C9D0004C008DF8300096F84D00CDF824A000F002
:10C9E0000F008DF844001A98284357D1BBF10E0F61
:10C9F0000ED096F84B00BBF1140F24D002284DD86E
:10CA00001698CDF82C90CDE907908DF828B03EE02F
:10CA10002D9849468268684602F009F900283AD004
:10CA200016980D9000200890CDE90F9A36F8480F1F
:10CA3000ADF83100B0788DF8330002208DF8380061
:10CA4000CDF81C9023E0022828D8484602F0CEF802
:10CA50000546484602F0D9F8169908910D91CDF88F
:10CA60002C900AFB00F1A088CDF81C9080B2B1FB9D
:10CA7000F0F00D9900FB05100D904FEA5A00CDE93A
:10CA80000F9002208DF8380012208DF8280007A999
:10CA90002D9807F0AAF831B0BDE8F08F1A988543B9
:10CAA0004BD096F84B00022847D8002219A8B16E47
:10CAB0000AF004FC074601282ED1249860B30088B0
:10CAC000C0F307200E2801D0062825D1249D28690F
:10CAD0000D90288980B2109006F15400044602F0AF
:10CAE00094F8002800DA4C4668680022010C491EC0
:10CAF00083B20091114602A85B1E02F0EAF9002001
:10CB000003460090092202A9204601F0D9FE02A89E
:10CB10000F9002208DF838001698CDF82C90CDE9B2
:10CB200007908DF828B007A92D9807F05EF8012F1F
:10CB3000B1D119A80AF062FBADE797E80F0020AC6D
:10CB400084E80F0020A80790484602F05EF817908E
:10CB5000484602F04BF8069020A802F056F8054629
:10CB600020A802F043F880465C46BBF1060F04D1D2
:10CB700096F84B00022800D910241A9838B10F2CCF
:10CB80000CD0112C0AD0122C0AD0062C25D020460D
:10CB900004F0EFF81990142C07D023E010241DE0C6
:10CBA0001424204604F0E5F8199005EB45000090A8
:10CBB00011F0B6FB04F0F6FA870011F0B1FB04F0B7
:10CBC000D7FA04F0D6F847430098B7FBF0F7404691
:10CBD000474500DD074600981DE01524204604F077
:10CBE000C8F81990204604F0C4F86843039011F087
:10CBF00097FB04F0D7FA870011F092FB04F0B8FA23
:10CC000004F0B7F847430398B7FBF0F740464745B1
:10CC100000DD0746039878430CF0E8FB1590A8B1B7
:10CC200008908DF8284023981F90781E219926900F
:10CC30000844239020A80B90142C08D00E2C17D059
:10CC4000204604F096F86843099086E1FEE7690003
:10CC50000991159A05FB07F102EB41010D91CDE910
:10CC60000F0502208DF8380012208DF8280074E19D
:10CC700008990D91CDE90F0502208DF83800B6F81E
:10CC80004800ADF8310096F84A008DF833000020D6
:10CC9000089062E12098CDE91B0122981D9023980D
:10CCA0001E90D9F804004242D9F8000041421BA866
:10CCB00002F002F91A9878B1159A3098CDE904B2C9
:10CCC000CDE902600699CDE9001ADDE916231BA91A
:10CCD0002D9808F089FC9EE096F84B0002287CD342
:10CCE0001BA801F083FF0746BBF1060F16D0142CDA
:10CCF0003DD00E2C3AD01C981B9A199900FB0AF0D3
:10CD000002FB010116984FF0000808441490159892
:10CD10001999019005FB01F003907AE0DDE91B12FF
:10CD20000AFB021116984FF0000E01444FF0FF0865
:10CD3000159A19E0002010E002EB800311F800C002
:10CD400083F802C011F800C083F801C011F800C0D8
:10CD500002F820C083F80380401CA842ECDB02EB01
:10CD6000850251440EF1010EBE45E3DB53E04FEA6C
:10CD70005A011C980191484316991C9A01EB4001F5
:10CD80001B984FF0000801EB40010291019901FB53
:10CD9000020206984143169800EB410010440590AA
:10CDA000159803900D980490680027901EE000BF2E
:10CDB000DDE90210279A0CF08FFBDDE904012A4619
:10CDC0000CF08AFBDDE9011000EB410002900599AF
:10CDD000019808440590039800E084E000EB4500CA
:10CDE0000390049808F1010828440490B845DFDB5B
:10CDF00011E0039A149901980CF06EFB01991998AF
:10CE000008F1010805FB00101499019001EB0A00DC
:10CE10001490B845EDDB96F84B00022863D9B16C4D
:10CE20008046C0F1FF070191142C1ED0122C1CD09B
:10CE30000E2C7AD020A801F0DEFE01460198C2B285
:10CE400012FB08F3C0F3072212FB08F003900198CD
:10CE5000C0F3074212FB08F2DDF864C0002001FBBA
:10CE60000CF1DDF854E005915DE0C1F3C40111FB64
:10CE700008F014900198C0F30720810811FB08F016
:10CE800005900198C0F30740C10811FB08F001901C
:10CE90001598009020A801F0AEFE864600204FF4C1
:10CEA000FC621EE0DDE9001331F810804FEAD82162
:10CEB00011FB07314FF4784303EAC10C059BC8F31B
:10CEC000451111FB073102EAD1018C44149B08F093
:10CED0001F0111FB0731009B0CEB112123F81010EF
:10CEE000401C7045DEDB20E01EF8001011FB07310E
:10CEF0004FEA112C0EF800C00EEB0001DDF80CC05B
:10CF000091F8018018FB07CC4FEA1C2C81F801C076
:10CF100091F802C01CFB072C4FEA1C2C81F802C0C0
:10CF20001999084405998142DED807A92D9806F081
:10CF30005CFE2398401C2190269908441F99239059
:10CF400088420ADD2391142C07D120A801F04EFE5F
:10CF50001599684301EB40000D9021991F9881427B
:10CF60007FF798AE159809F067FC94E52DE9F0413C
:10CF70000446807A0D4640F00200A0721E4800264A
:10CF8000016DA14200D146652078012801D0022818
:10CF90002FD115B1606FA84201D1666715B1A06E9F
:10CFA000A8420DD1A76E57B1224614213846A66675
:10CFB00010F085FA3A46142120460AF08FFD15B18B
:10CFC000E06EA84201D1E66615B1206FA8420CD1EF
:10CFD000206F48B122461421266710F070FA3246BD
:10CFE000142120460AF07AFD15B1A06FA84200D1A5
:10CFF000A667BDE8F0810000E04E00202DE9F04179
:10D00000044690F83C0000F0030001283CD1E16A9E
:10D01000A06BB1FBF0F0216BB1FBF0F200FB121141
:10D02000A26B520802FB0011B1FBF0F2216300FB7E
:10D030001211A26B520802FB00116163204600210D
:10D040000EF07CFD0546002120460EF09BFD0746B4
:10D05000284609F0E6FB054620460DF083FD06460E
:10D060002046FEF70BFE0246216BE819414306EB12
:10D07000D67305EBD570BDE8F0415B10A3EB600003
:10D08000411A104610F016BCBDE8F08110B50446F8
:10D090000069B0B1A069A8B16068A0B103F0A0F8C0
:10D0A000021D04F12400216911F04FF8002807D077
:10D0B000042104F130000CF0B6F80348E0630120CD
:10D0C00010BDFEE7FEE7FEE73172000810B504462A
:10D0D0000069B0B1A069A8B16068A0B103F080F8A0
:10D0E000021D04F12400216911F02FF8002807D057
:10D0F000042104F130000CF096F80348E0630120AD
:10D1000010BDFEE7FEE7FEE76B5B020870B50D4C55
:10D11000064600200D460A4620602121304610F0C8
:10D12000CEF9206858B1017839B1294612F0E8F9F2
:10D1300028B13046216813F021FC002070BD012089
:10D1400070BD0000240100202DE9F0418CB01F4685
:10D1500014460D4606460FF07BF9002839D0A5424B
:10D1600037D04FF4B470854201DDA5F5B475844223
:10D1700001DDA4F5B474F16A0D440C44854201DD6F
:10D18000A5F5B475844201DDA4F5B4740AAA04A916
:10D190003046FEF7A1FB394630460EF017FA8046BE
:10D1A0003046394651220EF0C1FB06A908B10122D2
:10D1B00000E00022CDE90048CDE902210A982B4683
:10D1C00082B2DDE9040104F045FA06A930460FF009
:10D1D000E1F80CB0BDE8F08110B588B0044606AAAD
:10D1E00004A9FEF779FB6B4604A92046069AFEF7D0
:10D1F000EDFC204600F0DCFA011E03DD0246684625
:10D2000001F008FD694620460FF0C4F808B010BDD3
:10D21000F0B50646A1F57F408DB00F46FF384DD0E2
:10D22000B06BB8424AD9306B00EB071102A801F08D
:10D2300057FC06A930460DF0B7FC002130460EF031
:10D2400051FB0446002130460EF0FEFA05463046FA
:10D250000DF0B0FC03F09CFF0A2190FBF1F2A2421A
:10D2600001DB90FBF1F490FBF1F2AA4201DB90FBB1
:10D27000F1F506980299021B11440291079A03994D
:10D28000521B1144039104990844204404900799C7
:10D290000598084428440590306CB8420AD1706B58
:10D2A00030F81700400505D502A801F09FFC03994E
:10D2B000081A039002A930460FF06CF80DB0F0BDCB
:10D2C0002DE9FF470446006F0D46A84274D9204659
:10D2D0000DF059FC804620460DF06AFD064694F894
:10D2E0007400010705D500F00700012807D00228C7
:10D2F00063D004B02046BDE8F0470FF030B80021FD
:10D3000020460EF0DEF90746002120460EF0B1FA65
:10D31000616938440844A0EB060920464FF4A02177
:10D3200048220EF003FB06464FF4003120460EF073
:10D330004DFC074660690090A0690190E069029089
:10D34000206A03900199F019091A01910399084480
:10D350000390206F401EA84216D908FB05F1B1FBCF
:10D36000F0F202EB0901891BC91B6A1C009108FB42
:10D3700002F1B1FBF0F101EB0900304438440290B6
:10D38000694620460FF006F8002D3FD0681E08FBC6
:10D3900000F1206F401EB1FBF0F202EB0901891B86
:10D3A000C91B009108FB05F1B1FBF0F101EB09008D
:10D3B00030443844029025E028E0002120460EF059
:10D3C00046FA8146206F08EB0901B1FBF0F7002116
:10D3D00020460EF076F9824607FB05F8002120462C
:10D3E0000EF047FA616950444144451869462046A9
:10D3F0000DF0DAFBA81B0090384400990290A1EBD5
:10D4000009000090694620460EF0C4FFBDE8FF8782
:10D4100070B505460EF05EFC044628460DF0F6FB9E
:10D42000844201DB012070BD002070BD28B10A28B4
:10D4300003D00D2801D00020704701207047000064
:10D440002DE9F74F0D4686B00446CD490EF08FFC0E
:10D4500000287CD12046FEF78DFA82462046FEF752
:10D46000B4FE5FEA000972D0BAF1000F6FD0204617
:10D47000FEF77CFA07462046FEF7A3FE80462046CC
:10D48000002188220EF052FAC6B2204600218B22DB
:10D490000EF04CFAC0B20390296807EB0A006FF057
:10D4A000030303EB8000D5F808C051F82720095882
:10D4B0005CF800000844A0EB020B6A6808EB090066
:10D4C00003EB8000EB6852F82810125818581044EB
:10D4D000401A0290002120460EF087F8012806D15C
:10D4E00016B1022E02D002E0022600E0002604F16E
:10D4F0001400019001F089FB0090019801F076FB87
:10D500008246012E38D0022E4FD0032E4FF000015C
:10D51000204606D00EF017F9296851F82710084464
:10D5200051E00EF010F9296851F8271000EB0109BD
:10D53000002120460EF007F90646002120460EF095
:10D540000BF93044ABEB00000090608D00E014E17B
:10D5500040F400606085039801287CD002287BD0CD
:10D5600003284FF00001204632D00EF0FEF86A6822
:10D5700052F828104718B8E000992046ABEB010993
:10D5800000210EF0E0F80646002120460EF0E4F8F7
:10D590002968301A00EBD07051F8272009EBD971B7
:10D5A000491001EB600010440DE020460EF092FBA4
:10D5B000296851F8272002EB0B010E1A00212046A2
:10D5C0000EF0CAF8301A8146608D20F40060C1E781
:10D5D0000EF0CBF86A6852F8281047180021204650
:10D5E0000EF0C3F80546002120460EF0A3F802997C
:10D5F0002844A1EB000A608D40F4806060852046DD
:10D600000EF068FB0099884204D120460DF0FEFA26
:10D61000504524D060690290A0690390E0690490AD
:10D62000206A059020460EF09AFEDDE9001001F018
:10D630005AFC5146019801F051FC20460EF08FFE35
:10D6400002AA2E2120460FF03AFF20460DF02EFBB5
:10D650002246272101E021E039E00FF030FF20468B
:10D6600000216A220EF062F90646204600216B2254
:10D670000EF05CF9054620460EF02CFB8246204653
:10D680000DF0C4FA3F4A0146C6F3417053104FF003
:10D6900080584FF0640C01282BD035E0029800210F
:10D6A000A0EB0A0620460EF060F80746002120464F
:10D6B0000EF040F86A68381A00EBD07052F8281063
:10D6C00006EBD672521002EB60000F180DE02046F8
:10D6D0000DF09CFA6A68029952F8282011440D1A3C
:10D6E000002120460EF026F82F1A608D20F480606D
:10D6F00084E726F0C040904206DC404500DB181A63
:10D7000000FB0AF090FBFCF6C5F34170012809D13B
:10D7100025F0C040904205DC404500DB181A484324
:10D7200090FBFCF5089A09EB060178199268114400
:10D7300062698D1A0899C9680844A169461A55EAB0
:10D7400006001AD020460EF00AFE60692844606187
:10D75000E0692844E061A0693044A061206A304457
:10D76000206220460EF0FBFD09B0324629462046D5
:10D77000BDE8F04F00230EF09BBE09B0BDE8F08F6E
:10D7800001000600FEFFFF1F0A880368934201D0D4
:10D79000981A704740684988401A70470A780368A9
:10D7A000934201D0981A704740684978401A7047F0
:10D7B0002DE9F0414FF4403604463C2231460EF04C
:10D7C000B5F805462046422231460EF0AFF8054432
:10D7D000314620460EF0C5F800283146204602DDCD
:10D7E0000EF0BFF802E00EF0BCF8404205443146AE
:10D7F00020460EF0BCF800283146204602DD0EF02F
:10D80000B6F802E00EF0B3F8404205442046382254
:10D8100031460EF08BF8074620463B2231460EF08B
:10D8200085F83844854200DD2846BDE8F08170B5B2
:10D83000054608F06FFD0446284608F06FFD0646D1
:10D840000DF034FA05462F2C01D02E2C0BD10021DF
:10D8500030460BF0C7F9284615F0C8FD2846BDE84C
:10D86000704018F085B970BD2DE9F0438DB00746C2
:10D870001D46164689460846DDF850800DF0BCF975
:10D880000446414648460DF08FF92246114640466F
:10D8900001F0C0F907F11804022E05D0012E32D094
:10D8A00000200DB0BDE8F08398E80E00D8F80C0019
:10D8B00003908DE80E000022694648460EF092F96A
:10D8C0006A46214604A801F0B2F90028E9D004AC68
:10D8D00094E80F0008AC84E80F00022208A948462B
:10D8E0000EF080F908A94246084601F0A0F9002888
:10D8F000D7D094E80F0085E80F000522114628468E
:10D9000001F088F90AE042462146684601F08FF9A5
:10D910000028C6D09DE80F0085E80F000120C0E771
:10D92000F8B504460E46001D01F060F90546201DBD
:10D9300001F06BF900960246217D2B46206804F029
:10D940009AFB002800D1FEE7F8BD70B504460DF043
:10D95000BBF80646002506E0A068006850F82500E0
:10D96000FFF7F3FF6D1CB542F6D3608DC1070CD0F5
:10D9700020F00100608520460FF0F6F820460FF0F9
:10D980001FF816B120460BF0ABF9608D810708D562
:10D9900020F0020060852046BDE8704000210EF0B6
:10D9A00076BE70BD2DE9F0478046089D1F46A86AE7
:10D9B00000FB01F39B12002807DD934207DD00BF47
:10D9C00095F8340080070DD48BE09342F8DBCB1937
:10D9D00043439B12002808DD934239DA95F834005E
:10D9E00080077ED40120BDE8F0879342F6DC686AA8
:10D9F000521C504340F395000312C0B2FF2200288E
:10DA000028D000BF2E6BC0F1FF0404FB06F4A2EB8C
:10DA1000242600BFA3EB0104A14636D0002C15DB61
:10DA2000BC4213DAC0F1FF00C6F1FF014843A2EB8C
:10DA30006020C1B295F83400800701D5C1F1FF0123
:10DA400018F8040014F080F908F80400641C1CE0C5
:10DA5000686ACEE74FF0FF06DCE7002C10DBBC4223
:10DA60000EDAA6EB6000C1B295F83400800701D54C
:10DA7000C1F1FF0118F8040014F066F908F8040079
:10DA8000286B641C361ABC4202DA286BB042E4DB15
:10DA9000BC4218DA002C16DB686A704380127043AF
:10DAA000C0F34721A86A002801DAC1F1FF0195F807
:10DAB0003400800701D5C1F1FF0118F8040014F00B
:10DAC00043F908F8040095F83400800707D5494663
:10DAD000B94506DC00290DDB404609E001E0641C85
:10DAE00001D500207FE7BC4204DC391B08EB0400B1
:10DAF0000BF0F1FD022076E72DE9F05F06460A9F64
:10DB00008A461D46786A00FB02F18C12002800DD6F
:10DB1000641C97F83430544502DA980707D4D5E0EE
:10DB20008C120AEB050CA44502DA98077ED483E038
:10DB3000521C424341F3950142F395044FEA2129D7
:10DB4000221204F0FF08C9B2A9EB0A04914505D0DE
:10DB5000002803DA11B9FF219146641E914528D1AE
:10DB6000002C0CDBAC420ADA01EB080041089807F4
:10DB700001D5C1F1FF01305D14F0E6F8305597F89A
:10DB80003400641C800706D5A9EB0A01A9424DDACE
:10DB90008EE030460AE0AC4200DD2C46002C45D039
:10DBA00006DD00BFA5EB040106EB04000BF093FDBE
:10DBB00089E04FF0FF0B002844DAB86A404248433E
:10DBC0004FEAA028002C0DDBAC420BDA08FB01F079
:10DBD000C0F34721980701D5C1F1FF01305D14F072
:10DBE000B3F83055796AA8F1FF0041438812641EEA
:10DBF00011D4AC420FDAC8F1FF014143ABEB612015
:10DC0000C1B297F83400800701D5C1F1FF01305D42
:10DC100014F09AF8305597F83400A41C800709D501
:10DC2000A9EB0A01491EA9424DDC00E04EE00029A3
:10DC3000AFDC48E0AC4202DD0120BDE8F09F002CE3
:10DC4000B0DA40E0C1F1FF00B96A41434FEAA128D0
:10DC5000002C0EDBAC420CDA00FB08F0ABEB6020D2
:10DC6000C1B2980701D5C1F1FF01305D14F06CF825
:10DC70003055796AC8F1FF0041438912641C0ED403
:10DC8000AC420CDA4843C0F3472197F834008007D0
:10DC900001D5C1F1FF01305D14F056F8305597F809
:10DCA0003400641C800707D5A9EB0A01A9420DDCEA
:10DCB0000029BFF66EAF06E0AC4200DD2C46002C1A
:10DCC00004D03FF76FAF4FF00200B6E74FF000000F
:10DCD000B3E7FEB5C46A09F08FFE054609F0D6FE2B
:10DCE00004280CD1216C204661640CF08AFF0646A2
:10DCF00009F0B4F818B10021304609F024F928469B
:10DD000009F0C4FE012804D0284609F0BFFE03280C
:10DD100009D16946284609F08DFE20460199FDF794
:10DD2000D9FE20646064204607F08CFF206B10B998
:10DD300020460EF014FB206C029002AA20212046FF
:10DD40000FF0BDFBFEBD000010B5582109480BF0D7
:10DD50006AFA00222121084813F08EFA054CAC3CE7
:10DD6000C4F8A800A434F8F75BF8002020706070B5
:10DD700010BD00008C4F0020515E00082DE9F041DD
:10DD800005460F480E460024074616E00168A942E2
:10DD900000D01DB94168B14209D046B101463846AC
:10DDA0000BF036FA0028F1D12046BDE8F08116F0DC
:10DDB00025F8F8F735F8012438460BF017FAF1E7A3
:10DDC0008C4F002070B505460A480C4606460BF0FD
:10DDD0000DFA0BE00168A94204D14168A14207D0C5
:10DDE000002C05D0014630460BF012FA0028F1D184
:10DDF00070BD00008C4F002010B504465822002151
:10DE00000BF025FC4FF4FA70206300206062642060
:10DE1000E062012060640448206294F8540040F0FD
:10DE2000080084F8540010BD99DE00082DE9F8437D
:10DE300004464FF48060174600901E46D4E90C203B
:10DE400088460023089D19460BF008FB33463A46E6
:10DE50004146009503F02CF8626AE16A891A414351
:10DE600002EBA120BDE8F88308B5B0F94E2000927E
:10DE7000B0F94C30B0F94A20B0F94810FFF7D6FF9E
:10DE800008BD08B54FF480610022009140F2512393
:10DE90001146FFF7CBFF08BD38B504464FF480604C
:10DEA0000090D4E90C20002319460BF0D7FA626ADF
:10DEB000E16A891A414302EBA12038BDD0E90C1276
:10DEC0008A4201DBC06A7047406A70470020F7F75A
:10DED000BFBF10B5029C20F8481F83804280C480D9
:10DEE00010BD01617047494241637047416170470D
:10DEF0000163704710F8542F61F3C302027070473A
:10DF0000416070470162704781637047C163704729
:10DF10004164704701647047C1607047C1617047D8
:10DF200041624FF00041C0E90A127047016070473A
:10DF300010B542F2107442F2F673A04200D91846AE
:10DF4000A14200D91946A24200D91A460A23401D0F
:10DF5000491D521DB2FBF3F2B1FBF3F1B0FBF3F03C
:10DF6000120502EB8121084400F1004010BD0000C1
:10DF700070B5054620480BF05EF9040028D0582201
:10DF800029460BF0A9FA2868A84200D124601A4853
:10DF9000AC3890F8A51014F8540F61F3410004F860
:10DFA000040913F013F901C414F8540900071FD52C
:10DFB000A16939B120468847616A01446162E16A1A
:10DFC0000844E062204616F037F8686818B900E0A7
:10DFD000FEE7A86810B1204615F04EFF626812B146
:10DFE000616A20689047A26812B12046616A904732
:10DFF000F7F716FF204670BD8C4F002010B5D0E912
:10E000000E431B1B02E000BF03F5B473002BFBDBC8
:10E010004FF4B474A34202DBA3F5B473FAE7994258
:10E020000FDC03EBD372B1EB620FC16C02DA41F08B
:10E03000080101E021F00801C0F84C1041F0100186
:10E0400017E0C3F5B474944203DCC16C41F00801DD
:10E05000F4E7C1F5B474944203DCC16C41F00801EB
:10E0600005E01A448A4207DBC16C21F0080121F067
:10E070001001C164012010BD002010BD10B50C4678
:10E0800087212D22C4E90E120020C4E90B014900AA
:10E090006163E16C21F00601E16413492164E16CE4
:10E0A000606441F008016420C4E9120121F001001C
:10E0B000E0641001206513F089F86065606BA0656D
:10E0C000E06C022120F01000E06420460BF039FDE6
:10E0D0004FF4447120460EF037FF2046BDE8104053
:10E0E0000D210FF00EBA00000080FFFF2DE9F04374
:10E0F000BBB0044608F012F90546204608F045F981
:10E10000814614AA31A92846FDF7E6FB1498002899
:10E110001ADD684603F087FA6A46002128460DF0AA
:10E1200030FEDDE93101CDE90B01A96BE86A084455
:10E130000990E96BE86A08440A901498ADF8340035
:10E140006946484603F03CFA4FF4003841462846F9
:10E150000DF086FB0746414628460DF0A2FB064619
:10E16000414628460DF0C4FB0446414628460DF0C2
:10E170004AFBB74201DD394600E03146844201DD09
:10E18000224600E00246914205DDB74201DD3846F5
:10E1900004E0304602E0844200DD204614990C1A67
:10E1A000002C19DD684603F03EFA6A4641462846CF
:10E1B0000DF0E7FDDDE93101CDE90B01D5E90B01FA
:10E1C00008440990696BE86AADF8344008440A9045
:10E1D0006946484603F0F4F936AB31A92846149A4B
:10E1E000FDF7F4FC15A805F0C1FA15AA4FF440316B
:10E1F00028460DF026FF36AA15A9484605F0A0F8D6
:10E200003BB0BDE8F08300002DE9F04F89B08A46AD
:10E21000FE480CF004FC01287DD1504608F07AF845
:10E220000546504608F07AF804464FF0640B4FF468
:10E23000B479022D13D0082D6ED0032DFCD00E2DF5
:10E240006BD00F2D6AD0132D69D0182D68D01A2DE0
:10E2500061D109B05046BDE8F04FFFF747BF09F064
:10E26000CBFB050057D009F011FC012853D101A9BF
:10E27000284609F0DFFB05AA03A92046FDF72CFB81
:10E2800003990198401A019002990498081A029083
:10E2900094F84C00C00731D14FF4003120460DF006
:10E2A00095F9054605984FF48031401B05902046AE
:10E2B0000DF056FD0028059806D1C11700EB9171AD
:10E2C000B5EBA10F00DA8D10401B0590012801DA93
:10E2D000012005900198029A404302FB0201059833
:10E2E0004043814206DDE06C40F00101E16412F040
:10E2F0006DFF606594F84C00C0070CD0019911B90E
:10E300000298002807D0D4E90E06864201DA06F505
:10E31000B476029805E0ABE0C0E0D9E0F6E0FBE0BF
:10E3200061E100F075FEE16A401AA16B451A01E057
:10E3300005F5B475002DFBDB4846854202DBA5F5EB
:10E34000B475FAE705984FF41D714843B0FBFBF72D
:10E35000322003F0FFF84FF4B4714843B0FBF7F2FA
:10E3600094F84C002946C0F3C0072046FFF746FE4C
:10E3700000287DD0A06BA26D311AA2EB0008A5EB9E
:10E380000800002801DD024600E042424FF48C7391
:10E390009A4205DD94F84C20120709D5002508E0C3
:10E3A000E26C5FEAC26C04D4120701D54D4200E072
:10E3B0000D4677B1E16C0A071ED4CA061CD40028AA
:10E3C00000DC4042984217DD67F3C3010025E16499
:10E3D00012E08FB9E26C5FEA027C0DD55FEAC26C95
:10E3E0000AD4002800DC4042C0F5B470984203DD36
:10E3F00067F3C3020D46E264A5EB0805606D12F0F9
:10E40000DFFE216D41434FF47A70B1FBF0F085429D
:10E4100002DC4042854200DA0546D4E91132A16BA4
:10E42000D01A771AFF0097FBF0F0001DC71745447C
:10E4300000EB177005EB2010256C00920844324663
:10E440000BF00CF8064694F84C00C0F3410002288B
:10E4500003D1A06C811B606C0E18206CB04211D0EF
:10E4600012F0B4FE60653146204600F018FA00E074
:10E4700011E0AE4206D00022202120460FF01FF806
:10E48000012808D1606CB04202D0A06CB04202D129
:10E4900012F09CFE606509B0BDE8F08FE06C20F0E2
:10E4A00001012046E1640CF0ACFB054608F0D6FC07
:10E4B000044609F0A1FA09F0E9FA0428EBD1002C8E
:10E4C000E9D009B02846BDE8F04F002108F03BBD77
:10E4D000504607F04EFF256C132806D0112804D0B3
:10E4E000142804D0122802D005E0691C00E0691E3F
:10E4F000204600F0D4F9206CA842CCD009B02046C8
:10E50000BDE8F04F002220210EF0D9BF504607F0A1
:10E510004FFF256C2918EBE7504607F047FF0546EB
:10E5200003AA01A92046FDF7D7F9A068002600B18B
:10E53000066A002120460DF049F8804603993044D0
:10E54000081A0299029A01440091019903900B184C
:10E55000121A091A04A800F0BCFC47F6FF7204A8BE
:10E56000296800F01AFC4FF0000AC0BB2868019A25
:10E5700001684068891A029A801A00F049FDE16A30
:10E58000401AA16B471A01E007F5B477002FFBDBB7
:10E590004846874202DBA7F5B477FAE703984FF4C1
:10E5A0001D714843B0FBFBF9322002F0D3FF4FF45A
:10E5B000B4714843B0FBF9F239462046FFF71EFD1F
:10E5C00068B108EB4602114604A800F023FB47F6A9
:10E5D000FF7204A8296800F0E0FB28715BE7FFE701
:10E5E00085F804A057E700210DF03AF9074600210D
:10E5F00020460DF056F90646002120460DF078F928
:10E600000546002120460DF0FEF801E0D81203086F
:10E61000B74201DD394600E03146854201DD2A4638
:10E6200000E00246914205DDB74201DD384604E0D4
:10E63000304602E0854200DD284680464FF44039EE
:10E64000494620460DF00CF90746494620460DF094
:10E6500028F90646494620460DF04AF9054649463E
:10E6600020460DF0D0F8B74201DD394600E03146D2
:10E67000854201DD2A4600E00246914205DDB742AF
:10E6800001DD384604E0304602E0854200DD2846E0
:10E69000801CA0EB08052046FFF78AF84419504675
:10E6A00007F084FE0168A14200DD0C460460F2E63A
:10E6B00070B50C460546114600F076F8214628460E
:10E6C000BDE8704000F0B6B870B50C46054611467E
:10E6D00000F006F821462846BDE8704000F032B848
:10E6E00070B505460C46B1F5B47F01DDA1F5B474F3
:10E6F000D5E90E10421AA4EB010101D502F5B4725E
:10E70000002901DA01F5B4718B1A002B00DC531AD1
:10E71000B42B03DD28460DF022FE0DE0914203DA12
:10E7200000230246214604E08A4205DA00232246FD
:10E7300001462846FEF708FD2846EC63BDE8704018
:10E740001BF01EB970B505460C46B1F5B47F01DD6E
:10E75000A1F5B474D5E90E010A1AA1EB040101D5A3
:10E7600002F5B472002901DA01F5B4718B1A002B9D
:10E7700000DC531AB42B03DD28460DF0F0FD0DE04C
:10E78000914203DA00232246014604E08A4205DA78
:10E790000023024621462846FEF7D6FC2846AC63F5
:10E7A000BDE870401BF0ECB870B505460C46B1F5FD
:10E7B000B47F01DDA1F5B474D5E90C10421AA4EBC5
:10E7C000010101D502F5B472002901DA01F5B47135
:10E7D0008B1A002B00DC531AB42B03DD28460DF0F6
:10E7E000BEFD0DE04FF40033914202DA02462146AD
:10E7F00003E08A4204DA224601462846FEF7A4FCDA
:10E800002846FEF7E9FC28466C63BDE87040FEF739
:10E81000E3BC000002E000BF01F5B4710029FBDB9E
:10E820004FF4B472914202DBA1F5B471FAE7C16210
:10E830000DF095BD70B505460C46B1F5B47F01DD10
:10E84000A1F5B474D5E90C010A1AA1EB040101D5B4
:10E8500002F5B472002901DA01F5B4718B1A002BAC
:10E8600000DC531AB42B03DD28460DF078FD0DE0D3
:10E870004FF40033914202DA2246014603E08A4215
:10E8800004DA024621462846FEF75EFC2846FEF7DB
:10E89000A3FC28462C63BDE87040FEF79DBC036CCA
:10E8A0008B420CD0826C8A4200DA1146426C8A425A
:10E8B00000DD11468B4202D001641BF061B8704745
:10E8C000F0B50D688C68D1F80CE0641BD0E90065E8
:10E8D0004F68DDF814C0AEEB0707162A75D2DFE8E3
:10E8E00002F0C7C71A272D2F454D5D0B6567757B55
:10E8F0007D8F97999B9DA1BD8268A2EB060E0EF1BC
:10E90000010E621C0EEBDE7E4FEA6E0E02EBD2723F
:10E91000AEEB620233E08068821B601C521C02EB8B
:10E92000D272521000EBD070A2EB600200208AE09D
:10E930008068621C801B401C821AF7E700220DE0F1
:10E940008268A2EB060E0EF1010E621C0EEBDE7E5B
:10E950004FEA6E0E02EBD272AEEB6202C06807F1B4
:10E96000010E401B401CA0EB0E006CE0826804F11D
:10E97000010E921B521CA2EB0E02EFE70022C068B0
:10E98000A0EB050E0EF1010E781C0EEBDE7E4FEAB9
:10E990006E0E00EBD070AEEB600054E0826804F1C4
:10E9A000010E921B521CA2EB0E02E8E700220AE0C5
:10E9B0008068821B601C521C02EBD272521000EB6A
:10E9C000D070A2EB6002F8433DE051E08068621C29
:10E9D000801B401C821AF6E700220DE08268A2EB41
:10E9E000060E0EF1010E621C0EEBDE7E4FEA6E0E7D
:10E9F00002EBD272AEEB6202C068401B401C22E008
:10EA0000826804F1010E921B521CA2EB0E02F3E786
:10EA1000E2438BE7E243B2E7E2439FE78068821B71
:10EA200000200FE08268C068921BA0EB050E0EF17B
:10EA3000010E781C0EEBDE7E4FEA6E0E00EBD070FE
:10EA4000AEEB6000521C324428441A446044C1E9D1
:10EA5000002022443844C1E90220F0BD8268C06829
:10EA6000921B401B07F1010E401CA0EB0E00E9E7D2
:10EA700000225BE70A6802604A6842608A68826036
:10EA8000C968C16070470A6802604A6842608A6863
:10EA90008260C968C16070470A6802604A68426063
:10EAA0008A688260C968C16070470A6802604A6803
:10EAB00042608A688260C968C16070470A68026003
:10EAC0004A6842608A688260C968C16070470A68A3
:10EAD00002604A6842608A688260C968C1607047A3
:10EAE0000A6802604A6842608A688260C968C160D8
:10EAF00070470A6802604A6842608A688260C96832
:10EB0000C16070470A6802604A6842608A68826031
:10EB1000C968C16070472DE9F0470C4606461546A6
:10EB20001146204600F0E6F800285CD00022294675
:10EB3000204600F09CF800284FF0000051D1E76813
:10EB400061682368A7EB010C6F68A2687F1AA2EBCB
:10EB50000309002F05DD08C60F4486E88600012062
:10EB6000361FE96862688A1AACEB0203002B0CDDE1
:10EB7000E268914209DA06EB001C2768A2684CF8AB
:10EB8000047B0B448CE80E00401C6968626891426B
:10EB900000DC1146EA68E3689A4200DB1A46531A21
:10EBA0002F682268BF1A002F0BDD002B09DD06EB52
:10EBB0000018174448F8042B01EB030C88E8821076
:10EBC000401CAA682468151BA9EB0504002C08DD6D
:10EBD00006EB00151444C5E900210B44C5E90243C6
:10EBE000401CBDE8F0874FF0FF30FAE7C16840688D
:10EBF000081A401C704702688168891AC268406818
:10EC0000101A401C491C4843704781680068081A64
:10EC1000401C704703685B1A036083681944816075
:10EC20004168891A4160C1681144C160704770B57C
:10EC30000B681468A34200DC234603604D685468E7
:10EC4000A54200DD2C4644608E689568AE4200DA2D
:10EC500035468560C968D268914200DB1146C160C3
:10EC60000120AB4201DC8C4200DD002070BD7CB590
:10EC70000D460446006809681646884238DB61681C
:10EC80006A68914234DBA268AB689A4230DCE26881
:10EC9000EB689A422CDC4EB3CDE90001324669465E
:10ECA000284600F07AF8002821D0D4E90110CDE9F7
:10ECB000000132466946284600F06FF8002816D059
:10ECC000E1682068CDE9000132466946284600F037
:10ECD00064F800280BD0D4E90201CDE900013246E6
:10ECE0006946284600F059F8002800D001207CBD74
:10ECF00000207CBD02688B689A420DDC82680B683C
:10ED00009A4209DB4268CB689A4205DCC0684968D0
:10ED1000884201DB01207047002070477CB50D461A
:10ED20000446806809681646884234DBE0686968F2
:10ED3000884230DB2168A86881422CDC6068EA6880
:10ED4000904228DC2EB3CDE90010324669462846B1
:10ED500000F023F8E8B9D4E90110CDE9000132460A
:10ED60006946284600F019F898B9E1682068CDE9AD
:10ED7000000132466946284600F00FF848B9D4E948
:10ED80000201CDE9000132466946284600F005F847
:10ED900008B100207CBD01207CBD2DE9FF41144657
:10EDA0000E460A68016805468A422EDBA868824240
:10EDB0002BDC72686B689A4227DBEF68BA4224DC6E
:10EDC000002C5DDD401A401C00EBD0704210F81A98
:10EDD000401C00EBD0704010824200DA10468442A2
:10EDE00000DD0446009128680022204402906868F3
:10EDF000019068683146204403906846FFF7CDFFD4
:10EE000038B102982044029032E0002004B0BDE8FE
:10EE1000F081E8680022001B0190E8680390314609
:10EE20006846FFF7BAFF18B10298204402900DE03F
:10EE3000A8680022001B0090A8680290314668462E
:10EE4000FFF7ABFF30B10098001B00900198001B4A
:10EE5000019010E0686801906868002220440390E7
:10EE600031466846FFF799FF50B10098001B0090AB
:10EE7000039820440390314668460FF0C5F8C5E773
:10EE80000120C3E710B50C6813689C4200DA2346E2
:10EE900003604C6853689C4200DA234643608C68E8
:10EEA00093689C4200DD23468360C968D268914222
:10EEB00000DC1146C16010BD03680B440360836829
:10EEC00019448160416811444160C1681144C160C6
:10EED000704710B5029C80E81E0010BD4268491EB4
:10EEE0001144C16070470268491E11448160704737
:10EEF00042688A4201D80020704702681AB1C0688F
:10EF000001FB00207047FEE770B50446006800254D
:10EF100010B107F091FC25606560A56070BD00210F
:10EF2000FFF7E6BF10B50446231D002083E8070065
:10EF300001FB02F00AF05AFA2060002800D1FEE737
:10EF400010BD70B5044600680D46A0B1D4E90101BA
:10EF5000884203D12046091D00F00EF8D4E90001D3
:10EF6000E26801FB020029460AF0B6FA6068401C1C
:10EF70006060012070BDFEE770B50D46C1680446B3
:10EF8000694300680FF08EF930B1A56020606068B9
:10EF9000A84200D9656070BDFEE740687047000078
:10EFA0002DE9F04781468A46002012F0D7F9044641
:10EFB0004FF000080E4F16E0204612F0CFF905463C
:10EFC000A068B8420ED1E668316849450AD1716837
:10EFD000514507D1204612F077F9304607F02CFC56
:10EFE0004FF001082C46002CE6D14046BDE8F087E2
:10EFF000F5EF000870B5C568D5E9004612F064F970
:10F00000284607F019FC3046A446BDE8704060472A
:10F010000022002801DA01224042002901DA494297
:10F02000921C884207D9C1EB011101EB4101B1FBF0
:10F03000F0F3103205E0C0EB001000EB4000B0FB35
:10F04000F1F30020D9B216290BD92C2900D80120C0
:10F05000292900D8401C252900D8401C20290BD97B
:10F060000BE0022900D30120062900D3401C0A2905
:10F0700000D3401C0F2900D3401C1844D10601D5F1
:10F08000C0F15A0091074FEAC27105D509B1B430F9
:10F0900005E0C0F1B40002E009B1C0F5B47080B27F
:10F0A0007047C16000680DF05AB900684FF0FF3238
:10F0B0000168C26001F15002904202D18268CA62C6
:10F0C00005E001F16002904201D182688A63006824
:10F0D0000DF045B910B50C4600206421C4E90C01BF
:10F0E000A063E062E06360642064A06494F8701040
:10F0F00021F03F0184F8701084F84C0004F15001B5
:10F10000204600F0A2F804F16001204600F09DF8CE
:10F11000082120460DF018FF102120460DF014FFA5
:10F1200020460022BDE81040114600F0CDB810B5D1
:10F130000C46002104F15000FEF720FE04F16000AF
:10F14000BDE810400021FEF719BE00002DE9F04196
:10F150000D462F480BF063FC01284FD1284607F0DD
:10F16000D9F80446284607F0D9F88046182C0AD06A
:10F17000012C45D0082C43D01A2C3FD12846BDE89D
:10F18000F041F9F749BA4FF400310AF0C2FF0446E2
:10F19000284607F00BF905460068A04200DD04464A
:10F1A000002140462C600CF05EFB074600214046E3
:10F1B0000CF07AFB0646002140460CF09CFB04460E
:10F1C000002140460CF022FBB74201DA394600E04C
:10F1D0003146844201DA224600E00246914205DAD5
:10F1E000B74201DA384604E0304602E0844200DAF1
:10F1F0002046002802DA2968081A2860BDE8F08154
:10F2000008F13C014046BDE8F0410DF0C3B80000F4
:10F21000FC12030890F8700000F00700704790F8A7
:10F22000701001F00701022901D0006B7047C16E18
:10F23000491C01D0806E7047806B7047C16D491CBE
:10F2400001D0806D7047C06A704708600020486038
:10F250008860401EC860704790F8701001F0070188
:10F2600001290AD1016B002907DA426B002A04DD6B
:10F27000806B884201D1012070470020704738B56B
:10F28000134690F8702002F00702022A1BD1D0E941
:10F290000C428A4201DD0D4600E01546AC4201DD1C
:10F2A000214602E08A4200DC1146C26A8A4200DA44
:10F2B0001146826B8A4206D0009300F1600300F190
:10F2C000380200F023F838BDF8B5C56A13468D4200
:10F2D0001AD0D0E90C428A4201DD0E4600E0164603
:10F2E000B44201DD214602E08A4200DC1146826B15
:10F2F0008A4200DD11468D4206D0009300F1500392
:10F3000000F12C0200F002F8F8BD0000F0B597B053
:10F3100007461C981C4616460D4668B3E068401C1C
:10F3200040D0A068C4E90105002118461560FEF729
:10F3300025FD6846FEF760FD21466846FEF7F6FDAE
:10F3400019496846FEF7DCFD4FF4807200216846DB
:10F35000FEF7E6FD15496846FEF7C3FD3846002175
:10F3600064220CF0E3FA01466846FEF7C1FD6846E8
:10F37000FEF7FEFD17B0F0BD00211846FEF7FEFCBB
:10F380004FF0FF30E060384635600CF0E8FF0021B8
:10F390002046FEF7F3FC17B021463846BDE8F040A2
:10F3A000FFF753BF3068BDE7A3F00008ABF00008DB
:10F3B00070B58C6C0D462CB1206C18B102F0BBFC02
:10F3C000002020642846BDE87040FCF7C6B8000065
:10F3D0002DE9FF4F088C85B0C0F30725E81F1E46B6
:10F3E0000C46039003280BD9102D09D0112D07D0FE
:10F3F0000F2D05D0122D03D0132D01D0142D1ED1A9
:10F40000D4F848805FEA08001AD0D8F800000190CC
:10F41000284601F091FC81460798FFF7F6FB8346EA
:10F42000207C01280FD00020824670686FF0604178
:10F43000C84231D10398032807D8102006E00020E5
:10F4400009B0BDE8F08F0C20EEE7284602900020BE
:10F45000009001235A46D8F84000029902F00BFEB2
:10F46000070013D1D8F8400020B102F064FC00205E
:10F47000C8F8400000200090012259465848029BDD
:10F4800002F018FC0700DAD0C8F84070079907C9E5
:10F4900086E80700F16006E0401C7060F068401CE0
:10F4A000F060D8F8407007997068D7F81080C96884
:10F4B0008842C4DC0399032946D80822B2FBF9F13B
:10F4C0003268B2FBF1F301FB132102910BFB09F14E
:10F4D0000123C91D03EBD1010391636B02FB09F208
:10F4E0000AEB8301238D9BB200FB031000EBD209D2
:10F4F000207C012810D0E068016901EB090600BFFB
:10F50000CDE900685B46216B2846029AF8F74AF875
:10F51000207C012814D050E0039809F067FF060012
:10F520000DD00020009032464946039B0198FCF71D
:10F5300031F80028E4D0304607F07EF97FE7FEE797
:10F54000304607F079F938E0102D39D0112D37D039
:10F550000F2D35D0122D33D0132D31D0142DEDD1E8
:10F5600039894FF000098DB2218D2B468AB200FBFC
:10F5700002A031684246090100EBD101CDF80090AC
:10F580000198FCF707F80028D8D1616A0C200A0C12
:10F59000218D8BB202FB03007268C1F34E0102FBA6
:10F5A0000100316808EB050201445B46CDF800908C
:10F5B0000198FBF7EFFF0028C0D10120E7623FE789
:10F5C0000BFB09F1CB08218D8AB200FB02A0316848
:10F5D000424601FB09F100EBD10100200090E7E772
:10F5E000D84F002038B50D46C968287C144620B194
:10F5F000012807D0022825D016E00C22204609F069
:10F600006BFF24E0084607F071F915A10FF078FFB1
:10F6100050B96B460C22214605F1140007F0CDF9D4
:10F6200010B900980C2801D0002038BD2078192886
:10F6300002D06070192020702068202141EA10401B
:10F64000608004E00120A080E0800E2060702068CF
:10F65000C1B2192902D0400C40006080012038BDA1
:10F6600062696E0010B507F0E3FD040011D009498E
:10F6700007F0D0FE0849204607F0CEFE0749204695
:10F6800007F0C6FE0649204607F0C0FE05A020612F
:10F6900010BDFEE7E5F50008A9F60008D1F3000863
:10F6A000B1F3000842494E002DE9F04782464FF081
:10F6B0000008087C90B00C464546C146012801D0A0
:10F6C00088B34FE0E06807F011F95EA10FF018FF72
:10F6D00098B92046FCF776F906000ED00C20A664F7
:10F6E00009F084FE070007D00222E16807F01AF94A
:10F6F00038B1384607F0A0F89FE0002010B0BDE810
:10F70000F0873760216AC1F30720090C090729D463
:10F71000C11F032923D90B3803285ED82146504640
:10F72000F7F75CFE04E007E021465046F7F7E0FEFD
:10F730008046012816D150E0E66830690028DDD007
:10F740003088C0F30727206A000C00070AD4F81F8E
:10F7500003280CD80846FCF735F90028CED0E0790C
:10F760000028E1D02046FBF7F8FE4046C6E7A7F1A7
:10F770000B000328084604D8FCF724F90028BDD064
:10F78000CCE7FCF71FF93168090CC90601D53546ED
:10F7900009E000F1240530890004000C09D031464D
:10F7A000284602F015FBE56228890004000C11D000
:10F7B00012E01822314608A8F0F7C0FF384601F0E1
:10F7C000BBFA099989B24843C01DC008ADF82800AA
:10F7D00008A9E5E7208D28810125E76A5FB339464E
:10F7E000204607F0BFFD060027D0BE4208D02046C5
:10F7F000FBF7B3FE2046FCF7E5F8C661E66201E0E0
:10F80000E062C5B9A079B0B907F08AFC98B1207C54
:10F810008DF81000E0680390E26A02A9D0680290B7
:10F820005046A36C07F0CAFC38B160642046FCF770
:10F83000C9F8C0F81C90012060E72046FBF78DFE58
:10F840005BE7000062696E0010B50C46102120468F
:10F850000DF07AFB2046BDE810404FF480610AF0BD
:10F8600070B9000010B5014603480AF0D1FC044607
:10F870000AF034FD204610BD2013030870B504467D
:10F88000806B154688420FD9606B30F81120AA436F
:10F8900020F811202046FDF7BBFC680504D5204662
:10F8A000BDE870400DF0A6BA70BD70B50E460546B5
:10F8B000002405E0324621462846FFF7DFFF641C9E
:10F8C000A86BA042F6D870BD084600214FF6FF7223
:10F8D0008163C0E90F1201634163C1624164014960
:10F8E00000F0ECBA4413030810B5014603480AF0CF
:10F8F0008FFC04460AF0F2FC204610BD601303089A
:10F9000010B50C46086B06F097FF606B06F094FF8D
:10F9100000202063606310BD2DE9FE4F8A46FE483B
:10F920000BF07DF8012833D1504606F0F3FC064673
:10F93000504606F0F3FC00270446182E02D02F2E66
:10F9400048D02BE0E06BA146002821D00025D9F853
:10F950002C800FE0D9F8340030F81500400508D5A8
:10F96000E06BB8B120460BF0FDF8E16BB0FBF1F1B4
:10F9700011E06D1C58F82500002809D0E7A10FF010
:10F98000BFFD002804D058F8250000780028E1D1F8
:10F99000BDE8FE8F0021504606F089FD2E2E1DD0B9
:10F9A0004FF6FF75012E1BD0022E59D0082E69D0BC
:10F9B000062E7CD0032E7BD0102E7AD0112EE7D0CD
:10F9C000122EE5D00E2E75D01A2EE1D15046F9F741
:10F9D0003DFDDDE7E16A00F071FAD9E72046F9E77D
:10F9E000504606F09DFC06462046216CFDF710FCB3
:10F9F00008F002F808F04AF8012801D003281AD1CB
:10FA00006946304608F016F869462046FBF708FEBE
:10FA10002564A842BCD0616B31F81010C1F380128C
:10FA2000002AB5D1C1F300110029B1D101462064EB
:10FA30002046FDF7EDFB206CA842A9D0616B31F8A0
:10FA40001000C0F340210029A2D1C0F3802166E05C
:10FA5000206C029002AA202120460DF030FD97E78D
:10FA6000206CA84294D0504606F05AFC694607F034
:10FA7000E1FF69462046FBF7D3FD216C814287D028
:10FA8000204659E0216CA9423CD0626B32F811004B
:10FA9000C0F3C013CBB1C0F38013B3B9C30503D512
:10FAA00094F84430DB0718D040F4807003E02EE077
:10FAB00040E044E08DE022F8110094F84400C007D3
:10FAC00003D02046216C12F010F9216C606B30F8E5
:10FAD0001100C0F3402131B902E020F48070E5E765
:10FAE000C0F3802171B1C0F3801159B9C0F3001087
:10FAF00040B9206C029002AA202120460DF0DFFCC4
:10FB00000128ACD12046216CFDF782FB40E7206C38
:10FB1000A842A4D0616B31F81000C0F34011002955
:10FB20009DD1C0F38011002999D1C0F300100028A5
:10FB30008ED02DE72046216CFDF76AFB47E0A06BD5
:10FB400000288CD0504606F0EBFB074607F09EFFDE
:10FB500006462FB9002007F061FF07F097FF064621
:10FB600020460BF04EF807F079F9216CA942CDD16F
:10FB7000022E02D0042E2AD148B394F8441000205B
:10FB8000A26BC90701D113E0401C82421DD9616BF1
:10FB900031F81010C1F30013002BF5D1C1F380131D
:10FBA000002BF1D1C1F300210029EDD00DE0401C64
:10FBB00082420AD9616B31F81010C1F30013002B97
:10FBC000F5D1C1F380110029F1D12064E0E625646C
:10FBD000DEE62046216CFDF71BFB504606F0C9FB14
:10FBE000132813D0142835D004264FF00809122802
:10FBF00052D0112886D1002120460BF025FE8046E8
:10FC0000206CA84274D12764626BA3E0206CA842E8
:10FC100002D13846276401E0401C2064A36B98425F
:10FC200000D32764666B226C07E0491C216499426B
:10FC300000D32764206C90426DD0216C36F81100FF
:10FC4000C0F3001CBCF1000FEFD1C0F380100028FE
:10FC5000EBD157E7206CA84201D1276400E000B93E
:10FC6000A06B401E20640346626B09E019B1491E77
:10FC70000846216402E0A06B401E2064984267D0D1
:10FC8000216C32F81100C0F30016002EEED1C0F343
:10FC900080100028EAD135E7002120460BF0D4FD82
:10FCA0008046206CA84213D12764626B04E0491C93
:10FCB0002164A06B81424BD2216C32F81100C0F359
:10FCC0000013002BF3D1C0F380100028EFD119E707
:10FCD000216B01EB0010FEF798FF0346206C216BAF
:10FCE000024601EB00152D6805EB630CA36B25E0C4
:10FCF0003CE000BF06EB001506EB02174D59CF594B
:10FD0000BD421ADD01EB00152D68654515DC09EBD8
:10FD100000154F5904E01BE0601303080A000000BF
:10FD200007EB0805654508DB656B35F81050C5F332
:10FD3000801717B9C5F3001515B1401C8342D9D8F7
:10FD4000834245D8DEE6491C2164A06B814201D381
:10FD50002564D7E6216C32F81100C0F30013002BA4
:10FD6000F1D1C0F380100028EDD1CBE6216B01EB7F
:10FD70000010FEF74AFF226C216B01EB02131B6897
:10FD800003EB600310B21EE006EB001506EB021752
:10FD90004D59CF59BD4214DA01EB00152F68A7EB7E
:10FDA00008059D420DDC09EB00154D599D4208DB0D
:10FDB000656B35F81050C5F3801717B9C5F30015FA
:10FDC00025B1401E00B20028DEDA9BE60028B9DB30
:10FDD000206497E62DE9F0410F46A1F57F41FF39F8
:10FDE00015D00546806BB84211D30024264609E0A1
:10FDF000E86A641C09A150F82400761C0FF080FB0F
:10FE000000B9641CBE42F3D1A86BB04202D10020FD
:10FE1000BDE8F081E86A50F82400F9E70A00000024
:10FE2000006C7047836B8B4204D9406B30F8110033
:10FE3000824301D0002070470120704770B504460E
:10FE4000806B0E461546B0421BD994F84400C0079B
:10FE500006D0E80504D54FF480712046FFF725FD54
:10FE6000606B30F81610294320F8161031462046F2
:10FE7000FDF7CEF9680504D52046BDE870400CF0CA
:10FE8000B9BF70BD70B50E460546002405E0324688
:10FE900021462846FFF7D2FF641CA86BA042F6D883
:10FEA00070BD10B50446806B4200606B09F014FB16
:10FEB0002046E16ABDE81040AFF300802DE9F04F25
:10FEC00097B00D0004467DD0F5F72CFF00212722C6
:10FED0002046E5620BF02AFDC0B200271290394699
:10FEE00020460BF0C3FC0646394620460BF0E6FBE5
:10FEF0008046394620460BF0CFFB400700D54644EC
:10FF0000002080460146274620460A960BF0F6FC64
:10FF10000646414638460BF0D1FB814641463846FD
:10FF20000BF0BAFB800700D54E44002120460F9607
:10FF30000BF0D8FC0390002120460BF085FC0890C4
:10FF400020460AF020FE069020460AF00BFEE16BE8
:10FF50000027C1F101020399A94601FB020010909C
:10FF600038467BE04FF0000B5D4607E0606B791987
:10FF700030F81100FBF709FC83446D1C59F825008B
:10FF800040B13FA10FF0BCFA20B159F8250000782C
:10FF90000028EBD14DB31098E16B00FB08F0B0FBEB
:10FFA000F1F20F981318039A08FB02300E90109884
:10FFB00008F101025043B0FBF1F0039B0F9908FBDD
:10FFC000031100E058E0401E084414900899069878
:10FFD000C5F1010201FB02000D90002801DA0020AA
:10FFE0000D904FF0000A564630E009F1040032E06F
:10FFF000606B30F81700FBF7C8FB01460D9800FB5B
:020000040801F1
:100000000AF0B0FBFBF208988A4406FB00200D9A28
:100010000AFB02F1B1FBFBF1089A491E06FB021232
:100020001299012904D101460698801A069A521A9B
:100030000A9901440A98131814980090206B0E9A9C
:1000400000EB0710FEF745FF761C7F1CAE42CFD3B6
:1000500009EB8500001D814608F10100E16B804637
:1000600041453FF67FAF20460CF0C4FE17B0204656
:10007000BDE8F04F0CF073B917B0BDE8F08F000089
:100080000A00000070B50446806B0D46A84203D8F4
:10009000A5F57F40FF380AD12046216CFDF7B8F85E
:1000A000204629462564BDE87040FDF7B1B870BD13
:1000B0002DE9F04117460E46040017D0BEB104F1F9
:1000C0001C00054609F028FDE06888B120683A4622
:1000D0003146C36820469847040001D000F056F826
:1000E000284609F01BFD2046BDE8F081FEE7FEE74B
:1000F000284609F013FD0020F6E72DE9F0411746E8
:100100000E46040016D0B6B104F11C00054609F0F5
:1001100003FDA06880B13A4631462046F6F70BF958
:10012000040001D000F032F8284609F0F7FC204620
:10013000BDE8F081FEE7FEE7284609F0EFFC00206D
:10014000F6E72DE9F0470546DDE9089A00681E4606
:10015000174688468047040012D004F10C010020A5
:10016000A76081E84106C4E90058696820468847CD
:1001700038B104F11C0009F0CDFC2046BDE8F08741
:10018000FEE7204606F058FB0020F7E700B5020026
:1001900006D000F027F810465DF804EB00F013B825
:1001A000FEE730B14168491E416001D50021416040
:1001B0007047FEE710B528B100F005F8BDE8104023
:1001C00006F03ABBFEE710B18168401A7047FEE7BF
:1001D00008B108447047FEE708B140687047FEE781
:1001E0001030704718B14168491C41607047FEE704
:1001F00030B131B101600021C0E9011201737047D3
:10020000FEE7FEE708B1007B7047FEE720B14168DA
:10021000002902D0FFF7C5BFFEE7704780680028BD
:1002200000D0012070472DE9F04116460D0004462C
:100230000DD004F11C00074609F06EFC314628463B
:10024000FFF7E4FF2846FFF7C7FF08B10DE0FEE720
:100250002846FFF7D7FF40B12846FFF7B4FFA26951
:10026000314690472846FFF7A5FF3846BDE8F041E4
:1002700009F054BC002800D0016270472DE9F0411C
:100280000F460C464FF4FD612186012084F83200B0
:1002900084F83300A18684F8360084F83700002003
:1002A000A063E06304F221104FF45272002109F0C0
:1002B000CEF900210846324B782506E028B14207E6
:1002C000B2F1604F08D0072808D253F8202000BFB1
:1002D00004EB800632640EE02AA2F9E701EB81020A
:1002E00004EB820204EB800682F8215102F2211213
:1002F000491CC9B23264401CC0B23828DED322A0E7
:10030000C4F81C013846FFF7EFFA04F14001E0623F
:10031000FFF7D4FD54F82C0F4FF40871FFF7B2FD2E
:1003200000231F221949206809F0FAFB64200DF010
:100330005FFD014620680DF091FA4FF4042120681A
:1003400009F0FFFB012138460DF0FBF80121206880
:100350000DF003F90022022138460DF066FA94F9F7
:100360000A202189384600F015F894F9073094F9ED
:100370000620A1883846BDE8F04100F0ABB8000087
:10038000280100200A00000000000000D1AB000896
:10039000343070472DE9F05F044688B2A08655B22C
:1003A00084F83650012184F8371082464021E06AF3
:1003B000FFF77BFA002640223146E06AFFF73EFD58
:1003C000761C072EF7D3564629463046FBF734FDF8
:1003D0008346012229463046FBF7D0FA06460746F7
:1003E0004FF001080BEB060910E000BF07EB870197
:1003F00004EB8100434636A2142100F221100EF0D6
:1004000033FE08F1010000F0FF087F1CB945EDD86C
:10041000691E5046FBF710FD0025801B401CC7B22B
:1004200013E000BF05EB850104EB81003B4628A2E9
:10043000142100F221100EF017FE4022E91DE06A9F
:10044000FFF7FCFC7F1CFFB26D1CB542EAD306EB44
:100450000B05012713E000BF05EB850104EB8100CC
:100460003B461BA2142100F221100EF0FDFD40229C
:10047000E91DE06AFFF7E2FC7F1CFFB26D1C2A2D2C
:10048000EAD32046FCF7CDF8E06AFFF7C9FCA0F5F7
:100490007F41FF3903D0F11DE06AFFF7F3FD2046ED
:1004A0000BF05DFF20460AF00FFB064600250BE02F
:1004B000294620460AF0C9FAE16A814203D0224661
:1004C00020210CF0FCFF6D1CB542F1D3BDE8F09F7C
:1004D00025640000018680F8322080F83330FCF774
:1004E000A0B810B50C46142104F12C0008F09BFEB6
:1004F000182104F1380008F096FE00206064606561
:10050000A064A0656420E064E065206520660320A7
:10051000A0660520E0660A2020676FF00040606654
:1005200094F8740020F00700401C20F0080084F8C4
:10053000740010BD70B50C4601F12C0617E000BF29
:1005400008F054FE050012D0287C400702D46868E9
:1005500006F072F9287C800702D4286806F06CF94E
:100560002946304608F00CFF284606F065F9206B56
:1005700000283046E4D108F019FE04F1380509E0FE
:1005800008F034FE06460146284608F0F9FE3046DB
:1005900006F052F9E06B00282846F1D1BDE8704022
:1005A00008F004BE2DE9FC410E4649480AF037FA2E
:1005B000012864D1304605F0ADFE0546304605F011
:1005C000ADFE0446012D11D0082D5AD01A2D56D15A
:1005D000304605F0DAFE054601462046F7F709FEEB
:1005E00004F12C0008F094FE98B36AE007F004FAD6
:1005F000694607F01FFA009960692546081A0090BD
:1006000028460AF0D5FB0099471828460AF0BBFA9D
:100610000646002128460BF02CF9381A4FF0000747
:100620001CD4B04202DD2F6F7F1E17E095F87410C6
:1006300001F00701012902D002290BD00EE0296F39
:10064000491E414306EBD67001EB6000B0FBF6F7A4
:1006500004E01DE0296F4143B1FBF6F7606EB8423C
:100660000DD039462046FCF72BFE2046616EFCF784
:1006700027FE20460022202167660CF020FFBDE8FF
:10068000FC81616EFCF71CFE6FF000406066F6E7CF
:1006900094F8740000F00700012804D0022807D065
:1006A00003280AD00DE029462046F9F74AFF08E062
:1006B00029462046F9F74DFE03E029462046FAF781
:1006C00007F929462046BDE8FC41F7F7ADBC00001C
:1006D000841303082DE9F04F8BB017460E46050032
:1006E0001C4609D04EB1286FB84207D800202060C0
:1006F00058600BB0BDE8F08FFEE7FEE728460AF031
:1007000042FA804628460AF02DFA059095F87400C2
:1007100000F00700012804D0032809D0022817D0D0
:100720005EE0296F08FB07F0491EB0FBF1F056E0D0
:10073000CDF80080317C3068C1F3C00205EB820146
:1007400050F82700CA6D496D002308F087FE46E087
:1007500005F12C000490069008F04CFD82464FF401
:10076000A02128460BF073F80890002128460BF0D2
:100770006EF801460290286F4FF0000BC0F10103A4
:1007800003FB0181B1FBF0F9A8EB09017943401E9D
:10079000B1FBF0F02060069808F041FD06E0B142A0
:1007A00006D00BF1010B049808F036FD0100F6D1DC
:1007B0000299CAF1010308EB0100296F7843B0FBED
:1007C000F1F009FB0BF1B1FBFAF10144089800FBD1
:1007D0000392B2FBFAF000EBD07001EB60002060F6
:1007E000002128460AF06DFF8046002128460BF0C4
:1007F00040F8216840440844206028460AF0D8FAAE
:100800002168081A206095F87400000701D4F06888
:1008100000E00020C119286F059BB1FBF0F200FB3E
:100820001210716851F82000317CC1F3001205EB01
:1008300082014A6CC96C801A5843891A90FBF1F006
:10084000181A6060002128460BF05BF8616840448C
:100850000844606028460AF06DFB6168081A606011
:1008600047E7000010B50CA0C86201200C460863E1
:100870000221204609F065F90821204609F061F9B6
:100880004FF48061204609F05CF92046BDE8104035
:1008900010210CF059BB0000436865636B20626F48
:1008A0007800000010B591F830000C46C00704D164
:1008B000E06A05F0C1FF0020E06210BD2DE9F04FB5
:1008C000CFB0054605F02AFD0446284605F05DFD3B
:1008D0004390002120460BF028F93B9005F0A1FF42
:1008E00005462046002127220BF020F8C0B201283F
:1008F00014D000272046002130220BF017F80646BE
:10090000002120460BF000F800EB06084FF0000134
:1009100020462FB10AF0CEFF064604E00127E9E7A2
:100920000AF0AAFF0644002120460AF093FF8346FE
:100930004FF4003120460AF09FFF82464FF4003109
:1009400020460AF0B7FF81464FF4003120460AF0F6
:10095000DBFF40904FF4003120460AF05DFF02902B
:10096000204668224FF400310AF0E0FF0190204653
:1009700069224FF400310AF0D9FF00901EA802F05E
:10098000F5FE1EAA4FF4003120460BF05AFB57B17A
:10099000E069801B411BA1EB0A010590A1EB090056
:1009A000401C039008E060693044421903900AEB50
:1009B00009001044401E0590A16901EB080042198E
:1009C00004900299409808441044401E06900398F1
:1009D000459004984690059847900698DDE90021D7
:1009E000489045A8FEF716F945AA1EA9439802F0BB
:1009F000A7FC002120460BF0BCF80646002120464B
:100A00000BF0A8F8034600206FF060410096CDE996
:100A10000110E16A49A83B9A0FF00CFD09A801F00A
:100A200065FE09AA002120460BF04DFAE06A1090FD
:100A300003A8FEF7DBF8401B00EBD07040103FB17D
:100A4000039AA2EB0B01499A3E91891A3C9106E068
:100A5000059A02EB0B01499A3C9111443E91A2691F
:100A6000404410444A993D9008443F903CAA09A94B
:100A7000439801F00AFE4FB0BDE8F08F2DE9F04F2A
:100A800085B00F463B4809F0CAFF012861D13846BE
:100A900005F040FC0546384605F040FC04464FF49E
:100AA0000036312D09D0182D56D01A2D51D105B050
:100AB0003846BDE8F04FFFF701BF384605F076FC39
:100AC0000546002120460BF030F8814605F0A9FECE
:100AD0000746002120460BF04CF8804600212046B6
:100AE0000BF038F800216FF06042CDF80080CDE9BE
:100AF000012103464A4603A8E16A0FF09BFC00214E
:100B000020460AF0A7FE8346314620460AF0B4FE8E
:100B10008146314620460AF0CDFE824631462046C7
:100B20000AF0F2FE8046314620460AF075FE014684
:100B300007EB0800084407EB0902039902EB0A03DC
:100B40005A1802EB0B0129600499884200DC084620
:100B5000686005B0BDE8F08F384605F027FC054613
:100B60003146204609F0D5FA2968814200DD084661
:100B70002860EEE7A8130308F0B5184D0446C1F34A
:100B800041706E1064274FF0805C012809D121F07C
:100B9000C040A84205DC604500DB301A584390FB9A
:100BA000F7F1C2F34170012809D122F0C040A842F8
:100BB00005DC604500DB301A584390FBF7F29442A5
:100BC00001DA204600E01046884201DA0846F0BD0E
:100BD000944201DA2046F0BD1046F0BDFEFFFF1F33
:100BE000F0B5184D0446C1F341706E1064274FF004
:100BF000805C012809D121F0C040A84205DC604595
:100C000000DB301A584390FBF7F1C2F34170012822
:100C100009D122F0C040A84205DC604500DB301A53
:100C2000584390FBF7F2944201DA204600E0104668
:100C3000884201DA0846F0BD944201DA2046F0BD50
:100C40001046F0BDFEFFFF1FFF2916D0B1B102888C
:100C5000D30A13FB01F31B0A63F3CF22C2F345133C
:100C600013FB01F31B0A63F34A1202F01F0313FB89
:100C700001F1090A61F30402028070470222002197
:100C800008F0E5BC10B50346FF2A13D09AB18B4299
:100C900010D041EA0140121D0849D40843EA03423A
:100CA00008400A40121A624300EB5210084040EA22
:100CB000104080B210BD084610BD00001FF8E007CC
:100CC000002208B51146104600F077F80090BDF8F4
:100CD00000009DF8021040EA014008BDC0F3074142
:100CE000C2B201EB410101EB8201C0F307200844CD
:100CF000C0F3C700704738B50C460546FFF7E0FF64
:100D00002246294600F064F80090BDF800009DF8E6
:100D1000021040EA014038BD10B50C4600F0A2F8C0
:100D20000346204600F09EF8834201D1012010BD09
:100D3000002010BD01607047801F102817D2DFE827
:100D400000F00E080A0C0E080A0C0E1214141012F1
:100D500010100120704702207047042070470820BF
:100D600070471020704718207047202070470020DF
:100D7000704700B5FFF7E0FFC01DC00800BDC01FF1
:100D80000F280BD2DFE800F0080808080808080858
:100D90000A080A0A08080800012070470020704766
:100DA00008B5020A8DF80120C0F307418DF8000054
:100DB000BDF8000040EA014008BD08B503468DF8C3
:100DC00001108DF80020BDF8000040EA034008BD86
:100DD00078B5C1F30744C2F1FF0314FB03F4C0F379
:100DE000074515FB024404EBC41505EBC434C4F3FA
:100DF000C754C1F3072515FB03F5C0F3072616FBFF
:100E0000025505EBC51606EBC535ED0D8DF8015005
:100E1000C9B211FB03F1C0B210FB021000EBC0110C
:100E200001EBC030C00D8DF80000BDF8000040EAB5
:100E3000044078BDC178FF290FD079B1827812FBC8
:100E400001F2120A8270427812FB01F2120A427019
:100E5000027812FB01F1090A017070470422002197
:100E600008F0F5BBC0F30721C0F30742090201EB0C
:100E70000241C0B208447047010C01F0F8010902B8
:100E8000020A02F0FC0201EBC201C0B201EBD00089
:100E900080B27047FF2208B511461046FFF78DFF5C
:100EA0000090BDF800009DF8021040EA014008BD26
:100EB0002DE9FC5F05000C9C74D04FF48067BD42A7
:100EC00070D001EB4108581A00EB4001A1EB080972
:100ED000C8F58061A01AA1EB090B02EB420A00EBF6
:100EE0004001A1EB0A00CAF580610090081A2C4667
:100EF0000026019043464A4659462046F6F7FFFB36
:100F0000401B002801DD014600E04142012940DD8F
:100F10000BFB04F101EB4101891201EB4901614333
:100F200008EBA122002A01DD114600E0514201290F
:100F30000CDDC117890241EA90518002D317EFF707
:100F4000F8FA18B1241A761C082ED3DB00262C00E0
:100F500001D534461DE0BC4201DD3C4619E0434664
:100F60004A4659462046F6F7CAFB411B002900DCD9
:100F7000291A01290DDD854201DD264600E02746BC
:100F8000B81B00EBD07006EB6004B44201D0BE4247
:100F9000E5DBDDE9002102B053462046BDE8F05F05
:100FA000F6F7ADBBBDE8FC9F18B100F5387005F051
:100FB00093B9FEE72DE9F843DFF8788107460E463E
:100FC00008F1040008F037F904007CD04FF44471B4
:100FD00008F06DFB4FF0FF302760C4E90160002589
:100FE000C4E903056561A06B40F48030A0638220F2
:100FF000A061122084F83B004C2008F01BFAC4F8D2
:10100000A802011E76D0D4F8AC220AB1204690473F
:10101000D4F8A8027F1E761E4560D4F8A802856029
:10102000D4F8A802C760D4F8A8020661D4F8A812C0
:1010300094F83B0008750120C4F8600210F0C6F86F
:10104000C4F8FC02102104F5197008F0ECF8D8F887
:1010500014604546224621213748C8F8144010F054
:101060000BF9C4F8F80278B310F084F868B30FF005
:10107000F9FF00BFC4F8F402002009F0B9F9C4F880
:10108000C402002004F52E7409F0B2F9A06000201B
:1010900009F0AEF96060002009F0AAF92060E0686C
:1010A0000CF052F860680CF04FF820680CF04CF827
:1010B000022160680BF048FF022120680BF044FF1A
:1010C0000021E06802E014E015E015E00CF038FBC8
:1010D000002160680CF034FB002120680CF030FB2C
:1010E000A068A4F52E740BF03AF96E61A6B114E075
:1010F00000E0FEE7FEE7FEE700200CF063FE074697
:1011000005200CF05FFE01460C48009000233A4693
:1011100020460FF0B3FFADE76C610023352208498C
:101120002046FFF741FFD4F8F80210F0B2F920464C
:10113000BDE8F883E04E0020A9120108600D030805
:101140005176000818B907484069002809D0D0F83E
:10115000602209B1012101E04FF0FF311144C0F8D4
:1011600060127047E04E00200021016370470000CC
:1011700018B903484069002801D090F83B00704737
:10118000E04E00200148406970470000E04E00201A
:1011900010B90348406908B18069704782207047E0
:1011A000E04E002018B908484069002808D090F89F
:1011B000F01201F00701012903D0032901D00068D2
:1011C0007047406870470000E04E002018B903489F
:1011D0004069002801D0D0F8C4027047E04E0020DA
:1011E00018B903484069002801D0D0F8B802704708
:1011F000E04E002018B903484069002801D0D0F81B
:10120000BC027047E04E00200100034801D007F007
:10121000FFBF07F0EBBF0000E44E002018B9034801
:101220004069002801D0D0F8C0027047E04E00208D
:1012300018B903484069002801D0D0F8C8027047A7
:10124000E04E002008B902484069D0F8F402704727
:10125000E04E002018B908484069002808D090F8EE
:10126000F01201F00701012903D0032901D04068E1
:101270007047006870470000E04E0020006A0028B8
:1012800000D001207047000018B9064840690028C6
:1012900004D0D0F86002002801DD01207047002052
:1012A00070470000E04E00202DE9F041434C28B18A
:1012B000C168216110F0E6F8206902E0FFF762FFE3
:1012C0002061002878D0416A002975D00A69002A77
:1012D00072D0C96800296FD00022362100F070F862
:1012E0002069D0F8C0020CF00FFD2069D0F8C802C8
:1012F00008B10CF009FD2069D0F8C4020CF004FD1F
:101300002069D0F8BC020CF0FFFC2069D0F8B802CC
:101310000CF0FAFC20690026D0F8C012B9B10DF02B
:1013200043F812F0FDFB12F043F92069D0F85C128B
:1013300079B10022392100F043F82069FFF79EFFC0
:1013400048B3206990F8390001280BD023E0C0F899
:101350005C6203F0FDFE2069BDE8F0410022372108
:1013600000F02EB800254FF03C080FE005F50F7196
:10137000415C51B900F5197007F0ACFF226908EB28
:10138000051111448EC980E88E006D1C2069D0F8CB
:101390005C12A942EAD820694FF4007200213C3067
:1013A00008F055F920692022002100F50F7008F09F
:1013B0004EF92069CBE7FFE7BDE8F081E04E002061
:1013C00070B588B00E46044615461C21684608F0E4
:1013D0006EF9009404F538700194ADF808600122AC
:1013E00069460495044605F02FF8012804D100222F
:1013F0006946204605F028F808B070BD2DE9FF5F6A
:101400001F46DDF838B016465FEA0108814616D05F
:101410004846FFF7ADFE03904846FFF7C3FE8246FD
:101420004846FFF717FF0546BAF1000F08D03DB157
:101430004046039900F052FB404502D0FEE7FEE72C
:10144000FEE736B13046039900F048FBB04200D0C9
:10145000FEE75046039900F033FE0446BBF1000F4F
:1014600004D004FB05F0B84203D9FEE7B7FBF4F55E
:10147000B5B1CDE9004809F51C7002972A465146DE
:101480008046039B00F002FD8DE8D00009F5237033
:101490002A4651460446039B00F0F8FC16B900E0CA
:1014A000FEE7002422464146484600F007F804B013
:1014B00059464846BDE8F05F00F016B818B9044830
:1014C0004069002802D0C0E907124162704700005D
:1014D000E04E002018B903484069002800D081621E
:1014E00070470000E04E002018B90348406900280A
:1014F00001D080F839107047E04E002010B504008C
:1015000003D113484469002C21D0C4F8F412D4F854
:10151000D00204281BD1D4F8B402006809F0D4FA30
:10152000002814D1D4F8B402406809F0CDFA00289C
:101530000DD1D4F8B402806809F0C6FA002806D1AB
:10154000D4F8B4020068BDE810400FF07BBD10BDB8
:10155000E04E002000B501004FF000000ED0FFF774
:1015600017FE48435030B0F5A07F08DB0020FFF79E
:101570000FFE4843A021503090FBF1F000BD012048
:1015800000BD70B504460D46542007F053FF95E8A2
:101590004E0008304EC02ECD80E82E0004F1180118
:1015A00020302EC92EC0012140F84819A16B11B975
:1015B000A06370BD11460A68002AFBD1086070BDA7
:1015C0007FB5064691F83C000C4602282AD9206ACD
:1015D000002827D0D4E90901884223D0A08EE16AEF
:1015E000091A0091216B081A0190A18EE06A084443
:1015F000401E0290A18E206B0844401E0390694655
:101600003046FFF7BEFF0546402007F0EFFE4022C0
:101610002146E86407F060FF08202871294630461B
:1016200000F048FE7FBD38B504464022002108F096
:101630000EF801202062FF2084F83C00FFF740FBF9
:101640000090BDF80000A0839DF80200A077402024
:10165000606138BD2DE9FF5F8246DDE910E48B460D
:10166000DDE90E800AEB020C03F5B475CDF804C079
:101670001E460BEB020C9146AAEB0203ABEB0207F2
:10168000CDF808C0A84505D1C4E900370198A0608D
:10169000029815E14FF4B475AE4201DDA6F5B476BB
:1016A000A84501DDA8F5B478A9EB000100915FEA37
:1016B0000E0104D000EBD07045106D1C00E0002539
:1016C0005A2196FBF1F098FBF1F1C0B2C9B204289F
:1016D00000D10320042900D10321884279D1464555
:1016E00077DC38B301284AD0022874D003286ED1A1
:1016F00006F15A0000B20FF0FBFF009948430AEBD5
:10170000E030401B206030B20FF0F2FF00FB09F028
:101710000BEBE030401B606008F15A0000B20FF0A4
:10172000E7FF00FB09F00AEBE0302844A0600FFA65
:1017300088F021E130B20FF0DBFF00995A364843C0
:101740000BEBE030401B606030B20FF0D1FF00FBCC
:1017500009F00AEBE0302844A0600FFA88F00FF09F
:10176000C7FF00FB09F00BEBE0302844E06008F114
:101770005A0000B20FF0BCFF0099484323E030B29A
:101780000FF0B6FF00FB09F00BEBE03028445A36AF
:10179000E06030B20FF0ACFF009948430AEBE03054
:1017A0002844A0600FFA88F00FF0A2FF0099484388
:1017B0000BEBE030401B606008F15A0000B20FF004
:1017C00097FF00FB09F00AEBE030401B2060BDE80A
:1017D000FF9F2AE0FFE706F15A0000B20FF088FFF2
:1017E00000FB09F00AEBE030401B206030B20FF044
:1017F0007FFF009948430BEBE0302844E0600FFA8C
:1018000088F00FF075FF00FB09F00BEBE030401B98
:10181000606008F15A0000B20FF06AFF0099484377
:101820000AEBE0302844A060D1E7C8B1012849D0D4
:10183000022872D003287FF427AF0029FBD108F1DA
:101840005A0000B203900FF053FF074606F15A000A
:1018500000B202900FF04CFF87427CDA039893E0CD
:101860000129E8D108F15A0000B20FF041FF00FB56
:1018700009F00AEBE030401B20600FFA88F001907D
:101880000FF036FF074630B280460FF031FF874237
:1018900001DA019800E040460FF02AFF00995A361D
:1018A00048430BEBE030401B606030B20FF020FF8C
:1018B00000FB09F00AEBE0302844A06002982844BD
:1018C000E06084E70229B6D1581B20600FFA88F047
:1018D0000FF00EFF00FB09F00BEBE030401B6060E7
:1018E00006F15A0000B201900FF002FF074608F11E
:1018F0005A0000B280460FF0FBFE874201DD0198DE
:1019000000E040460FF0F4FE009948430AEBE03057
:101910002844A06030B24DE0FFE703298BD106F1E7
:101920005A0000B20FF0E4FE00FB09F00AEBE030D1
:10193000401B2060781B606008F15A0000B20FF075
:10194000D7FE00FB09F00AEBE0302844A0600FFA54
:1019500088F0804600E016E00FF0CAFE009900FB18
:1019600001F730B206460FF0C3FE009948438742A4
:1019700001DD404600E030460FF0BAFE00994843D2
:101980000BEBE0309BE702980FF0B2FE0099484362
:101990000AEBE030401B206030B20FF0A9FE00FBE4
:1019A00009F00BEBE030401B606001982844A06018
:1019B0000FFA88F00FF09CFE00FB09F0E0E710B58D
:1019C00004462C2107F07BFEFF2084F828000F201E
:1019D00084F829002C20606110BD2DE9F0470D46E8
:1019E00004000AD0206948B1606887B2060C2068FC
:1019F000010C890626D515B107E0FEE7FEE7C0F326
:101A00000721384600F05CFB0546208980B2A842D9
:101A100002D10120BDE8F0872088C0F30720FFF73E
:101A20008BF97843C01D4FEAD00A55450AD3208868
:101A30002B46C0F3072231463846F3F744FFE168EE
:101A4000814201D20020E5E72088C0F30720072863
:101A500017D0082817D0092817D00A2817D0002037
:101A6000218980008BB2AB4223D2711E22690027EC
:101A700003FB012305FB012103EB00090844804619
:101A800014E00220ECE70420EAE71020E8E74FF436
:101A90008070E5E75246494607F0B8FD20897F1C73
:101AA00081B2A8EB0500A9EB01098046B742F1D34A
:101AB00012E02169002708448146C8460AE05246E0
:101AC000494607F0A3FDA16819FA81F908EB050062
:101AD00080467F1CB742F2D325819AE70A46014629
:101AE000014800F003B80000A84F002030B483681C
:101AF0000C461BB1204630BC1146184730BC0020B4
:101B00007047F0B589B0040035D0208986B289B31A
:101B1000002004900590A0884FF0FF3280B2401E54
:101B20000690606802EB1040079004AA6846FDF733
:101B30007EF800282AD06846FDF767F8002825DDE2
:101B40006846FDF753F8002820DDDDE90012204645
:101B500000F056F905462088C0F30720FFF7ECF89F
:101B600004466846FDF751F800FB04F1C91DCF108B
:101B7000019C13E000E0FEE700221146204600F041
:101B80003FF96168090C714307F095FD09B0F0BD9C
:101B90003946284607F08FFD3544641C0398A0425F
:101BA000F6DAF3E72DE9F05F044600880D46C0F34E
:101BB000072110881F46C0F307209146814200D0BC
:101BC000FEE72DB12846FDF720F8064617B117E0CD
:101BD000A08886B22088C0F30720C11F03290ED831
:101BE000072813D0082813D0092813D00A2813D0A7
:101BF00000208200D9F81010206907F06DFC77B141
